:06000000D1EF06F0120032
:0600080004EF08F01200F5
:100018000CEF08F012001DEE00F02DEE00F0F86A6B
:06002800EDEF06F01200EE
:1000300000003E0E006E016AFC0E026E036A046A46
:10004000076808680968066A1200D9CFE6FFE1CFA1
:10005000D9FFE65204501EE1040108BF1AD0400E39
:10006000E66E600EE66E000EE66E95EC06F0E5526A
:10007000E552E552010E046EDF6A400EDF5C09E2D4
:10008000DF50EA6AA00FE96E000EEA22EF6ADF2A6B
:10009000F4D717D100016051080A01E10DD10F0A10
:1000A00001E1D3D0010A01E1CAD0030A67E0010AE5
:1000B00058E0070A44E0010A01E003D10001020E02
:1000C000A06F00013A0EA16F0001010EA26F0001A6
:1000D000010EA36F0001A46B100EA56FA66BA76B9A
:1000E00001C0A8F002C0A9F003C0AAF0100E0001E0
:1000F000A95F000E0001AA5B0001AB6B0001030EBB
:10010000AC6F0001F80EAD6FAE69AF6BB06B000164
:10011000080EB16FB26BB36BB46B0001B56904012B
:100120000CBF0CD0400EE66EA00EE66E000EE66E22
:100130005BEC06F0E552E552E552046AC2D00001DC
:10014000615107E13F0E006EF80E016E0268036A0E
:1001500006D03E0E006E016AFC0E026E036A046A4F
:10016000B0D0040E056E0028055C06E20400AED88F
:10017000F0EC04F0052AF7D7046AA3D0E868071862
:1001800005E1E868081802E1E868091806E161C0BD
:1001900007F062C008F063C009F007500001611960
:1001A00008E108500001621904E1095000016319D7
:1001B00000E143E1DF6A00016551DF5C3EE2000ED1
:1001C000075C100E0858000E09582CE300285B6EDF
:1001D0005C6A0A0ED8905B365C36E806FBE15D6A25
:1001E0005CBE5D685B50075C5C5008585D50095808
:1001F00019E23A0E0001D8806555DF24EA6A660FDD
:10020000E96E000EEA22EF50E66E0650E96EEA6AE9
:10021000E9BEEA680A0EE926000EEA22E552E75036
:10022000EF6E062A072A000E0822000E09223A0E57
:10023000065C01E15ED8DF2ABED7046A42D059D8F5
:10024000076808680968046A3CD00001070EA06FBF
:1002500061C0A1F062C0A2F063C0A3F064C0A4F0CA
:1002600065C0A5F061C0F6FF62C0F7FF63C0F8FF8C
:10027000DF6A00016551DF5C0FE209003A0E000100
:10028000D8806555DF24EA6AA60FE96E000EEA22DF
:10029000F5CFEFFFDF2AEDD704010CBF0CD0400EE5
:1002A000E66EA00EE66E000EE66E5BEC06F0E55222
:1002B000E552E552046A05D06592656A68D8FF0088
:1002C00000D0E552E552E7CFD9FF1200F66A05509B
:1002D000F76EF86AD890F736F836F736F836140E17
:1002E000A66EF29E550EA76EAA0EA76EA682A694C3
:1002F0001200D9CFE6FFE1CFD9FFE652DF6A000E48
:10030000E76E0618E8AE02D0063403D0E750D88076
:10031000065436E206505B6E5C6A5D6A5BAE02D0E4
:100320005C685D685B50075CF66E5C500858F76E61
:100330005D500958F86EDF50EA6A0A0FE96E000E48
:10034000EA22EF50F56E0D00DF2A0606065009E09E
:10035000DF50EA6A0A0FE96E000EEA22EF50F56EEE
:1003600001D0F5680C00DF2A240EA66EF29E550E11
:10037000A76EAA0EA76EA682065001E00606BFD79A
:10038000A694066AE552E552E7CFD9FF1200D9CF0D
:10039000E6FFE1CFD9FFE652DF6AFF0EDF5C0AE23B
:1003A000E868E85005E0E80600D000D000D0F9D7B2
:1003B000DF2AF3D7E552E552E7CFD9FF1200D9CFB4
:1003C000E6FFE1CFD9FFE652645032E162960401C4
:1003D00000513C0BE842E8420D0828E1180E0219D2
:1003E00023E1040E031920E1100E026F040E036FC7
:1003F000DF6ADF505B6E5C6A080E5B5C000E5C5867
:1004000013E2DF50EA6A180FE96E040EEA22EF5099
:10041000E66EDF50EA6A100FE96E040EEA22E5523A
:10042000E750EF6EDF2AE5D711D80AD046D808D0BA
:10043000040E645C03E162965CD802D0000E01D029
:10044000010EE552E552E7CFD9FF1200D9CFE6FF02
:10045000E1CFD9FFE652040104BF046B556A516A2B
:10046000526A536A546A87EC03F0DF6ADF505B6EAE
:100470005C6A010E5B5C000E5C5819E2525017E199
:10048000F76ADF34FE0BF736F66E5A0EF6260F0EBD
:10049000F7220900F5CF5BF00800F5CF5CF004D03F
:1004A0005CC0FAFF5B50F96EFBDFDF2ADFD7EDD8C7
:1004B000E552E552E7CFD9FF1200020E515C0EE182
:1004C000A7D80401180E026F040E036F080E016F07
:1004D00000BD02D0C80E0BD0880E09D014D904017B
:1004E000080E016F100E026F040E036F8C0E006F6A
:1004F0001200040E575C0AE112C438FF0F01385194
:10050000000802E2050E01D0030E576E51040FE100
:1005100010D8020E555C03E10401840E06D00401DC
:1005200004BD02D0C80E01D0880E046F120083EF04
:1005300003F0D9CFE6FFE1CFD9FF020EE126080E86
:10054000535C000E54580DE253C0DEFF54C0DDFF73
:10055000555002E1010E03D0550406E1020E556E1E
:1005600003D0080EDE6EDD6A040104930491010ECF
:10057000DB500413DFCF05F4DE50535EDD50545AD8
:100580000001180EE26F040EE36F58A21CD0D9CF01
:10059000E9FFDACFEAFFEE50ED1030E0E0C0F6FF01
:1005A000E1C0F7FF0800F550E2C0E9FFE3C0EAFF51
:1005B000EF6EE22B000EE323E02BE123DF06010EBA
:1005C000E6E2DB06E4D7D9CFE9FFDACFEAFFEE5067
:1005D000ED1014E0E0C0E9FFE1C0EAFFEF50E2C037
:1005E000E9FFE3C0EAFFEF6EE22B000EE323E02B0E
:1005F000E123DF06010EE7E2DB06E5D7020EE15C50
:1006000002E2E16AE552E16EE552E7CFD9FF12005E
:10061000D9CFE6FFE1CFD9FF020EE126030E040198
:100620000015E76E010EE7CFDBFF01C4DFFFDE50F0
:100630005326DD5054220001180EE06F040EE16FC6
:10064000D9CFE9FFDACFEAFFEE50ED1014E0E0C0B9
:10065000E9FFE1C0EAFFEF50E2C0E9FFE3C0EAFFD3
:10066000EF6EE22B000EE323E02BE123DF06010E09
:10067000E7E2DB06E5D7020EE15C02E2E16AE55261
:10068000E16EE552E7CFD9FF1200659852500BE1B9
:100690000401080E016F100E026F040E036F840E2A
:1006A000006F04011ED0040110AF1DD05350165D21
:1006B0005450175904E216C453F017C454F039DFEC
:1006C000010E516E0401080E016F100E026F040E30
:1006D000036F800E006F0401180E066F040E076F83
:1006E000C80E046F1200020E516E0401056BC80E95
:1006F000046F0401080E016F180E026F040E036FE1
:10070000C80E006F1200516A0401046B120004014C
:100710001051600BE842E842E842E842E842000932
:1007200001E012001151070A43E00B0A41E0070AF9
:1007300034E0010A24E00B0A20E0020A1EE0030A6A
:100740001AE0080A10E0010A0CE00F0A08E0030AA8
:1007500001E01200010E526E040E576E1200D9EF26
:1007600003F029EF04F0010E526E0001590EE06F04
:10077000000EE16F0ED04DEF04F08EEF04F0010E8D
:10078000526E14510001E06FE16B5A0EE027000E2B
:10079000E1235892010E536E1200010E526E145155
:1007A000EA6A5A0FE96E000EEA2212C4EFFF120045
:1007B0001200800E0401105D4BE11351030A2DE07D
:1007C000010A0BE0030A43E1010E526E00019A0E8A
:1007D000E06F0E0EE16F120E38D0010E526E125104
:1007E000F66EF76AD890F636F736500EF6260F0EEC
:1007F000F7220900F5CFE0F00A00F5CFE1F0020E94
:100800000001F76AE025F66EE151F7220900F5CF05
:1008100053F00A00F5CF54F01AD0010E526E125167
:10082000F66EF76AD890F636F736540EF6260F0EA7
:10083000F7220900F5CFE0F00A00F5CFE1F0E0C0C3
:10084000F6FFE1C0F7FF0800F550536E546A588276
:100850001200010E526E0F0EE66E270EE66E0F0EA0
:10086000E66EC9EC05F0E552E552E552010EE66E82
:100870005A0EE66E000EE66EC9EC05F0E552E55242
:10088000E55212C459F00401125103E1050E576EEE
:100890001200060E576E46EF06F00401186B196B36
:1008A000040110511F0B020A0EE0030A09E0010ABD
:1008B0002AE1010E526E58A026D00401188323D0DD
:1008C000010E526E20D0010E526E14510F0B080D06
:1008D000F3505C6A000F5B6E040E5C221451800BB7
:1008E00001E0010E040DF35000015B24E26F000EE5
:1008F0005C20E36FE2C0E9FFEA6EEF50040B03E017
:100900000401010E186F520408E10001180EE06F97
:10091000040EE16F5892020E536E1200040112058C
:100920000CE110511F0B000908E1010E526E030E7D
:10093000115D02E1588001D05890125134E11051FC
:100940001F0B020830E114510F0B00092CE0010EBF
:10095000526E14510F0B080DF3505C6A000F5B6E62
:10096000040E5C221451800B01E0010E040DF350C3
:1009700000015B24E26F000E5C20E36F030E0401B4
:10098000115D02E1840E03D014AF07D0400EE2C027
:10099000E9FFE3C0EAFFEF6E1200880EE2C0E9FF54
:1009A000E3C0EAFFEF6E120065A60CD8570409E118
:1009B00065BA07D0626A0F01366B36813689020E3E
:1009C000576E1200656A0F01366B6586010E576E11
:1009D0001200656A0F01366B576A1200E9EF04F0E6
:1009E000575001E112006250040B05E00F0136512F
:1009F000040B01E083D865B212006250010B05E0E0
:100A00000F013651010B01E093D86250100B05E045
:100A10000F013651100B01E01FD86250200B05E08A
:100A20000F013651200B01E071D8030E575C01E233
:100A30001200566A040E565C0EE26250080B0BE080
:100A40000F013651080B07E0DFEC01F0000901E16E
:100A50006296562AEFD71200D9CFE6FFE1CFD9FF31
:100A6000020EE12636CFDFFF0F01040E366F6298CB
:100A700065828C50040B01E0010E5B6E8C50080BFC
:100A800001E0010E5B10E76E010EE7CFDBFF8C96F5
:100A90008C94A198A0880300A150100B05E1D050C0
:100AA000080B02E10300F8D7A098DF500F013613BE
:100AB000010EDB50E8B08C86E8A08C96010EDB506E
:100AC000E8B08C84E8A08C94D50E4F6E020E506E68
:100AD0004FC05BF050C05CF04F06000E505A5B50A8
:100AE0005C1002E00400F4D7020EE15C02E2E16A6D
:100AF000E552E16EE552E7CFD9FF120065920F0192
:100B0000369562A402D06294FCD712000F0126A190
:100B10000DD0800E0401005D07E1840E0401045D28
:100B200003E104018C0E006F0F012691629A1200FE
:100B3000636A626A0F019F0E376F0F017B0E366F7B
:100B40000F01386B0F0EE66E270EE66E0F0EE66E87
:100B500020D8E552E552E5520F01160E266F62A627
:100B600005D0629600D000D00000F9D7659883ECDC
:100B700003F00401080E016F0401100E026F040E51
:100B8000036F04018C0E006F5890596A030E576E64
:100B90001200D9CFE6FFE1CFD9FFFD0EDBCFE9FF91
:100BA000FE0EDBCFEAFFFC0EDB5004E0EE6AFC0E2B
:100BB000DB06F9D7E552E7CFD9FF12000401105147
:100BC0001F0B010801E01200145101E01200060E93
:100BD000115D21E11351230A1DE0010A0DE0030A12
:100BE00019E1020E526E590405E10001BE0EE06FDC
:100BF0000E0EE16F090E0CD0020E526E590405E183
:100C00000001330EE06F0F0EE16F590403E11D0E7A
:100C1000536E546A588204011051600BE842E84256
:100C2000E842E842E842010801E0120011510B0AD3
:100C300026E0080A19E0090A12E0080A09E00B0A8E
:100C400005E0080A01E0120044EF06F045EF06F067
:100C5000020E526E00014A0EE06F000E0BD0020E23
:100C6000526E13C44AF01200020E526E00014B0E77
:100C7000E06F000EE16F5892010E536E1200020EEB
:100C8000526E12C44BF01200120012004C6A0F0197
:100C90001E0E276F0401400E096F200E0A6F040E0E
:100CA0000B6F880E086F0401600E0E6F040E0F6F3D
:100CB000400E0C6F1200D9CFE6FFE1CFD9FFE6520C
:100CC000FC0EDB50400805E2400EF36EFC0EF3CF45
:100CD000DBFFDF6AFC0EDB50DF5C19E2DF50E76E02
:100CE000FD0EDBCFE9FFFE0EDBCFEAFFE750E92682
:100CF000000EEA22EF50E66EDF50EA6A600FE96EFE
:100D0000040EEA22E552E750EF6EDF2AE3D7FC0E2D
:100D1000DBCF0DF4400E04010C170C7D880E0C1374
:100D2000E552E552E7CFD9FF1200D9CFE6FFE1CF78
:100D3000D9FF4C6A040108BF2FD0FC0EDBCF5BF05B
:100D40000951D8805B5403E2FC0E09C4DBFF4C6AF6
:100D5000FC0EDB504C5C19E24C50EA6A200FE96E45
:100D6000040EEA22EF50E66E4C50E76EFD0EDBCF2C
:100D7000E9FFFE0EDBCFEAFFE750E926000EEA228C
:100D8000E552E750EF6E4C2AE3D70401400E096F9D
:100D90000817087D880E08134C50E552E7CFD9FF9D
:100DA00012001DEE00F02DEE00F0F86AF66A100E4B
:100DB000F76E0800F550FF0808E1010EF66E100E00
:100DC000F76E0800F550FF0806E080AE02D000EF95
:100DD00008F080AEFED701D812000DD8040034D838
:100DE00037D8060E575C05E16550020B02E125EC91
:100DF00000F0F4D71200600ED36E9B8C580E4F6E2D
:100E0000020E506E4FC05BF050C05CF04F06000EFB
:100E1000505A5B505C10F6E165A604D06592656A95
:100E2000C7EC01F00F01140E396F576A586A596AFE
:100E300019EC00F04D6A4E6A8C968C9495969594B8
:100E40000F01486B496B1200D4EC04F0F0EF04F092
:100E50004D504E1004E1100E4D6E270E4E6E4D0695
:100E6000000E4E5A060E575C02E28C868C94060EDB
:100E7000575C12E14D504E100FE10001E65102E1C6
:100E80008C868C94030EE65D02E18C968C84E62BB6
:100E9000E651030801E2E66B1200120100020000B5
:100EA0000008D8043C0002000102000109022900E8
:100EB000010100C032090400000203000000092102
:100EC00011010001221D00070581034000010705F3
:100ED00001034000010403090434034D0069006369
:100EE0000072006F00630068006900700020005409
:100EF000006500630068006E006F006C006F0067A3
:100F0000007900200049006E0063002E002603488F
:100F100000490044002000550053004200200042D8
:100F2000006F006F0074006C006F0061006400656A
:100F30000072000600FF0901A101190129401500F6
:100F400026FF00750895408100190129409100C0D5
:100F5000AC0EAC0ED50ED90E0D0FBC0BC00EF36E41
:100F600000EE00F00E0E01D81200EA6002D0EE6A28
:0C0F7000FCD7F350E9601200EE6AFCD7D9
:06100000B8EF7AF01200C7
:0610080028EF08F01200C1
:06101800F4EF41F01200AC
:10102A000300DDF5000000060000E1000000D4F531
:10103A000000B70E000009000000D2F50000F30519
:10104A00000002000000E9CFE4FFEACFE4FFE65225
:10105A00D9CFE6FFDACFE6FFE1CFD9FFE2CFDAFF59
:10106A00E6529EA0E9D29E90FE0ECF6E3D0ECE6E47
:10107A0019C530F50501316B0501010E326F050105
:10108A001A511B111C111D1117E0D880000E050101
:10109A001A55000E1B55190E1C55000E1D5506E259
:1010AA0005011A6B1B6B1C6B1D6B06D005011A0719
:1010BA00000E1B5B1C5B1D5B05011A511B111C11E9
:1010CA001D1102E00501326B0501000501E03DD169
:1010DA000501115112111311141107E105011551DE
:1010EA0016111711181101E12FD10501D7510DE180
:1010FA00050119A302D08C8E01D08C9E050119A777
:10110A0002D08C8A01D08C9A0FD00501D7050CE148
:10111A00050119A302D08B8401D08B94050119A76C
:10112A0002D0898401D08994050111511211131139
:10113A00141164E0010EE96E050EEA6E0E01B75154
:10114A00EE240E01B76F0E01B851EE200E01B86FF2
:10115A000E01B951EE200E01B96F0E01BA51EE20FF
:10116A000E01BA6FB7CE4CF0B8CE4DF0B9CE4EF0F4
:10117A00BACE4FF04C6A4D6A4E6A800E4F164C50EA
:10118A004D104E104F1028E0B7CEB7FEB8CEB8FEBD
:10119A00B9CEB9FEBACEBAFE0E01BA9F010E05014A
:1011AA0030110501306F0501010E316F050111077C
:1011BA00000E125B135B145B050119A307D005012E
:1011CA002807000E295B2A5B2B5B06D00501282B1A
:1011DA00000E29232A232B23050109510501012782
:1011EA0005010A510501022305010B5105010323DB
:1011FA0005010C51050104230501326B0501155146
:10120A0016111711181164E0050EE96E050EEA6E43
:10121A000E01BB51EE240E01BB6F0E01BC51EE2034
:10122A000E01BC6F0E01BD51EE200E01BD6F0E0105
:10123A00BE51EE200E01BE6FBBCE4CF0BCCE4DF0BF
:10124A00BDCE4EF0BECE4FF04C6A4D6A4E6A800E4D
:10125A004F164C504D104E104F1028E0BBCEBBFE1F
:10126A00BCCEBCFEBDCEBDFEBECEBEFE0E01BE9F36
:10127A00040E050130110501306F0501010E316FB1
:10128A0005011507000E165B175B185B050119A708
:10129A0007D005012C07000E2D5B2E5B2F5B06D0B5
:1012AA0005012C2B000E2D232E232F2305010D5172
:1012BA000501052705010E510501062305010F51F8
:1012CA000501072305011051050108230501326BA9
:1012DA000501315139E00501D75107E1050130B166
:1012EA008C8C050130B58C8809D00501D70506E13B
:1012FA00050130B18B8C050130B5898A00000000E8
:10130A0000000000000000000000000000000000D3
:10131A0000000000000000000000000000000000C3
:10132A0000000000000000000000000000000000B3
:10133A0000000501D75103E18C9C8C9805D005016A
:10134A00D70502E18B9C899AD7D0030E0501005D6F
:10135A0001E0A0D00501E45101E179D005012105A0
:10136A00DF6E05011E511F1137E1DF50EA6A310FA6
:10137A00E96E0E0EEA22EF500E01EA6AAC25E96E1A
:10138A00AD51EA22EF6AEA6ADF34FE0BEA36E96E09
:10139A00790EE9260E0EEA22EE6AED6AEA6ADF346F
:1013AA00FE0BEA36E96E490EE9260E0EEA22EE6ACD
:1013BA00ED6ADF50EA6A310FE96E0E0EEA22EF6A31
:1013CA00EA6ADF34FE0BEA36E96E010EE9260E0EF2
:1013DA00EA22EE6AED6A3BD0EA6ADF34FE0BEA36AD
:1013EA00E96E790EE9260E0EEA2222C5EEFF23C522
:1013FA00EDFFEA6ADF34FE0BEA36E96E490EE926AA
:10140A000E0EEA221EC5EEFF1FC5EDFFDF50EA6A87
:10141A00310FE96E0E0EEA2220C5EFFFEA6ADF34C9
:10142A00FE0BEA36E96E010EE9260E0EEA22EE50AE
:10143A00ED100DE1EA6ADF34FE0BEA36E96E010EC1
:10144A00E9260E0EEA221EC5EEFF1FC5EDFF0E01AC
:10145A00B6510501205D1DE10E01B05105011E19AD
:10146A0004E10E01B15105011F190AE10501010E3E
:10147A00D86F0501D46B0501E35101E08A9809D0C0
:10148A000501D86B0501010ED46F0501E35101E096
:10149A008A8832D0040E0501005D2EE1050124512F
:1014AA0024E025C54CF026C54DF0D8904D324C327B
:1014BA00D8904D324C324C50BB6EE1C54EF0E2C56D
:1014CA004FF0040ED8904E364F36E804FBE1300E4A
:1014DA004E16000E4F16CF0EBA1400014E104C6E67
:1014EA004FC04DF04C50BA6E04D0BB6ACF0EBA143E
:1014FA00BA6E0501010E326F0501325101E190D039
:10150A0005011A511B111C111D1101E089D0050199
:10151A00006B0501275101E07ED034C500F535C5C1
:10152A0001F536C502F537C503F538C504F539C5E1
:10153A0005F53AC506F53BC507F53CC508F53DC5B1
:10154A0009F53EC50AF53FC50BF540C50CF541C581
:10155A000DF542C50EF543C50FF544C510F545C551
:10156A0011F546C512F547C513F548C514F549C521
:10157A0015F54AC516F54BC517F54CC518F54DC5F1
:10158A0019F54EC51AF54FC51BF550C51CF551C5C1
:10159A001DF552C51EF553C51FF554C520F555C591
:1015AA0021F556C522F557C523F558C524F559C561
:1015BA0025F55AC526F50501346B0501356B366BE1
:1015CA00376B386B0501396B3A6B3B6B3C6B05012A
:1015DA00456B466B476B486B0501496B4A6B4B6B16
:1015EA004C6B05014D6B05014E6B4F6B506B516B8C
:1015FA000501526B536B0501546B0501556B0501CF
:10160A00566B576B0501586B0501596B5A6B0501EF
:10161A00010E276F05D005011A6B1B6B1C6B1D6B26
:10162A008050800B06E00501DF5106E08150010B76
:10163A0003E10501010EDE6FE552E552E5CFDAFF5F
:10164A00E7CFD9FFE552E5CFEAFFE5CFE9FF110081
:10165A00D9CFE6FFDACFE6FFE1CFD9FFE2CFDAFF53
:10166A00E652DF6ADFCF00F0020EE76E0018E8AE3E
:10167A0002D0E73402D0E750005C3CE2DFCFE9FF5A
:10168A00EA6AE9BEEA68D890E936EA36D890E936D5
:10169A00EA36010EE926050EEA22010EEE6EEE6A20
:1016AA00EE6AEE6ADFCFE9FFEA6AE9BEEA68D89035
:1016BA00E936EA36D890E936EA36110EE926050EF9
:1016CA00EA22EE6AEE6AEE6AEE6ADFCFE9FFEA6ABA
:1016DA00E9BEEA68D890E936EA36D890E936EA36B9
:1016EA00090EE926050EEA22EE6AEE6AEE6AEE6A4B
:1016FA00DF2AB8D70501006B0501196B05011A6BC2
:10170A001B6B1C6B1D6B05011E6B1F6B0501206B90
:10171A000501216B0501226B236B0501010E276F61
:10172A00CD82CD9ECD9CCD9ACD98CD96CD94FE0EF0
:10173A00CF6E3D0ECE6ECD809F809E909D80928012
:10174A009F9C010EE66EE66A5EEC4DF0E552E552AC
:10175A00010EE66E0B0EE66E5EEC4DF0E552E552BA
:10176A008D8496948D829692898C929C8D80969087
:10177A008B8294928C9C959C8C9E959E8C98959825
:10178A008C9A959A949E828E0000000000000000B8
:10179A00000000000000000000000000000000003F
:1017AA000000000000000000000000000000948E0D
:1017BA00829E0501010EE36F0501010EE46F8A980E
:1017CA0093980501010ED46F0501D76B0501010E2F
:1017DA00D86F0501DD6B0501D96BDA6BDB6BDC6B4E
:1017EA000501DE6B9380F19E0501010EDF6F939672
:1017FA008196A1EC25F0E552E552E5CFDAFFE7CF75
:10180A00D9FF1200D9CFE6FFDACFE6FFE1CFD9FF41
:10181A00E2CFDAFFE652E652E652DF6A010EDB6AEF
:10182A00020EDB6AE66AD9CFE6FFDACFE6FF010EDF
:10183A00E66EBCEC55F0E552E552E552E552E66A31
:10184A00D950010FE66E000EDA20E66E030EE66E40
:10185A00BCEC55F0E552E552E552E5520701B451A8
:10186A0001E008D1DF043FE1D950010FE96E000E13
:10187A00DA20EA6EEE50ED1018E10501010EE36F71
:10188A00E46B000EE66EE66AE66EE66AB6CEE6FF40
:10189A00E66EE66A4EEC75F0006E070EE15C02E257
:1018AA00E16AE552E16E005013D0D950010FE96E9A
:1018BA00000EDA20EA6E010EEE1806E1ED5004E1A0
:1018CA000501E36B010E03D00501010EE36FE46F1E
:1018DA00000EE66EE66AD8C5E6FF93EC21F0E55203
:1018EA00E552E552C5D0020EDF5C4AE1D950010F3C
:1018FA00E96E000EDA20EA6EEE50ED1009E10501FC
:10190A00D76B96909492959C959E9598959A31D07E
:10191A00D950010FE96E000EDA20EA6E010EEE18B8
:10192A0012E1ED5010E10501010ED76F9680948205
:10193A00958C958E9588958A94949294949C929A73
:10194A009592929295D0D950010FE96E000EDA2045
:10195A00EA6E020EEE1801E08BD0ED5001E088D05D
:10196A000501020ED76F96809482958C958E958884
:10197A00958A94849284948C928A9582928278D061
:10198A00040EDF5C07E1010EDBCFB0FE020EDBCFF7
:10199A00B1FE6ED0050EDF5C07E1010EDBCFAEFEB5
:1019AA00020EDBCFAFFE64D0080EDF5C17E1D95020
:1019BA00010FE96E000EDA20EA6E180ED880EE5496
:1019CA00000EED5407E2180EF36E010EF3CFDBFFA3
:1019DA00020EDB6A010EDBCFAAFE4AD0090EDF5CDB
:1019EA0017E1D950010FE96E000EDA20EA6E060EF1
:1019FA00D880EE54000EED5407E2060EF36E010E87
:101A0A00F3CFDBFF020EDB6A010EDBCFABFE30D079
:101A1A000A0EDF5C07E1010EDBCFB2FE020EDBCF5E
:101A2A00B3FE0DD00B0EDF5C07E1010EDBCFB2FE79
:101A3A00020EDBCFB3FE1CD00C0EDF5C07E1010EF9
:101A4A00DBCFB4FE020EDBCFB5FE12D00D0EDF5C8B
:101A5A000FE1D950010FE96E000EDA20EA6EEE505E
:101A6A00ED1004E00501010EDF6F02D00501DF6B06
:101A7A0018EC4CF0E552E552E552E552E5CFDAFFB3
:101A8A00E7CFD9FF1200D9CFE6FFDACFE6FFE1CFE1
:101A9A00D9FFE2CFDAFF200EE12402E3E168E65241
:101AAA00E16EDE6ADE6ADE6ADD6ADD52DD52040E4E
:101ABA00DB6A050EDB6A060EDB6A070EDB6A080EB6
:101ACA00DB6A090EDB6A0A0EDB6A0B0EDB6A0C0E96
:101ADA00DB6A0D0EDB6A0E0EDB6A0F0EDB6A100E76
:101AEA00DB6A110EDB6A120EDB6A130EDB6AE66A28
:101AFA00D950040FE66E000EDA20E66E070EE66E87
:101B0A00BCEC55F0E552E552E552E552E66AD95089
:101B1A00060FE66E000EDA20E66E070EE66EBCECE5
:101B2A0055F0E552E552E552E552E66AD950080FFA
:101B3A00E66E000EDA20E66E060EE66EBCEC55F096
:101B4A00E552E552E552E552E66AD9500C0FE66EC7
:101B5A00000EDA20E66E060EE66EBCEC55F0E55293
:101B6A00E552E552E552D950040FE96E000EDA202B
:101B7A00EA6EA80ED880EE54610EED5405E2AE0E60
:101B8A00006EDC0E1AEF12F0D950060FE96E000E45
:101B9A00DA20EA6EA80ED880EE54610EED5405E202
:101BAA00800E006EDC0E1AEF12F0040EDBCF00F08E
:101BBA00050EDBCF01F0040E005C000E015805E2B1
:101BCA00560E006EDC0E1AEF12F0060EDBCF00F096
:101BDA00070EDBCF01F0040E005C000E015805E28F
:101BEA002E0E006EDC0E1AEF12F00701B45102E05D
:101BFA002DEF12F0080EDBCF10F0090EDBCF11F03B
:101C0A000A0EDBCF12F00B0EDBCF13F010C038F048
:101C1A0011C039F012C03AF013C03BF0080EDBCF06
:101C2A003DF0090EDBCF3EF00A0EDBCF3FF00B0E84
:101C3A00DBCF40F0F5EC79F034C00CF035C00DF094
:101C4A0036C00EF037C00FF00C0EDBCF14F00D0EBD
:101C5A00DBCF15F00E0EDBCF16F00F0EDBCF17F031
:101C6A0014C038F015C039F016C03AF017C03BF06E
:101C7A000C0EDBCF3DF00D0EDBCF3EF00E0EDBCFB0
:101C8A003FF00F0EDBCF40F0F5EC79F00C50342426
:101C9A00086E0D503520096E0E5036200A6E0F5010
:101CAA0037200B6E08C038F009C039F00AC03AF084
:101CBA003B6EE5EC69F039C004F03AC005F03BC070
:101CCA0006F03CC007F039C0E6FF3AC0E6FF3BC069
:101CDA00E6FF3CC0E6FFF5EC71F0E552E552E5524D
:101CEA00E55238C000F039C001F03AC002F03BC0FA
:101CFA0003F038C039F001C03AF002C03BF003C02B
:101D0A003CF055EC6BF0140E38C0DBFF150E39C0F1
:101D1A00DBFF160E3AC0DBFF170E3BC0DBFF0501E7
:101D2A002751FDE04E6B4F6B506B516B4D6B8D9095
:101D3A008B92D950080FE96E000EDA20EA6ED8901D
:101D4A00030EEB50000A08E6000EEE5C000EEE5899
:101D5A00000EEE58000EEE5820E2020E4D6F080EED
:101D6A00DBCF38F0090EDBCF39F00A0EDBCF3AF0C1
:101D7A000B0EDBCF3BF03D683E683F684068F5ECF0
:101D8A0079F0080E34C0DBFF090E35C0DBFF0A0EFE
:101D9A0036C0DBFF0B0E37C0DBFFD9500C0FE96EE4
:101DAA00000EDA20EA6ED890030EEB50000A08E61D
:101DBA00000EEE5C000EEE58000EEE58000EEE58C5
:101DCA0022E2080E05014D114D6F0C0EDBCF38F0E3
:101DDA000D0EDBCF39F00E0EDBCF3AF00F0EDBCF54
:101DEA003BF03D683E683F684068F5EC79F00C0EC0
:101DFA0034C0DBFF0D0E35C0DBFF0E0E36C0DBFF35
:101E0A000F0E37C0DBFF080EDBCF39F0090EDBCF30
:101E1A003AF00A0EDBCF3BF00B0EDBCF3CF03C3442
:101E2A00000E3C1809E6D880FF0E3954FF0E3A54CA
:101E3A00FF0E3B54000E3C5404E2000E006EDC0E12
:101E4A00F4D20C0EDBCF39F00D0EDBCF3AF00E0ECA
:101E5A00DBCF3BF00F0EDBCF3CF03C34000E3C18DE
:101E6A0009E6D880FF0E3954FF0E3A54FF0E3B5450
:101E7A00000E3C5404E2D20E006EDB0ED6D2040EE3
:101E8A00DBCF3AF0050EDBCF3BF0CEEC69F039C080
:101E9A0004F03AC005F03BC006F03CC007F0AC0EB7
:101EAA003E6EC50E3F6EA70E406E470E416E51EC58
:101EBA006AF039C000F03AC001F03BC002F03CC001
:101ECA0003F0140EDBCF0CF0150EDBCF0DF0160E5F
:101EDA00DBCF0EF0170EDBCF0FF00CC038F00DC0C1
:101EEA0039F00EC03AF00FC03BF0E3EC69F039C0AC
:101EFA0008F03AC009F03BC00AF03CC00BF039C008
:101F0A003EF03AC03FF03BC040F03CC041F000C058
:101F1A0039F001C03AF002C03BF003C03CF0FEECDD
:101F2A0069F0180E39C0DBFF190E3AC0DBFF1A0E32
:101F3A003BC0DBFF1B0E3CC0DBFF180EDBCF00F003
:101F4A00190EDBCF01F01A0EDBCF02F01B0EDBCF2E
:101F5A0003F0080EDBCF08F0090EDBCF09F00A0EFA
:101F6A00DBCF0AF00B0EDBCF0BF008C038F009C04C
:101F7A0039F00AC03AF00BC03BF0E5EC69F039C021
:101F8A0004F03AC005F03BC006F03CC007F039C087
:101F9A003EF03AC03FF03BC040F03CC041F000C0C8
:101FAA0039F001C03AF002C03BF003C03CF051ECFA
:101FBA006AF055EC6BF038C035F539C036F53AC0E1
:101FCA0037F53BC038F5080EDBCF45F5090EDBCFF8
:101FDA0046F50A0EDBCF47F50B0EDBCF48F5060EAA
:101FEA00DBCF3AF0070EDBCF3BF0CEEC69F039C01D
:101FFA0008F03AC009F03BC00AF03CC00BF0060EEC
:10200A00DBCF3AF0070EDBCF3BF0CEEC69F039C0FC
:10201A000CF03AC00DF03BC00EF03CC00FF039C0D6
:10202A003EF03AC03FF03BC040F03CC041F008C02F
:10203A0039F009C03AF00AC03BF00BC03CF051EC51
:10204A006AF039C004F03AC005F03BC006F03CC063
:10205A0007F0040EDBCF3AF0050EDBCF3BF0CEECF7
:10206A0069F039C014F03AC015F03BC016F03CC014
:10207A0017F0040EDBCF3AF0050EDBCF3BF0CEECC7
:10208A0069F039C018F03AC019F03BC01AF03CC0E8
:10209A001BF039C03EF03AC03FF03BC040F03CC0B4
:1020AA0041F014C039F015C03AF016C03BF017C021
:1020BA003CF051EC6AF039C010F03AC011F03BC064
:1020CA0012F03CC013F039C03EF03AC03FF03BC0BA
:1020DA0040F03CC041F004C039F005C03AF006C0F7
:1020EA003BF007C03CF0BEEC6AF039C000F03AC0E1
:1020FA0001F03BC002F03CC003F0140EDBCF28F025
:10210A00150EDBCF29F0160EDBCF2AF0170EDBCF28
:10211A002BF028C038F029C039F02AC03AF02BC079
:10212A003BF0E3EC69F039C024F03AC025F03BC03B
:10213A0026F03CC027F0140EDBCF30F0150EDBCFB3
:10214A0031F0160EDBCF32F0170EDBCF33F030C092
:10215A0038F031C039F032C03AF033C03BF0E3EC2A
:10216A0069F039C02CF03AC02DF03BC02EF03CC0CB
:10217A002FF039C03EF03AC03FF03BC040F03CC0BF
:10218A0041F024C039F025C03AF026C03BF027C000
:10219A003CF051EC6AF039C020F03AC021F03BC063
:1021AA0022F03CC023F03E6A3F6A406A400E416E0C
:1021BA0051EC6AF039C01CF03AC01DF03BC01EF069
:1021CA003CC01FF039C03EF03AC03FF03BC040F07F
:1021DA003CC041F000C039F001C03AF002C03BF007
:1021EA0003C03CF0FEEC69F01C0E39C0DBFF1D0E8B
:1021FA003AC0DBFF1E0E3BC0DBFF1F0E3CC0DBFFFD
:10220A00080EDBCF04F0090EDBCF05F00A0EDBCF98
:10221A0006F00B0EDBCF07F004C038F005C039F02A
:10222A0006C03AF007C03BF0E5EC69F01C0EDBCFC4
:10223A003EF01D0EDBCF3FF01E0EDBCF40F01F0E2F
:10224A00DBCF41F051EC6AF039C000F03AC001F03E
:10225A003BC002F03CC003F0210E3E6EE60E3F6E1C
:10226A005B0E406E400E416E51EC6AF055EC6BF01D
:10227A0038C03DF539C03EF53AC03FF53BC040F5A0
:10228A00180EDBCF00F0190EDBCF01F01A0EDBCFF0
:10229A0002F01B0EDBCF03F00C0EDBCF08F00D0EA5
:1022AA00DBCF09F00E0EDBCF0AF00F0EDBCF0BF0FF
:1022BA0008C038F009C039F00AC03AF00BC03BF048
:1022CA00E5EC69F039C004F03AC005F03BC006F00D
:1022DA003CC007F039C03EF03AC03FF03BC040F086
:1022EA003CC041F000C039F001C03AF002C03BF0F6
:1022FA0003C03CF051EC6AF055EC6BF038C039F58C
:10230A0039C03AF53AC03BF53BC03CF50C0EDBCF81
:10231A0049F50D0EDBCF4AF50E0EDBCF4BF50F0E4E
:10232A00DBCF4CF50C0EDBCF04F00D0EDBCF05F046
:10233A000E0EDBCF06F00F0EDBCF07F004C038F02D
:10234A0005C039F006C03AF007C03BF0E5EC69F089
:10235A001C0EDBCF3EF01D0EDBCF3FF01E0EDBCF97
:10236A0040F01F0EDBCF41F051EC6AF039C000F0AB
:10237A003AC001F03BC002F03CC003F0210E3E6EB1
:10238A00E60E3F6E5B0E406E400E416E51EC6AF0F7
:10239A0055EC6BF038C041F539C042F53AC043F507
:1023AA003BC044F5040EDBCF00F0050EDBCF01F095
:1023BA00060EDB50001803E1070EDB50011814E08B
:1023CA0005013D513E113F1140110EE1D880000E2A
:1023DA004555000E4655000E4755000E485504E275
:1023EA00A70E006EDB0E21D0040EDBCF00F0050E27
:1023FA00DBCF01F0060EDB50001803E1070EDB50BD
:10240A00011820E0050141514211431144111AE11A
:10241A00D880000E4955000E4A55000E4B55000E45
:10242A004C5510E27C0E006EDB0E016E026A00C093
:10243A00E6FFE66E02C0E6FF1FEC79F0E552E552D0
:10244A00E55206D00501010E346F276B18EC4CF0EB
:10245A00200EE15C02E2E16AE552E16EE552E5CF67
:10246A00DAFFE7CFD9FF1200D9CFE6FFDACFE6FFCE
:10247A00E1CFD9FFE2CFDAFF3F0EE12402E3E168C0
:10248A00E652E16E0C0EDB6A0D0EDB6A0E0EDB6A9B
:10249A000F0EDB6A140EDB6A150EDB6A160EDB6A98
:1024AA00170EDB6AE66AD9CFE6FFDACFE6FF070E38
:1024BA00E66EBCEC55F0E552E552E552E552E66AA5
:1024CA00D950100FE66E000EDA20E66E060EE66EA2
:1024DA00BCEC55F0E552E552E552E552E66AD950B0
:1024EA00040FE66E000EDA20E66E060EE66EBCEC0F
:1024FA0055F0E552E552E552E552E66AD950080F21
:10250A00E66E000EDA20E66E070EE66EBCEC55F0BB
:10251A00E552E552E552E552E66AD950140FE66EE5
:10252A00000EDA20E66E060EE66EBCEC55F0E552B9
:10253A00E552E552E552E66AD9500C0FE66E000EF6
:10254A00DA20E66E060EE66EBCEC55F0E552E55270
:10255A00E552E5520701B45101E0D3D1D9CFE9FFE1
:10256A00DACFEAFFEECF00F0EECF01F0EECF02F0C5
:10257A00EFCF03F0005001100210031011E1040E16
:10258A00DBCF04F0050EDBCF05F0060EDBCF06F03D
:10259A00070EDBCF07F0045005100610071011E0F4
:1025AA00100EDBCF08F0110EDBCF09F0120EDBCFD5
:1025BA000AF0130EDBCF0BF0085009100A100B10AB
:1025CA0035E1080EDBCF0CF0090EDBCF0DF00A0E59
:1025DA00DBCF0EF00B0EDBCF0FF00C500D100E10F0
:1025EA000F1012E10C0EDBCF10F00D0EDBCF11F045
:1025FA000E0EDBCF12F00F0EDBCF13F010501110BE
:10260A001210131001E17DD1140EDBCF14F0150E58
:10261A00DBCF15F0160EDBCF16F0170EDBCF17F057
:10262A00145015101610171001E16BD1320EDB6A27
:10263A00330EDB6A340EDB6A350EDB6A310EDB6A77
:10264A008D908B92D950100FE96E000EDA20EA6E47
:10265A00D890030EEB50000A08E6000EEE5C000E5E
:10266A00EE58000EEE58000EEE5825E2310EDB5001
:10267A000209E76E310EE7CFDBFF100EDBCF38F031
:10268A00110EDBCF39F0120EDBCF3AF0130EDBCF8F
:10269A003BF03D683E683F684068F5EC79F0100E03
:1026AA0034C0DBFF110E35C0DBFF120E36C0DBFF74
:1026BA00130E37C0DBFFD950140FE96E000EDA2073
:1026CA00EA6ED890030EEB50000A08E6000EEE5CA4
:1026DA00000EEE58000EEE58000EEE5825E2310EAE
:1026EA00DB500809E76E310EE7CFDBFF140EDBCFB4
:1026FA0038F0150EDBCF39F0160EDBCF3AF0170E95
:10270A00DBCF3BF03D683E683F684068F5EC79F006
:10271A00140E34C0DBFF150E35C0DBFF160E36C0B3
:10272A00DBFF170E37C0DBFFD9CFE9FFDACFEAFFAD
:10273A00190EEECFDBFF1A0EEECFDBFF1B0EEECF2C
:10274A00DBFF1C0EEECFDBFFD950100FE96E000E37
:10275A00DA20EA6E290EEECFDBFF2A0EEECFDBFF80
:10276A002B0EEECFDBFF2C0EEECFDBFFD950040F82
:10277A00E96E000EDA20EA6E210EEECFDBFF220EA2
:10278A00EECFDBFF230EEECFDBFF240EEECFDBFF17
:10279A00D950080FE96E000EDA20EA6E1D0EEECF50
:1027AA00DBFF1E0EEECFDBFF1F0EEECFDBFF200E90
:1027BA00EECFDBFFD950140FE96E000EDA20EA6E75
:1027CA002D0EEECFDBFF2E0EEECFDBFF2F0EEECF60
:1027DA00DBFF300EEECFDBFFD9500C0FE96E000E97
:1027EA00DA20EA6E250EEECFDBFF260EEECFDBFFF8
:1027FA00270EEECFDBFF280EEECFDBFF010EF36EC6
:10280A00180EF3CFDBFF05012751FDE0180EDBCFD1
:10281A0034F5190EDBCF35F51A0EDBCF36F51B0E64
:10282A00DBCF37F51C0EDBCF38F51D0EDBCF39F5C4
:10283A001E0EDBCF3AF51F0EDBCF3BF5200EDBCFAA
:10284A003CF5210EDBCF3DF5220EDBCF3EF5230E04
:10285A00DBCF3FF5240EDBCF40F5250EDBCF41F56C
:10286A00260EDBCF42F5270EDBCF43F5280EDBCF52
:10287A0044F5290EDBCF45F52A0EDBCF46F52B0EA4
:10288A00DBCF47F52C0EDBCF48F52D0EDBCF49F514
:10289A002E0EDBCF4AF52F0EDBCF4BF5300EDBCFFA
:1028AA004CF5310EDBCF4DF5320EDBCF4EF5330E44
:1028BA00DBCF4FF5340EDBCF50F5350EDBCF51F5BC
:1028CA00360EDBCF52F5370EDBCF53F5380EDBCFA2
:1028DA0054F5390EDBCF55F53A0EDBCF56F53B0EE4
:1028EA00DBCF57F53C0EDBCF58F53D0EDBCF59F564
:1028FA003E0EDBCF5AF5276B0701E35102E018ECD5
:10290A004CF03F0EE15C02E2E16AE552E16EE5520B
:10291A00E5CFDAFFE7CFD9FF1200D9CFE6FFDACF4A
:10292A00E6FFE1CFD9FFE2CFDAFF100EE12402E39E
:10293A00E168E652E16EDE6ADE6ADE6ADD6ADD526F
:10294A00DD52040EDB6A050EDB6A060EDB6A070E31
:10295A00DB6A080EDB6A090EDB6A0A0EDB6A0B0EFB
:10296A00DB6A0C0EDB6A0D0EDB6A0E0EDB6A0F0EDB
:10297A00DB6AE66AD9CFE6FFDACFE6FF070EE66E34
:10298A00BCEC55F0E552E552E552E552E66AD950FB
:10299A00040FE66E000EDA20E66E060EE66EBCEC5A
:1029AA0055F0E552E552E552E552010EE66ED95070
:1029BA00080FE66E000EDA20E66E060EE66EBCEC36
:1029CA0055F0E552E552E552E5520E01BF5101E1DB
:1029DA00F5D1D9CFE9FFDACFEAFFEECF00F0EECF9B
:1029EA0001F0EECF02F0EFCF03F000500110021019
:1029FA00031002E10701B48D0701B45101E014D2BA
:102A0A00D9CFE9FFDACFEAFFD880FF0EEE54FF0EE6
:102A1A00EE54FF0EEE54000EEE5404E2490E006E20
:102A2A00DB0EBFD1040EDBCF39F0050EDBCF3AF057
:102A3A00060EDBCF3BF0070EDBCF3CF03C34000E3A
:102A4A003C1809E6D880000E3954000E3A54000E9C
:102A5A003B54000E3C5413E2D950040FE96E000EA9
:102A6A00DA20EA6E0C0EEECFDBFF0D0EEECFDBFFA7
:102A7A000E0EEECFDBFF0F0EEECFDBFF1ED0040EE5
:102A8A00DBCF38F0050EDBCF39F0060EDBCF3AF09C
:102A9A00070EDBCF3BF03D683E683F684068F5ECC7
:102AAA0079F00C0E34C0DBFF0D0E35C0DBFF0E0EC5
:102ABA0036C0DBFF0F0E37C0DBFF0C0EDBCF39F061
:102ACA000D0EDBCF3AF00E0EDBCF3BF00F0EDBCF55
:102ADA003CF03C34000E3C1809E6D880FF0E39540D
:102AEA00FF0E3A54FF0E3B54000E3C5404E2000E13
:102AFA00006EDC0E56D10C0EDBCF00F00D0EDBCFD4
:102B0A0001F00E0EDBCF02F00F0EDBCF03F000C098
:102B1A0038F001C039F002C03AF003C03BF0DFCF11
:102B2A003DF0010EDBCF3EF0020EDBCF3FF0030E8D
:102B3A00DBCF40F053EC7AF0D880190E3854000EEF
:102B4A003954000E3A54000E3B5404E2190E006E3A
:102B5A00DB0E27D1D9CFE9FFDACFEAFFEECF00F0BB
:102B6A00EECF01F0EECF02F0EFCF03F01F0E3D6E75
:102B7A00050E3E6E3F6A406A00C038F001C039F067
:102B8A0002C03AF003C03BF053EC7AF038C000F0D0
:102B9A0039C001F03AC002F03BC003F0D9500C0F23
:102BAA00E96E000EDA20EA6EEE50385CEE503958C3
:102BBA00EE503A58EE503B5815E30C0EDBCF04F0BA
:102BCA000D0EDBCF05F00E0EDBCF06F00F0EDBCFBE
:102BDA0007F0045005100610071004E0F30E006E0B
:102BEA00DA0EDFD0080EDBCF39F0090EDBCF3AF070
:102BFA000A0EDBCF3BF00B0EDBCF3CF03C34000E71
:102C0A003C1809E6D880000E3954000E3A54000EDA
:102C1A003B54000E3C5413E2D950080FE96E000EE3
:102C2A00DA20EA6E0C0EEECFDBFF0D0EEECFDBFFE5
:102C3A000E0EEECFDBFF0F0EEECFDBFF1ED0080E1F
:102C4A00DBCF38F0090EDBCF39F00A0EDBCF3AF0D2
:102C5A000B0EDBCF3BF03D683E683F684068F5EC01
:102C6A0079F00C0E34C0DBFF0D0E35C0DBFF0E0E03
:102C7A0036C0DBFF0F0E37C0DBFF0C0EDBCF39F09F
:102C8A000D0EDBCF3AF00E0EDBCF3BF00F0EDBCF93
:102C9A003CF03C34000E3C1809E6D880FF0E39544B
:102CAA00FF0E3A54FF0E3B54000E3C5404E2D20E7F
:102CBA00006EDB0E76D00C0EDBCF00F00D0EDBCFF4
:102CCA0001F00E0EDBCF02F00F0EDBCF03F000C0D7
:102CDA0038F001C039F002C03AF003C03BF0DFCF50
:102CEA003DF0010EDBCF3EF0020EDBCF3FF0030ECC
:102CFA00DBCF40F053EC7AF0D880190E3854000E2E
:102D0A003954000E3A54000E3B5404E2C30E006ECE
:102D1A00DA0E47D0D9CFE9FFDACFEAFFEECF00F0DB
:102D2A00EECF01F0EECF02F0EFCF03F01F0E3D6EB3
:102D3A00050E3E6E3F6A406A00C038F001C039F0A5
:102D4A0002C03AF003C03BF053EC7AF038C000F00E
:102D5A0039C001F03AC002F03BC003F0D9500C0F61
:102D6A00E96E000EDA20EA6EEE50385CEE50395801
:102D7A00EE503A58EE503B5821E30C0EDBCF04F0EC
:102D8A000D0EDBCF05F00E0EDBCF06F00F0EDBCFFC
:102D9A0007F0045005100610071010E09D0E006E93
:102DAA00DA0E016E026A00C0E6FFE66E02C0E6FFB6
:102DBA001FEC79F0E552E552E55236D0D950080FAA
:102DCA00E96E000EDA20EA6EEECFE6FFEECFE6FFFE
:102DDA00EECFE6FFEFCFE6FFD950040FE96E000E03
:102DEA00DA20EA6EEECFE6FFEECFE6FFEECFE6FFA1
:102DFA00EFCFE6FFD9CFE9FFDACFEAFFEECFE6FF62
:102E0A00EECFE6FFEECFE6FFEFCFE6FF03DB006E85
:102E1A000C0EE15C02E2E16AE552E16E0050070144
:102E2A00E35102E018EC4CF0100EE15C02E2E16AB8
:102E3A00E552E16EE552E5CFDAFFE7CFD9FF12009E
:102E4A00D9CFE6FFDACFE6FFE1CFD9FFE2CFDAFF4B
:102E5A00180EE12402E3E168E652E16EDE6ADE6AF8
:102E6A00DE6ADD6ADD52DD52040EDB6A050EDB6ABC
:102E7A00060EDB6A070EDB6A080EDB6A090EDB6ADE
:102E8A000A0EDB6A0B0EDB6A0C0EDB6A0D0EDB6ABE
:102E9A000E0EDB6A0F0EDB6A100EDB6A110EDB6A9E
:102EAA00120EDB6A130EDB6A140EDB6A150EDB6A7E
:102EBA00160EDB6A170EDB6AE66AD9CFE6FFDACFAF
:102ECA00E6FF070EE66EBCEC55F0E552E552E55218
:102EDA00E552E66AD9500C0FE66E000EDA20E66E6D
:102EEA00060EE66EBCEC55F0E552E552E552E552A7
:102EFA00E66AD950100FE66E000EDA20E66E060E6C
:102F0A00E66EBCEC55F0E552E552E552E552D9CFF2
:102F1A00E9FFDACFEAFFEECF00F0EECF01F0EECF15
:102F2A0002F0EFCF03F0005001100210031002E18B
:102F3A000701B48D100EDBCF00F0110EDBCF01F0CC
:102F4A00120EDBCF02F0130EDBCF03F0D9500C0FB9
:102F5A00E96E000EDA20EA6EEE500026EE500122EB
:102F6A00EE500222EE500322040E00C0DBFF050ED3
:102F7A0001C0DBFF060E02C0DBFF070E03C0DBFF4A
:102F8A000C0EDBCF04F00D0EDBCF05F00E0EDBCFFF
:102F9A0006F00F0EDBCF07F0D950100FE96E000EC6
:102FAA00DA20EA6EEE50045C006EEE500558016EAF
:102FBA00EE500658026EEE500758036E080E00C017
:102FCA00DBFF090E01C0DBFF0A0E02C0DBFF0B0E9E
:102FDA0003C0DBFF040EDBCF39F0050EDBCF3AF07E
:102FEA00060EDBCF3BF0070EDBCF3CF03C34000E85
:102FFA003C1809E6D880000E3954000E3A54000EE7
:10300A003B54000E3C5413E2D950040FE96E000EF3
:10301A00DA20EA6E140EEECFDBFF150EEECFDBFFE1
:10302A00160EEECFDBFF170EEECFDBFF1ED0040E1F
:10303A00DBCF38F0050EDBCF39F0060EDBCF3AF0E6
:10304A00070EDBCF3BF03D683E683F684068F5EC11
:10305A0079F0140E34C0DBFF150E35C0DBFF160EF7
:10306A0036C0DBFF170E37C0DBFFD9CFE9FFDACF57
:10307A00EAFFD880FF0EEE54FF0EEE54FF0EEE5418
:10308A00000EEE5404E2490E006EDB0E74D1140EEB
:10309A00DBCF39F0150EDBCF3AF0160EDBCF3BF063
:1030AA00170EDBCF3CF03C34000E3C1809E6D88002
:1030BA00FF0E3954FF0E3A54FF0E3B54000E3C5497
:1030CA0004E2000E006EDC0E56D1140EDBCF00F0C7
:1030DA00150EDBCF01F0160EDBCF02F0170EDBCF99
:1030EA0003F000C038F001C039F002C03AF003C062
:1030FA003BF0DFCF3DF0010EDBCF3EF0020EDBCF1F
:10310A003FF0030EDBCF40F053EC7AF0D880190E73
:10311A003854000E3954000E3A54000E3B5404E25F
:10312A00190E006EDB0E27D1D9CFE9FFDACFEAFFFD
:10313A00EECF00F0EECF01F0EECF02F0EFCF03F0CA
:10314A001F0E3D6E050E3E6E3F6A406A00C038F0A3
:10315A0001C039F002C03AF003C03BF053EC7AF0F8
:10316A0038C000F039C001F03AC002F03BC003F0A9
:10317A00D950140FE96E000EDA20EA6EEE50385C70
:10318A00EE503958EE503A58EE503B5815E3140EAB
:10319A00DBCF04F0150EDBCF05F0160EDBCF06F001
:1031AA00170EDBCF07F0045005100610071004E0D5
:1031BA00F30E006EDA0EDFD0080EDBCF39F0090EFF
:1031CA00DBCF3AF00A0EDBCF3BF00B0EDBCF3CF045
:1031DA003C34000E3C1809E6D880000E3954000E23
:1031EA003A54000E3B54000E3C5413E2D950080FD7
:1031FA00E96E000EDA20EA6E140EEECFDBFF150E32
:10320A00EECFDBFF160EEECFDBFF170EEECFDBFFA6
:10321A001ED0080EDBCF38F0090EDBCF39F00A0ECC
:10322A00DBCF3AF00B0EDBCF3BF03D683E683F68E0
:10323A004068F5EC79F0140E34C0DBFF150E35C08A
:10324A00DBFF160E36C0DBFF170E37C0DBFF140E8E
:10325A00DBCF39F0150EDBCF3AF0160EDBCF3BF0A1
:10326A00170EDBCF3CF03C34000E3C1809E6D88040
:10327A00FF0E3954FF0E3A54FF0E3B54000E3C54D5
:10328A0004E2D20E006EDB0E76D0140EDBCF00F015
:10329A00150EDBCF01F0160EDBCF02F0170EDBCFD7
:1032AA0003F000C038F001C039F002C03AF003C0A0
:1032BA003BF0DFCF3DF0010EDBCF3EF0020EDBCF5D
:1032CA003FF0030EDBCF40F053EC7AF0D880190EB2
:1032DA003854000E3954000E3A54000E3B5404E29E
:1032EA00C30E006EDA0E47D0D9CFE9FFDACFEAFF74
:1032FA00EECF00F0EECF01F0EECF02F0EFCF03F009
:10330A001F0E3D6E050E3E6E3F6A406A00C038F0E1
:10331A0001C039F002C03AF003C03BF053EC7AF036
:10332A0038C000F039C001F03AC002F03BC003F0E7
:10333A00D950140FE96E000EDA20EA6EEE50385CAE
:10334A00EE503958EE503A58EE503B5821E3140EDD
:10335A00DBCF04F0150EDBCF05F0160EDBCF06F03F
:10336A00170EDBCF07F0045005100610071010E007
:10337A009D0E006EDA0E016E026A00C0E6FFE66E6E
:10338A0002C0E6FF1FEC79F0E552E552E55236D06D
:10339A000701B45133E1D950080FE96E000EDA2063
:1033AA00EA6EEECFE6FFEECFE6FFEECFE6FFEFCF17
:1033BA00E6FFD950040FE96E000EDA20EA6EEECF6E
:1033CA00E6FFEECFE6FFEECFE6FFEFCFE6FFD9CF7F
:1033DA00E9FFDACFEAFFEECFE6FFEECFE6FFEECF68
:1033EA00E6FFEFCFE6FF16D8006E0C0EE15C02E2B4
:1033FA00E16AE552E16E005018EC4CF0180EE15CFF
:10340A0002E2E16AE552E16EE552E5CFDAFFE7CF83
:10341A00D9FF1200D9CFE6FFDACFE6FFE1CFD9FF15
:10342A00E2CFDAFF370EE12402E3E168E652E16E09
:10343A00DE6ADE6ADE6ADD6ADD52DD52040EDB6AAE
:10344A00050EDB6A060EDB6A070EDB6A080EDB6A0C
:10345A00090EDB6A0A0EDB6A0B0EDB6A0C0EDB6AEC
:10346A000D0EDB6A0E0EDB6A0F0EDB6AF60EDBCF81
:10347A0000F0F70EDBCF01F0F80EDBCF02F0F90E09
:10348A00DBCF03F000500110021003103FE1F20EEF
:10349A00DBCF04F0F30EDBCF05F0F40EDBCF06F042
:1034AA00F50EDBCF07F004500510061007102EE1C9
:1034BA00020EF36E100EF3CFDBFFFA0EDBCF00F035
:1034CA00FB0EDBCF01F0FC0EDBCF02F0FD0EDBCFF3
:1034DA0003F0190E3D6E3E6A3F6A406A00C038F03A
:1034EA0001C039F002C03AF003C03BF0F5EC79F0C4
:1034FA002A0E34C0DBFF2B0E35C0DBFF2C0E36C084
:10350A00DBFF2D0E37C0DBFF37EF1FF02A0EDB6A19
:10351A002B0EDB6A2C0EDB6A2D0EDB6A290EDB6AA8
:10352A008D908B92D950F60FE96EFF0EDA20EA6E73
:10353A00D890030EEB50000A08E6000EEE5C000E6F
:10354A00EE58000EEE58000EEE5825E2290EDB501A
:10355A000209E76E290EE7CFDBFFF60EDBCF38F064
:10356A00F70EDBCF39F0F80EDBCF3AF0F90EDBCFEE
:10357A003BF03D683E683F684068F5EC79F0F60E2E
:10358A0034C0DBFFF70E35C0DBFFF80E36C0DBFFB9
:10359A00F90E37C0DBFFD950F20FE96EFF0EDA20C1
:1035AA00EA6ED890030EEB50000A08E6000EEE5CB5
:1035BA00000EEE58000EEE58000EEE5825E2290EC7
:1035CA00DB500809E76E290EE7CFDBFFF20EDBCFEF
:1035DA0038F0F30EDBCF39F0F40EDBCF3AF0F50E0C
:1035EA00DBCF3BF03D683E683F684068F5EC79F018
:1035FA00F20E34C0DBFFF30E35C0DBFFF40E36C02B
:10360A00DBFFF50E37C0DBFFD950F60FE96EFF0E70
:10361A00DA20EA6ED890030EEB50000A08E6FF0E95
:10362A00EE5CFF0EEE58010EEE58000EEE5801E366
:10363A00DFD0FA0EDBCF00F0FB0EDBCF01F0FC0E81
:10364A00DBCF02F0FD0EDBCF03F0190E3D6E3E6AB2
:10365A003F6A406A00C038F001C039F002C03AF04F
:10366A0003C03BF0F5EC79F0040E34C0DBFF050E25
:10367A0035C0DBFF060E36C0DBFF070E37C0DBFFA7
:10368A00F60EDBCF00F0F70EDBCF01F0F80EDBCF42
:10369A0002F0F90EDBCF03F00F0E1F0B07E0D890F4
:1036AA000036013602360336E806F9E100C038F082
:1036BA0001C039F002C03AF003C03BF0040EDBCF80
:1036CA003DF0050EDBCF3EF0060EDBCF3FF0070ED6
:1036DA00DBCF40F053EC7AF038C0DEFF39C0DEFFB2
:1036EA003AC0DEFF3BC0DDFFDD52DD52F60EDBCF16
:1036FA0000F0F70EDBCF01F0F80EDBCF02F0F90E87
:10370A00DBCF03F00F0E1F0B07E0D890003601360F
:10371A0002360336E806F9E100C038F001C039F094
:10372A0002C03AF003C03BF0040EDBCF3DF0050EB9
:10373A00DBCF3EF0060EDBCF3FF0070EDBCF40F0CB
:10374A0053EC7AF0080E34C0DBFF090E35C0DBFFFC
:10375A000A0E36C0DBFF0B0E37C0DBFFD950FA0F5B
:10376A00E96EFF0EDA20EA6ED8801E0EEE54000EC5
:10377A00EE54000EEE54000EEE5401E37CD0080E17
:10378A00DBCF00F0090EDBCF01F00A0EDBCF02F02F
:10379A000B0EDBCF03F0100E1F0B07E0D89000369C
:1037AA00013602360336E806F9E100C038F001C0F6
:1037BA0039F002C03AF003C03BF0040EDBCF3DF013
:1037CA00050EDBCF3EF0060EDBCF3FF0070EDBCF58
:1037DA0040F053EC7AF00C0E38C0DBFF0D0E39C006
:1037EA00DBFF0E0E3AC0DBFF0F0E3BC0DBFF43D000
:1037FA00F60EDBCF00F0F70EDBCF01F0F80EDBCFD1
:10380A0002F0F90EDBCF03F000C038F001C039F046
:10381A0002C03AF003C03BF0FA0EDBCF3DF0FB0EDC
:10382A00DBCF3EF0FC0EDBCF3FF0FD0EDBCF40F0EE
:10383A0053EC7AF00F0ED890383639363A363B3692
:10384A00E806F9E1190E3D6E3E6A3F6A406A53EC9A
:10385A007AF038C0DEFF39C0DEFF3AC0DEFF3BC077
:10386A00DDFFDD52DD520C0EDB6A0D0EDB6A0E0E39
:10387A00DB6A0F0EDB6AD9CFE9FFDACFEAFFD8801D
:10388A00000EEE54800EEE54000EEE54000EEE546E
:10389A0027E2D9CFE9FFDACFEAFFEECFE6FFEECF94
:1038AA00E6FFEECFE6FFEFCFE6FF680E006EDA0E18
:1038BA00016E026A00C0E6FFE66E02C0E6FF1FEC78
:1038CA0079F0036E070EE15C02E2E16AE552E16E0D
:1038DA000350DE6A800EDE6EDE6ADD6ADD52DD527C
:1038EA00D9CFE9FFDACFEAFFEECF00F0EECF01F051
:1038FA00EECF02F0EFCF03F00050011002100310D8
:10390A0027E1F60EDBCF04F0F70EDBCF05F0F80E59
:10391A00DBCF06F0F90EDBCF07F0045005100610D6
:10392A00071016E03D0E006EDA0E016E026A00C044
:10393A00E6FFE66E02C0E6FF1FEC79F0E552E552BB
:10394A00E552010EDE6EDE6ADE6ADD6ADD52DD52A6
:10395A00D950FA0FE96EFF0EDA20EA6ED8801E0EF1
:10396A00EE54000EEE54000EEE54000EEE5429E210
:10397A00D9CFE9FFDACFEAFFEECF04F0EECF05F0B8
:10398A00EECF06F0EFCF07F0100E1F0B07E0D8902E
:10399A000436053606360736E806F9E1D9500C0F23
:1039AA00E96E000EDA20EA6E0450EE24006E05502D
:1039BA00EE20016E0650EE20026E0750EE20036ED6
:1039CA0016D0D9CFE9FFDACFEAFFEECF00F0EECF7B
:1039DA0001F0EECF02F0EFCF03F0100E1F0B07E05D
:1039EA00D8900036013602360336E806F9E100C0FF
:1039FA00DFFF010E01C0DBFF020E02C0DBFF030E78
:103A0A0003C0DBFFD9CFE9FFDACFEAFF110EEECF11
:103A1A00DBFF120EEECFDBFF130EEECFDBFF140E31
:103A2A00EECFDBFFD950F60FE96EFF0EDA20EA6E11
:103A3A00210EEECFDBFF220EEECFDBFF230EEECF01
:103A4A00DBFF240EEECFDBFF190EDB6A1A0EDB6AF0
:103A5A001B0EDB6A1C0EDB6AD950F20FE96EFF0EF1
:103A6A00DA20EA6ED890030EEB50000A08E6FF0E41
:103A7A00EE5CFF0EEE58010EEE58000EEE5801E312
:103A8A00B8D0F20EDBCF00F0F30EDBCF01F0F40E6C
:103A9A00DBCF02F0F50EDBCF03F00F0E1F0B07E0B2
:103AAA00D8900036013602360336E806F9E100C03E
:103ABA0038F001C039F002C03AF003C03BF0040EFE
:103ACA00DBCF3DF0050EDBCF3EF0060EDBCF3FF03D
:103ADA00070EDBCF40F053EC7AF038C0DEFF39C076
:103AEA00DEFF3AC0DEFF3BC0DDFFDD52DD52F20EE3
:103AFA00DBCF00F0F30EDBCF01F0F40EDBCF02F0E8
:103B0A00F50EDBCF03F00F0E1F0B07E0D89000363F
:103B1A00013602360336E806F9E100C038F001C082
:103B2A0039F002C03AF003C03BF0040EDBCF3DF09F
:103B3A00050EDBCF3EF0060EDBCF3FF0070EDBCFE4
:103B4A0040F053EC7AF0080E34C0DBFF090E35C0A2
:103B5A00DBFF0A0E36C0DBFF0B0E37C0DBFFD95086
:103B6A00FA0FE96EFF0EDA20EA6ED8801E0EEE54C6
:103B7A00000EEE54000EEE54000EEE5401E37CD01B
:103B8A00080EDBCF00F0090EDBCF01F00A0EDBCF07
:103B9A0002F00B0EDBCF03F0100E1F0B07E0D890DC
:103BAA000036013602360336E806F9E100C038F07D
:103BBA0001C039F002C03AF003C03BF0040EDBCF7B
:103BCA003DF0050EDBCF3EF0060EDBCF3FF0070ED1
:103BDA00DBCF40F053EC7AF00C0E38C0DBFF0D0E51
:103BEA0039C0DBFF0E0E3AC0DBFF0F0E3BC0DBFF16
:103BFA0043D0F20EDBCF00F0F30EDBCF01F0F40E70
:103C0A00DBCF02F0F50EDBCF03F000C038F001C0C5
:103C1A0039F002C03AF003C03BF0FA0EDBCF3DF0B8
:103C2A00FB0EDBCF3EF0FC0EDBCF3FF0FD0EDBCF11
:103C3A0040F053EC7AF00F0ED890383639363A36CF
:103C4A003B36E806F9E1190E3D6E3E6A3F6A406A64
:103C5A0053EC7AF038C0DEFF39C0DEFF3AC0DEFF2F
:103C6A003BC0DDFFDD52DD520C0EDB6A0D0EDB6A56
:103C7A000E0EDB6A0F0EDB6AD9CFE9FFDACFEAFF55
:103C8A00D880000EEE54800EEE54000EEE54000E54
:103C9A00EE5427E2D9CFE9FFDACFEAFFEECFE6FF0B
:103CAA00EECFE6FFEECFE6FFEFCFE6FF080E006E9F
:103CBA00DA0E016E026A00C0E6FFE66E02C0E6FF97
:103CCA001FEC79F0036E070EE15C02E2E16AE5524D
:103CDA00E16E0350DE6A800EDE6EDE6ADD6ADD5258
:103CEA00DD52D9CFE9FFDACFEAFFEECF00F0EECF0F
:103CFA0001F0EECF02F0EFCF03F0005001100210F6
:103D0A00031027E1F20EDBCF04F0F30EDBCF05F050
:103D1A00F40EDBCF06F0F50EDBCF07F004500510EA
:103D2A000610071016E0DD0E006ED90E016E026A4B
:103D3A0000C0E6FFE66E02C0E6FF1FEC79F0E5522E
:103D4A00E552E552010EDE6EDE6ADE6ADD6ADD529A
:103D5A00DD52D950FA0FE96EFF0EDA20EA6ED880EA
:103D6A001E0EEE54000EEE54000EEE54000EEE54EB
:103D7A0029E2D9CFE9FFDACFEAFFEECF04F0EECF9E
:103D8A0005F0EECF06F0EFCF07F0100E1F0B07E09D
:103D9A00D8900436053606360736E806F9E1D950D2
:103DAA000C0FE96E000EDA20EA6E0450EE24006E63
:103DBA000550EE20016E0650EE20026E0750EE20EE
:103DCA00036E16D0D9CFE9FFDACFEAFFEECF00F0C3
:103DDA00EECF01F0EECF02F0EFCF03F0100E1F0B83
:103DEA0007E0D8900036013602360336E806F9E1D4
:103DFA0000C0DFFF010E01C0DBFF020E02C0DBFFC5
:103E0A00030E03C0DBFFD9CFE9FFDACFEAFF150EB5
:103E1A00EECFDBFF160EEECFDBFF170EEECFDBFF8A
:103E2A00180EEECFDBFFD950F20FE96EFF0EDA2043
:103E3A00EA6E250EEECFDBFF260EEECFDBFF270E56
:103E4A00EECFDBFF280EEECFDBFF1D0EDB6A1E0E68
:103E5A00DB6A1F0EDB6A200EDB6A010EF36E100EA0
:103E6A00F3CFDBFF05012751FDE0100EDBCF34F560
:103E7A00110EDBCF35F5120EDBCF36F5130EDBCF85
:103E8A0037F5140EDBCF38F5150EDBCF39F5160EE4
:103E9A00DBCF3AF5170EDBCF3BF5180EDBCF3CF53F
:103EAA00190EDBCF3DF51A0EDBCF3EF51B0EDBCF2D
:103EBA003FF51C0EDBCF40F51D0EDBCF41F51E0E84
:103ECA00DBCF42F51F0EDBCF43F5200EDBCF44F5E7
:103EDA00210EDBCF45F5220EDBCF46F5230EDBCFD5
:103EEA0047F5240EDBCF48F5250EDBCF49F5260E24
:103EFA00DBCF4AF5270EDBCF4BF5280EDBCF4CF58F
:103F0A00290EDBCF4DF52A0EDBCF4EF52B0EDBCF7C
:103F1A004FF52C0EDBCF50F52D0EDBCF51F52E0EC3
:103F2A00DBCF52F52F0EDBCF53F5300EDBCF54F536
:103F3A00310EDBCF55F5320EDBCF56F5330EDBCF24
:103F4A0057F5340EDBCF58F5350EDBCF59F5360E63
:103F5A00DBCF5AF5276B370EE15C02E2E16AE552E4
:103F6A00E16EE552E5CFDAFFE7CFD9FF1200D9CFEC
:103F7A00E6FFDACFE6FFE1CFD9FFE2CFDAFF110E93
:103F8A00E12402E3E168E652E16EDF6A010EDB6AD0
:103F9A00020EDB6A030EDB6A040EDB6A050EDB6ABD
:103FAA00060EDB6A070EDB6A080EDB6A090EDB6A9D
:103FBA000A0EDB6A0B0EDB6A0C0EDB6A0D0EDB6A7D
:103FCA000E0EDB6A0F0EDB6A100EDB6A0501275143
:103FDA0002E1340502E0000502E1010EDF6E34055C
:103FEA002BE1346B090E45C5DBFF0A0E46C5DBFF24
:103FFA000B0E47C5DBFF0C0E48C5DBFF0D0E49C58E
:10400A00DBFF0E0E4AC5DBFF0F0E4BC5DBFF100EA2
:10401A004CC5DBFF456B466B476B486B496B4A6B7C
:10402A004B6B4C6B3D6B3E6B3F6B406B416B426B1A
:10403A00436B446B010E276F000529E1006B010EEB
:10404A0011C5DBFF020E12C5DBFF030E13C5DBFF32
:10405A00040E14C5DBFF050E15C5DBFF060E16C5DB
:10406A00DBFF070E17C5DBFF080E18C5DBFF116B58
:10407A00126B136B146B156B166B176B186B096B42
:10408A000A6B0B6B0C6B0D6B0E6B0F6B106BD950B5
:10409A00050FE96E000EDA20EA6EEECFE6FFEECFEC
:1040AA00E6FFEECFE6FFEFCFE6FFD950010FE96E4C
:1040BA00000EDA20EA6EEECFE6FFEECFE6FFEECF95
:1040CA00E6FFEFCFE6FFD9500D0FE96E000EDA20BA
:1040DA00EA6EEECFE6FFEECFE6FFEECFE6FFEFCFDA
:1040EA00E6FFD950090FE96E000EDA20EA6EEECF2C
:1040FA00E6FFEECFE6FFEECFE6FFEFCFE6FFDFCF3C
:10410A00E6FFE66AC80E006ED90E016E026A00C0AA
:10411A00E6FFE66E02C0E6FF1FEC79F0036E150EAD
:10412A00E15C02E2E16AE552E16E035018EC4CF000
:10413A00110EE15C02E2E16AE552E16EE552E5CF79
:10414A00DAFFE7CFD9FF1200D8C500F0016A00BE36
:10415A00016800C0E6FF01C0E6FFC30E026ED90E79
:10416A00036E046A02C0E6FFE66E04C0E6FF1FECB7
:10417A0079F0056E050EE15C02E2E16AE552E16E54
:10418A00055018EF4CF0D9CFE6FFDACFE6FFE1CFC2
:10419A00D9FFE2CFDAFFE652E652DE6ADD6A010EA5
:1041AA00E66ED9CFE6FFDACFE6FF030EE66EBCEC89
:1041BA0055F0E552E552E552E5520701B45115E1D1
:1041CA000501D80506E1DECFE6FFDDCFE6FFE66AA8
:1041DA0006D0DECFE6FFDDCFE6FF010EE66E9ED803
:1041EA00E552E552E55218EC4CF0E552E552E5523B
:1041FA00E5CFDAFFE7CFD9FF1200D9CFE6FFDACF52
:10420A00E6FFE1CFD9FFE2CFDAFFE652E652E65205
:10421A00E652E652DF6A010EDB6A020EDB6A010E23
:10422A00F36E030EF3CFDBFFE66AD9CFE6FFDACFF0
:10423A00E6FF010EE66EBCEC55F0E552E552E5529A
:10424A00E552010EE66ED950010FE66E000EDA2035
:10425A00E66E030EE66EBCEC55F0E552E552E55209
:10426A00E552010EE66ED950030FE66E000EDA2013
:10427A00E66E010EE66EBCEC55F0E552E552E552EB
:10428A00E552E76E040EE7CFDBFF0701B4513AE1CE
:10429A00030EDB50070805E2010EF36E030EF3CF9F
:1042AA00DBFFDF50010802E2010EDF6E030EDB5076
:1042BA00030F0E01B65D18E0000EE66EE66AE66EC2
:1042CA00E66AB6CEE6FFE66EE66A4EEC75F0006E7A
:1042DA00070EE15C02E2E16AE552E16E0050030E6C
:1042EA00DB50030F0E01B66F010EDBCFE6FF020EA5
:1042FA00DBCFE6FFDFCFE6FF11D8E552E552E55204
:10430A0018EC4CF0050EE15C02E2E16AE552E16E5E
:10431A00E552E5CFDAFFE7CFD9FF1200D9CFE6FFA2
:10432A00DACFE6FFE1CFD9FFE2CFDAFFE652E65273
:10433A00E652E652FD0EDB040BE1B0CEDEFFB1CE53
:10434A00DDFF020EB2CEDBFF030EB3CEDBFF0AD0D7
:10435A00AECEDEFFAFCEDDFF020EB4CEDBFF030E24
:10436A00B5CEDBFFFB0EDBCFE6FFFC0EDBCFE6FFB5
:10437A00020EDBCFE6FF030EDBCFE6FFB6CEE6FF8B
:10438A00DECFE6FFDDCFE6FF4EEC75F0006E070EDE
:10439A00E15C02E2E16AE552E16E0050040EE15C82
:1043AA0002E2E16AE552E16EE552E5CFDAFFE7CFD4
:1043BA00D9FF1200D9CFE6FFDACFE6FFE1CFD9FF66
:1043CA00E2CFDAFFE652E652E652E66AD9CFE6FFD4
:1043DA00DACFE6FF010EE66EBCEC55F0E552E55287
:1043EA00E552E552E76E020EE7CFDBFFDB5039E11B
:1043FA000701B45165E10501D75103E0020ED75D0B
:10440A0028E1DF50000821E2D75101E18D90DF0455
:10441A0003E18D848D82898C020EDF5C03E18D8439
:10442A008D82899C030EDF5C03E18D948D82899CC9
:10443A00040EDF5C03E18D848D92899C050EDF5C9E
:10444A0010E18D948D92899C0CD0D7510AE18D8010
:10445A0008D0D70506E1DF50000802E28C9201D0AD
:10446A008C82010EE66ED950010FE66E000EDA203C
:10447A00E66E010EE66EBCEC55F0E552E552E552E9
:10448A00E552E76E020EE7CFDBFFDB5017E10701CB
:10449A00B45116E10501D75108E1010EDB500008BD
:1044AA0002E28B920BD08B8209D0D70507E1010E6D
:1044BA00DB50000802E2899201D0898218EC4CF0A4
:1044CA00E552E552E552E552E5CFDAFFE7CFD9FFEB
:1044DA001200FE0E0501D95DFF0EDA59FF0EDB59F7
:1044EA00FF0EDC5905E2D92B000EDA23DB23DC238D
:1044FA0018EF4CF00501D951DA11DB11DC1105E096
:10450A00D907000EDA5BDB5BDC5B18EF4CF0D9CF26
:10451A00E6FFDACFE6FFE1CFD9FFE2CFDAFFE652D4
:10452A00E652E652E652E652E66AD9CFE6FFDACF1B
:10453A00E6FF070EE66EBCEC55F0E552E552E55291
:10454A00E552E76E040EE7CFDBFFDB500BE1DFCF6E
:10455A00D9F5010EDBCFDAF5020EDBCFDBF5030E60
:10456A00DBCFDCF518EC4CF0050EE15C02E2E16A07
:10457A00E552E16EE552E5CFDAFFE7CFD9FF120047
:10458A00D9C5E6FFDAC5E6FFDBC5E6FFDCC5E6FF0F
:10459A00BA0E006ED90E016E026A00C0E6FFE66E20
:1045AA0002C0E6FF1FEC79F0036E070EE15C02E23F
:1045BA00E16AE552E16E035018EF4CF0E66ADD0E4F
:1045CA00E66E050EE66E010EE66EBCEC55F0E5529F
:1045DA00E552E552E5520701B45101E0120018EF25
:1045EA004CF0DDC500F0016A00BE016800C0E6FFBC
:1045FA0001C0E6FFB30E026ED90E036E046A02C052
:10460A00E6FFE66E04C0E6FF1FEC79F0056E050EC4
:10461A00E15C02E2E16AE552E16E055018EF4CF006
:10462A00DEC500F0016A00BE016800C0E6FF01C0F5
:10463A00E6FFAD0E026ED90E036E046A02C0E6FFF3
:10464A00E66E04C0E6FF1FEC79F0056E050EE15C2C
:10465A0002E2E16AE552E16E05500501DE6B18EFF0
:10466A004CF09DBCFED716C1E6FF17C1E6FF00C19C
:10467A00E6FF01C1E6FFA10E006ED90E016E026AC5
:10468A0000C0E6FFE66E02C0E6FF1FEC79F0036E9B
:10469A00070EE15C02E2E16AE552E16E035018EFAF
:1046AA004CF0D9CFE6FFDACFE6FFE1CFD9FFE2CF70
:1046BA00DAFFE652E652E652E652E652DF6A010EA7
:1046CA00DB6A020EDB6A030EDB6AE66AD9CFE6FF13
:1046DA00DACFE6FF010EE66EBCEC55F0E552E55284
:1046EA00E552E552010EE66ED950010FE66E000E54
:1046FA00DA20E66E030EE66EBCEC55F0E552E552A2
:10470A00E552E552E76E040EE7CFDBFF010EE66ED7
:10471A00D950030FE66E000EDA20E66E010EE66E41
:10472A00BCEC55F0E552E552E552E5520701B451A9
:10473A0001E088D0D950010FE96E000EDA20EA6E46
:10474A00FF0ED880EE54030EED5407E2010EDB682B
:10475A00030EF36E020EF3CFDBFFDF50010802E215
:10476A00010EDF6E030EDB50010805E2010EF36E47
:10477A00030EF3CFDBFFDF0409E1040EDB5003086D
:10478A0005E10501E16B020EE26F06D0010EDBCFF7
:10479A00E1F5020EDBCFE2F5CAB415D0CB68FC0E08
:1047AA00CA140009CA6E9D920F0152815293F00EEB
:1047BA00BA140C09BA6E3F0EBA140009BA6E0E0189
:1047CA000E0ECC6FCA84030EDB502AE1DF5023E0C1
:1047DA00E1C500F0E2C501F0D89001320032D8906C
:1047EA00013200320050BB6EE1C502F0E2C503F0AF
:1047FA00040ED89002360336E804FBE1300E0216A6
:10480A00000E0316CF0EBA1400010210006E03C088
:10481A0001F0E85003D0BB6ACF0EBA14BA6E10D0BA
:10482A0005012751FDE0E1C559F5E2C55AF54E6B80
:10483A004F6B506B516BDFCF58F5040E346F276BFB
:10484A0018EC4CF0050EE15C02E2E16AE552E16E19
:10485A00E552E5CFDAFFE7CFD9FF12001200D9CF30
:10486A00E6FFDACFE6FFE1CFD9FFE2CFDAFF2B0E80
:10487A00E12402E3E168E652E16EDF6A010EDB6AD7
:10488A00020EDB6A030EDB6AF29E040E00C5DBFF32
:10489A00050E01C5DBFF060E02C5DBFF070E03C5C9
:1048AA00DBFF080E04C5DBFF090E05C5DBFF0A0E98
:1048BA0006C5DBFF0B0E07C5DBFF0C0E08C5DBFFC9
:1048CA000D0E09C5DBFF0E0E0AC5DBFF0F0E0BC569
:1048DA00DBFF100E0CC5DBFF110E0DC5DBFF120E40
:1048EA000EC5DBFF130E0FC5DBFF140E10C5DBFF71
:1048FA00150E11C5DBFF160E12C5DBFF170E13C509
:10490A00DBFF180E14C5DBFF190E15C5DBFF1A0EE7
:10491A0016C5DBFF1B0E17C5DBFF1C0E18C5DBFF18
:10492A001D0E19C5DBFF1E0E1AC5DBFF1F0E1BC5A8
:10493A00DBFF200E1CC5DBFF210E1DC5DBFF220E8F
:10494A001EC5DBFF230E1FC5DBFF240E20C5DBFFC0
:10495A00250E21C5DBFF260E22C5DBFF270E23C548
:10496A00DBFF280E24C5DBFF290E25C5DBFF2A0E37
:10497A0026C5DBFFF28E1E0EDBCF00F01F0EDBCF4B
:10498A0001F0200EDBCF02F0210EDBCF03F0005046
:10499A0001100210031002E0010EDF6E040EDB505C
:1049AA0002E0010EDF6E0501275106E1010EDF6EFE
:1049BA00F36E030EF3CFDBFFDF5014E0150EDBCFEF
:1049CA0000F0160EDBCF01F0170EDBCF02F0180E47
:1049DA00DBCF03F0005001100210031003E0DE5297
:1049EA00010EDD6EDF5016E0190EDBCF00F01A0E55
:1049FA00DBCF01F01B0EDBCF02F01C0EDBCF03F086
:104A0A00005001100210031005E0010EF36E020EB1
:104A1A00F3CFDBFF030EDBCFE6FFE66A020EDBCF46
:104A2A00E6FFE66A010EDBCFE6FFE66ADFCFE6FFC6
:104A3A00E66A900E006ED90E016E026A00C0E6FFA9
:104A4A00E66E02C0E6FF1FEC79F0036E0B0EE15C26
:104A5A0002E2E16AE552E16E03502B0EE15C02E2EA
:104A6A00E16AE552E16EE552E5CFDAFFE7CFD9FF19
:104A7A001200D9CFE6FFDACFE6FFE1CFD9FFE2CFC6
:104A8A00DAFF080EE12402E3E168E652E16EF29EE3
:104A9A0028C5DFFF010E29C5DBFF020E2AC5DBFF91
:104AAA00030E2BC5DBFF040E2CC5DBFF050E2DC53F
:104ABA00DBFF060E2EC5DBFF070E2FC5DBFFF28ECE
:104ACA00D950040FE96E000EDA20EA6EEECFE6FF47
:104ADA00EECFE6FFEECFE6FFEFCFE6FFD9CFE9FF55
:104AEA00DACFEAFFEECFE6FFEECFE6FFEECFE6FF44
:104AFA00EFCFE6FF860E006ED90E016E026A00C085
:104B0A00E6FFE66E02C0E6FF1FEC79F0036E0B0EBD
:104B1A00E15C02E2E16AE552E16E035018EC4CF006
:104B2A00080EE15C02E2E16AE552E16EE552E5CF88
:104B3A00DAFFE7CFD9FF1200F29E0501286B296B35
:104B4A002A6B2B6B2C6B2D6B2E6B2F6BF28E18EF47
:104B5A004CF00201000000000001320000000000D9
:104B6A000180004D00000002000000000000013238
:104B7A00000000000001A700FBFFDFFF015700EF64
:104B8A00FF0400014E00F2FF0700014C00F3FF088A
:104B9A0000014A00F5FF0A00014400F8FF0B00017A
:104BAA004800FAFF0D00014E00FCFF0F0001500003
:104BBA00FFFF100001320000000A00012E0002006F
:104BCA00090001330002000A00012D000400080058
:104BDA00012D0004000800012F0005000800013122
:104BEA000007000700012E00070006000132000836
:104BFA00000600013300090005000136000A00041E
:104C0A00000134000A0003000139000B000300010F
:104C1A003D000C0002000141000D000100014600A8
:104C2A000E0001000146000E00FFFF0141000D00C9
:104C3A00FFFF013D000C00FEFF013E000C00FDFFDE
:104C4A000139000B00FDFF0136000A00FCFF0133A9
:104C5A00000900FBFF0132000800FAFF01350008D5
:104C6A0000F9FF012E000600F9FF012E000600F9E7
:104C7A00FF012D000400F8FF012D000400F8FF01D8
:104C8A002E000200F7FF012E000200F7FF0132009A
:104C9A000000F6FF012D000000F7FF012E00FEFFC5
:104CAA00F7FF012900FEFFF8FF012B00FDFFF8FFC7
:104CBA00012F00FBFFF8FF012B00FBFFF9FF013179
:104CCA0000F9FFF9FF012E00F9FFFAFF013200F89F
:104CDA00FFFAFF013300F7FFFBFF013600F6FFFC86
:104CEA00FF013900F5FFFDFF013900F5FFFDFF0166
:104CFA003D00F4FFFEFF014100F3FFFFFF01460004
:104D0A00F2FFFFFF013200F6FF010001C6020000B8
:104D1A008E00015B00EEFFFEFF015100F0FFFDFF78
:104D2A00014800F3FFFAFF014100F5FFF9FF013CDA
:104D3A0000F7FFF8FF013A00FAFFF6FF013600FC20
:104D4A00FFF6FF013C00FFFFF4FF0128000100F815
:104D5A00FF0129000200F8FF0126000300F9FF0104
:104D6A002B000500F9FF012E000700FAFF012F00B2
:104D7A000800FBFF0133000900FBFF013F000C00A4
:104D8A00FCFF01000000000000020100000000001A
:104D9A000132000000000001CE003F006A0002005C
:104DAA0000000000000132000000000001120200B1
:104DBA000096FF0141000D000100013E000C0003B6
:104DCA00000134000A000300012F00080005000159
:104DDA0040000A000800013D0007000A00011B000C
:104DEA0002000500011B0002000500013C00010051
:104DFA000C00013700FFFF0B00012F00FDFF090027
:104E0A00013600FAFF0900013500F9FF0800013DEB
:104E1A0000F6FF0700013C00F5FF0500014400F31E
:104E2A00FF0400014600F2FF01000100000000003B
:104E3A000002010000000000013200000000000131
:104E4A00900164FF4AFF02000000000000013200E6
:104E5A000000000001A200FBFFE0FF012D00F7FFA8
:104E6A00FFFF012600F9FFFDFF011D00FBFFFDFF0B
:104E7A00012000FBFFFCFF012700FBFFFAFF012BCB
:104E8A0000FDFFF8FF012E00FEFFF7FF013200FFD1
:104E9A00FFF6FF0132000100F6FF0133000200F6BF
:104EAA00FF012B000300F8FF0127000500FAFF01AC
:104EBA002A000600FAFF012B000700FBFF012B0066
:104ECA000800FDFF012F000900FDFF01600013002B
:104EDA00FEFF019B001F000000012B00F9FF0500E7
:104EEA00012A00FAFF0600012700FBFF060001283D
:104EFA0000FCFF0700012400FCFF0600012400FE5D
:104F0A00FF0700012800FFFF0800012800FFFF0833
:104F1A0000012D0001000900012D00010009000116
:104F2A002F0003000900012D0004000800012800D9
:104F3A0004000700012E0006000700012E000700EA
:104F4A0006000132000800060001330009000500CE
:104F5A00013100090004000136000A00040001348E
:104F6A00000A000300016B0015000400017300171A
:104F7A00000100015000100000000151001000FE65
:104F8A00FF0148000E00FDFF014A000E00FBFF0171
:104F9A004A000E00FBFF0141000B00F9FF0140002F
:104FAA000A00F8FF0139000800F8FF013D00070078
:104FBA00F6FF013C000500F5FF0138000200F5FF8D
:104FCA000141000100F3FF0128000000F8FF012958
:104FDA0000FEFFF8FF012400FEFFF9FF012800FC94
:104FEA00FFF9FF012800FCFFF9FF012E00FAFFF983
:104FFA00FF012E00F9FFFAFF012B00F9FFFBFF0169
:10500A0087001B0000000196000000E2FF01DE039A
:10501A003AFF0000017D00E7FF0000016900EBFF95
:10502A000200015600EFFF0300014400F3FF0400F1
:10503A00013800F6FF0500013D00F6FF07000135C3
:10504A0000F8FF0700013D00F9FF0A00013A00FAE3
:10505A00FF0A00013F00FCFF0C00013D00FEFF0CAF
:10506A0000014600FFFF0E00015000010010000180
:10507A004E0004000F0001480006000D0001440024
:10508A0008000B00012000040005000127000600AB
:10509A0005000122000600030001260007000300A4
:1050AA00012400070002000129000800020001553E
:1050BA0000110001000100000000000002010000D0
:1050CA000000000132000000000001EA008A00E549
:1050DA00FF02000000000000013200000000000191
:1050EA006900EBFFFFFF015B00EEFFFDFF014F00D0
:1050FA00F1FFFBFF012200FAFFFDFF012200FAFF88
:10510A00FDFF013C00F7FFF8FF013900F9FFF7FF47
:10511A00013400FDFFF6FF013300FEFFF6FF013800
:10512A00000200F5FF0134000300F6FF0139000711
:10513A0000F7FF013C000900F8FF011D000500FD12
:10514A00FF0126000700FDFF014A000E00FBFF01D8
:10515A005B001200FDFF0164001400FFFF01640000
:10516A001400010001560011000300014F000F0056
:10517A0005000145000C000700013C000900080079
:10518A000139000700090001310004000900013754
:10519A000001000B00013200FFFF0A00013600FC8B
:1051AA00FF0A00013900F9FF0900013C00F7FF0876
:1051BA0000014300F4FF0600014A00F2FF05000166
:1051CA005600EFFF0300015F00EDFF010001000040
:1051DA00000000000201000000000001320000008F
:1051EA00000001770176FF4EFF0200000000000078
:1051FA000132000000000001A200FBFFE0FF012DC8
:10520A0000F7FFFFFF012600F9FFFDFF011D00FB6C
:10521A00FFFDFF012000FBFFFCFF012700FBFFFA57
:10522A00FF012B00FDFFF8FF012E00FEFFF7FF0133
:10523A003200FFFFF6FF0132000100F6FF013300E2
:10524A000200F6FF012B000300F8FF01270005000A
:10525A00FAFF012A000600FAFF012B000700FBFFF4
:10526A00012B000800FDFF012F000900FDFF01606E
:10527A00001300FEFF019B001F000000012B00F934
:10528A00FF0500012A00FAFF0600012700FBFF06BE
:10529A0000012400FCFF0600012800FCFF070001B2
:1052AA002400FEFF0700012800FFFF080001280074
:1052BA00FFFF0800012D0001000900012D00010077
:1052CA000900012F0003000900012800040007005B
:1052DA00012D0004000800012E0006000700012E1F
:1052EA000007000600013200080006000133000929
:1052FA00000500013100090004000136000A00041B
:10530A00000134000A000300016B001500040001CB
:10531A007300170001000150001000FFFF01500048
:10532A001000FFFF0148000E00FDFF014A000E00B9
:10533A00FBFF014A000E00FBFF0141000B00F9FFD1
:10534A000140000A00F8FF0139000800F8FF013D9A
:10535A00000700F6FF013C000500F5FF01380002D6
:10536A0000F5FF0141000100F3FF0128000000F8E9
:10537A00FF012900FEFFF8FF012400FEFFF9FF01EB
:10538A002800FCFFF9FF012800FCFFF9FF012E00AD
:10539A00FAFFF9FF012E00F9FFFAFF012B00F9FFCE
:1053AA00FBFF0187001B0000000196000000E2FFDE
:1053BA0001DE033AFF0000017D00E7FF00000169FA
:1053CA0000EBFF0200015600EFFF0300014400F367
:1053DA00FF0400013800F6FF0500013D00F6FF0753
:1053EA0000013500F8FF0700013D00F9FF0A00013E
:1053FA003A00FAFF0A00013F00FCFF0C00013D00E1
:10540A00FEFF0C00014600FFFF0E000150000100E4
:10541A001000014E0004000F0001480006000D00B4
:10542A0001440008000B00012000040005000124CB
:10543A0000060004000124000600040001260007FB
:10544A0000030001240007000200012900080002ED
:10545A0000015500110001000100000000000002D7
:10546A000100000000000132000000000001EA0013
:10547A008A00E5FF0200000000000001320000007F
:10548A000000016900EBFFFFFF015B00EEFFFDFF7B
:10549A00014F00F1FFFBFF012200FAFFFDFF01228D
:1054AA0000FAFFFDFF013C00F7FFF8FF013900F9A0
:1054BA00FFF7FF013400FDFFF6FF013800FEFFF59C
:1054CA00FF0133000200F6FF0134000300F6FF017A
:1054DA0039000700F7FF013C000900F8FF011D0031
:1054EA000500FDFF0128000700FCFF0149000E002E
:1054FA00FCFF015B001200FDFF0164001400FFFFC6
:10550A000164001400010001560011000300014F5C
:10551A00000F0005000145000C000700013C0009CE
:10552A0000080001390007000900013100040009E0
:10553A000001370001000B00013200FFFF0A0001E1
:10554A003600FCFF0A00013900F9FF0900013C009E
:10555A00F7FF0800014300F4FF0600014A00F2FFCA
:10556A000500015600EFFF0300015F00EDFF010097
:10557A0001000000000000020100000000000132EA
:10558A000000000000018D0189FF32FF02000000C7
:10559A000000000132000000000001960000001E19
:1055AA0000012C063C01000001A5000000DFFF01FC
:1055BA00300290FF0000012B000700FBFF012A00C8
:1055CA000600FAFF0127000500FAFF01270005007F
:1055DA00FAFF0126000300F9FF0124000200F9FF87
:1055EA000124000200F9FF0128000000F8FF012D44
:1055FA00000000F7FF012900FEFFF8FF012900FE65
:10560A00FFF8FF012D00FCFFF8FF012F00FBFFF858
:10561A00FF012B00FBFFF9FF012E00F9FFFAFF0142
:10562A002B00F9FFFBFF012F00F8FFFBFF01310000
:10563A00F7FFFCFF013600F6FFFCFF013400F6FF1E
:10564A00FDFF013900F5FFFDFF013C00F4FFFFFFFC
:10565A00017800E8FFFEFF014600F2FF0000014763
:10566A0000F2FF0200013D00F4FF0200013D00F4D8
:10567A00FF0200013B00F5FF0400013600F6FF04BB
:10568A0000013300F7FF0500013300F7FF050001B1
:10569A003100F9FF0700012E00F9FF0600012B0077
:1056AA00FBFF0700012B00FBFF0700012D00FCFF99
:1056BA000800012400FEFF0700012900FEFF080080
:1056CA00012D00000009000128000000080001293E
:1056DA00000200080001260003000700012600035B
:1056EA0000070001270005000600012A000600063F
:1056FA0000012E0007000600012F00080005000126
:10570A009100E3FF000002010000000000013200E6
:10571A000000000001C10074000000020000000047
:10572A00000001320000000000015F00EDFFFFFFF2
:10573A00015000F0FFFFFF014800F2FFFDFF0136B4
:10574A0000F6FFFCFF012800F9FFFCFF012700FA21
:10575A00FFFBFF012000FBFFFCFF012300FBFFFB17
:10576A00FF012200FDFFFAFF011B00FEFFFBFF0104
:10577A002000FEFFFAFF0123000000F9FF013200BA
:10578A000100F6FF0131000400F7FF0139000700AC
:10579A00F7FF0140000A00F8FF0145000C00F9FF7D
:1057AA000154001000FBFF0156001100FDFF0169C2
:1057BA00001500FFFF01690015000100015B0012DE
:1057CA00000300014F000F0005000122000600033C
:1057DA000001220006000300013C00090008000144
:1057EA0035000700080001360004000A00013200F3
:1057FA0001000A00013200FFFF0A00013600FCFF27
:10580A000A00013900F9FF0900014000F6FF08000B
:10581A00014300F4FF0600014F00F1FF05000156A5
:10582A0000EFFF0300016400ECFF0100010000002B
:10583A000000000201000000000001320000000028
:10584A0000011001FFFF5DFF0200000000000001DF
:10585A00320000000000014B000F00FFFF0146006C
:10586A000E00FFFF0148000E00FDFF013E000C0084
:10587A00FDFF013B000B00FCFF013C000B00FBFF9E
:10588A000136000900FAFF0135000800F9FF012A74
:10589A00000600FAFF012B000500F9FF01280004A9
:1058AA0000F9FF0128000400F9FF012B000300F8AA
:1058BA00FF0129000200F8FF0128000100F8FF019A
:1058CA002D000000F7FF0132000000F6FF012E0054
:1058DA00FEFFF7FF012E00FEFFF7FF012B00FDFF81
:1058EA00F8FF012F00FBFFF8FF012B00FBFFF9FF78
:1058FA00012E00FAFFF9FF013200F8FFFAFF013228
:10590A0000F8FFFAFF012F00F8FFFBFF013800F64D
:10591A00FFFBFF013400F6FFFDFF013900F5FFFD33
:10592A00FF013D00F4FFFEFF014100F3FFFFFF010D
:10593A004100F3FF0000016900EBFF000001600075
:10594A00EDFF0200015200F0FF0400014A00F2FFDD
:10595A000500014300F4FF0600013D00F6FF0700C1
:10596A00014000F7FF0900014000F8FF0A00013F6B
:10597A0000FAFF0B00013C00FBFF0B00013D00FE9B
:10598A00FF0C00013C00FFFF0C0001320000000A7E
:10599A0000012E0002000900012E00020009000188
:1059AA002D0004000800012D0004000800012F004A
:1059BA0005000800012E000700060001310007005B
:1059CA000700013200080006000133000900050043
:1059DA000136000A0004000134000A000300013EF7
:1059EA00000C000300013D000C0002000146000EFD
:1059FA000001000146000E00010001000000000045
:105A0A000002010000000000013200000000000155
:105A1A0039000000DEFF0200000000000001320031
:105A2A0000000000016900EBFFFFFF015B00EEFFD1
:105A3A00FDFF014F00F1FFFBFF012200FAFFFDFF0E
:105A4A00012400FAFFFCFF014000F6FFF8FF013DC8
:105A5A0000F9FFF6FF013600FCFFF6FF013C00FFEC
:105A6A00FFF4FF013C000100F4FF0136000400F6D8
:105A7A00FF013D000700F6FF0140000A00F8FF01A0
:105A8A0024000600FCFF0122000600FDFF0154006D
:105A9A001000FBFF015B001200FDFF016900150009
:105AAA00FFFF016400140001000156001100030009
:105ABA00014F000F00050001260007000300012026
:105ACA0000050004000143000A000900013900072B
:105ADA00000900013B0004000B0001370001000B24
:105AEA0000013C00FFFF0C00013600FCFF0A000128
:105AFA003D00F9FF0A00014000F6FF0800012000FE
:105B0A00FBFF0400012600F9FF0300014F00F1FF2B
:105B1A000500015B00EEFF0300016400ECFF0100D9
:105B2A000100000000000002010000000000013234
:105B3A00000000000001BC01B0FF02FF02000000EB
:105B4A000000000132000000000001AC00DEFFFB93
:105B5A00FF014300FDFF0D00013C00FFFF0C0001A7
:105B6A0028000100080001230001000700012400A9
:105B7A0002000700011D00030005000119000300CF
:105B8A0004000120000500040001190004000300BC
:105B9A00011D000500030001230007000100013375
:105BAA00000A0002000191001D0001000194028414
:105BBA00000000017300000017000196001E00009B
:105BCA00000173000000E9FF011D01390000000116
:105BDA00C9001700DFFF019001B0FF000001A0001B
:105BEA000000E0FF019600E2FF000001A0000000B3
:105BFA002000019E027AFF0000014600F2FF000029
:105C0A00012300F9FFFFFF011D00FBFFFDFF011546
:105C1A0000FDFFFDFF011B00FEFFFBFF011E00FF51
:105C2A00FFFAFF0147000200F2FF01000000000036
:105C3A000002010000000000013200000000000123
:105C4A0058075AFF5C0402000000000000013200FD
:105C5A000000000001C701A8FFE9FF0141000000A0
:105C6A00F3FF015C014400F1FF014C00F1FFFEFF6C
:105C7A00011001CBFFF4FF0141000000F3FF01C74F
:105C8A00015800E9FF013C0000000C00010701CDAA
:105C9A00FF0D00015700EFFF040001570011000437
:105CAA000001050133000B00013C0000000C00015B
:105CBA000601CDFF0C00016100EDFF040001610047
:105CCA001300040001060133000C0001410000002A
:105CDA000D000100000000000002010000000000A9
:105CEA000132000000000001FF00A8FF83FF02004C
:105CFA0000000000000132000000000001C6015847
:105D0A000016000141000000F3FF010501CDFFF577
:105D1A00FF016200EDFFFBFF0161001300FCFF01C0
:105D2A0005013300F5FF0141000000F3FF01050101
:105D3A00CDFFF5FF015700EFFFFCFF0157001100EF
:105D4A00FCFF0107013300F3FF013C000000F4FFF0
:105D5A0001C701A8FF170001410000000D00011052
:105D6A000135000C00014C000F000300015C01BC6E
:105D7A00FF0F0001410000000D00020100000000B9
:105D8A00000132000000000001AC00000099FF028F
:105D9A000000000000000132000000000001C601FE
:105DAA0058001600013C000000F4FF010601CDFF77
:105DBA00F4FF016200EDFFFBFF0160001300FDFF2D
:105DCA000106013300F4FF0141000000F3FF010561
:105DDA0001CDFFF5FF015700EFFFFCFF015700114E
:105DEA0000FCFF0107013300F3FF013C000000F44F
:105DFA00FF01C701A8FF170001410000000D0001C3
:105E0A00100135000C00014C000F000300015C0179
:105E1A00BCFF0F0001410000000D0002010000005C
:105E2A00000001320000000000019B000000A3FFF7
:105E3A0002000000000000013200000000000155CD
:105E4A0000110000000146000000F2FF015500EFBA
:105E5A00FF000001460000000E00020100000000E1
:105E6A0000013200000000000197001C00AAFF0296
:105E7A0000000000000001320000000000014100A3
:105E8A00FFFFF3FF012400F9FF0200012000FAFFDF
:105E9A000200011900FCFF0300012000FBFF0400BF
:105EAA00011D00FDFF0500011B00FEFF0500011B8F
:105EBA0000FEFF0500011E00000006000128000187
:105ECA000008000124000200070001240004000663
:105EDA00000123000500050001240006000400015A
:105EEA002B0008000300012E000900020001320005
:105EFA000A0000000137000B000000012E00090013
:105F0A00FEFF012B000800FDFF0128000700FCFF2F
:105F1A000123000500FBFF0124000400FAFF01260B
:105F2A00000300F9FF0123000000F9FF012300002C
:105F3A0000F9FF012200FDFFFAFF012200FDFFFA2E
:105F4A00FF012700FAFFFBFF012400FAFFFCFF0113
:105F5A002B00F8FFFDFF012E00F7FFFEFF013700BF
:105F6A00F5FFFFFF011500FCFF010001130100000E
:105F7A003700012300F9FFFFFF012000FAFFFEFFAF
:105F8A00011B00FBFFFEFF011600FCFFFEFF0119CB
:105F9A0000FDFFFCFF011500FDFFFDFF011500FFDD
:105FAA00FFFCFF011900FFFFFBFF011E000100FAC1
:105FBA00FF0120000400FBFF0123000500FBFF0195
:105FCA002B000800FDFF0100000000000002010094
:105FDA00000000000132000000000001500019001A
:105FEA002900020000000000000132000000000049
:105FFA0001CD000000D7FF012D0009000100012694
:10600A000007000300011C0004000400011500033E
:10601A000003000116000200040001190000000537
:10602A000001140000000400011600FEFF04000134
:10603A001200FEFF0300011500FDFF030001190015
:10604A00FCFF0300011600FCFF0200011900FBFF20
:10605A000100011900FBFF0100010000000000001F
:10606A000201000000000001320000000000019758
:10607A0000C4FFBCFF020000000000000132000063
:10608A00000000013E00FDFFF4FF011900FBFFFFC5
:10609A00FF011900FCFFFDFF011D00FDFFFBFF01D1
:1060AA002900FEFFF8FF0124000200F9FF01220087
:1060BA000300FAFF0120000500FCFF012000060092
:1060CA00FEFF0123000700FFFF0141000D00000051
:1060DA00012400FAFF0400011D00FDFF0500011B59
:1060EA0000FEFF0500011E00FFFF0600012300015C
:1060FA000007000124000200070001200004000537
:10610A000001270006000500012600070003000120
:10611A002B000800030001280008000100012D00DF
:10612A0009000100013C000C00FFFF0139000B00CF
:10613A00FDFF0138000A00FBFF012E000700FAFFED
:10614A000116000200FCFF0116000200FCFF011507
:10615A00000100FCFF0119000000FBFF011E000006
:10616A0000FAFF012200FDFFFAFF012000FCFFFBFD
:10617A00FF012300FBFFFBFF0132000A00000001C0
:10618A0037000000F5FF017C01B4FF0000015A004E
:10619A00EEFF0100011E00FAFF0100011900FBFFDA
:1061AA000100012F00F8FF0500012E00FAFF070089
:1061BA00012D00FCFF0800013200FFFF0A00012345
:1061CA00000100070001190001000500011B00027F
:1061DA00000500011D000300050001190004000369
:1061EA0000011D0005000300011E00060001000158
:1061FA002300070000000100000000000002010067
:10620A000000000001320000000000015A003500C1
:10621A00F6FF02000000000000013200000000004A
:10622A00012800F8FF0000012300F9FFFFFF012009
:10623A0000FAFFFEFF011D00FBFFFDFF011500FD37
:10624A00FFFDFF011500FDFFFDFF011500FFFFFC2B
:10625A00FF011500FFFFFCFF0115000100FCFF0113
:10626A0015000100FCFF0115000300FDFF011900E4
:10627A000300FCFF011B000500FEFF0120000600D1
:10628A00FEFF011E000600FFFF01280008000000B3
:10629A0001280008000000011E000600010001207C
:1062AA000006000200011D0005000300011500039D
:1062BA00000300011500030003000115000100049A
:1062CA000001150001000400011500FFFF04000190
:1062DA001500FFFF0400011500FDFF030001150072
:1062EA00FDFF0300011D00FBFF0300011B00FBFF74
:1062FA000200012300F9FF0100012300F9FF000059
:10630A00010000000000000201000000000001324C
:10631A000000000000019100CBFFBBFF020000005B
:10632A0000000001320000000000013E00FDFFF401
:10633A00FF011900FBFFFFFF011900FCFFFDFF0130
:10634A002200FDFFFAFF012400FEFFF9FF012900E8
:10635A000200F8FF011D000300FBFF0120000500F9
:10636A00FCFF0122000600FDFF01230007000000D8
:10637A000141000D00FFFF012700FAFF0500011D82
:10638A0000FDFF0500011B00FEFF0500011E00FFC6
:10639A00FF06000123000100070001200002000699
:1063AA000001240004000600012400060004000184
:1063BA00280007000400012B000800030001280040
:1063CA0008000100012D0009000100013C000C0039
:1063DA00FFFF0139000B00FDFF0138000A00FBFF37
:1063EA00012E000700FAFF0116000200FCFF011649
:1063FA00000200FCFF0115000100FCFF011900006A
:10640A0000FBFF011E000000FAFF012200FDFFFA57
:10641A00FF012000FCFFFBFF012300FBFFFBFF0144
:10642A0032000A0000000137000000F5FF017C017C
:10643A00B4FF0000015A00EEFF0100011E00FAFF3E
:10644A000100011900FBFF0100012F00F8FF050000
:10645A00012A00FAFF0600013100FCFF090001329F
:10646A0000FFFF0A00011E0001000600011E0001D4
:10647A00000600011B0002000500011900030004C8
:10648A0000011C0004000400011B000500020001B9
:10649A00200006000200012300070000000100009E
:1064AA0000000000020100000000000132000000AC
:1064BA000000015A003500F6FF020000000000004B
:1064CA0001320000000000012800F8FF000001244A
:1064DA0000F9FFFEFF011E00FAFFFFFF011D00FB8E
:1064EA00FFFDFF011500FDFFFDFF011500FDFFFD8A
:1064FA00FF011500FFFFFCFF011500FFFFFCFF0174
:10650A0015000100FCFF0115000100FCFF01190044
:10651A000300FCFF0115000300FDFF011B0005003D
:10652A00FEFF0120000600FEFF011E000600FFFF1D
:10653A000128000800FFFF01280008000100011ED1
:10654A00000600010001200006000200011B0005F0
:10655A0000020001190003000400011500030003F2
:10656A0000011500010004000115000100040001EA
:10657A001500FFFF0400011500FFFF0400011500CC
:10658A00FDFF0300011500FDFF0300011D00FBFFD5
:10659A000300011900FBFF0100012400F9FF0200BA
:1065AA00012300F9FF0000010000000000000201C1
:1065BA00000000000001320000000000016F00F737
:1065CA00FFBEFF02000000000000013200000000D0
:1065DA0000014B000F00000001C3000000D9FF01B9
:1065EA004B00F1FF000001C3000000270002010078
:1065FA000000000001320000000000017B00DBFF08
:10660A00C0FF02000000000000013200000000008C
:10661A0001370000000B000162027A000000013C11
:10662A00000000F4FF01DC00D4FF00000124000692
:10663A0000FCFF011D000300FBFF011D000300FB1E
:10664A00FF011E000000FAFF0123000000F9FF010C
:10665A002200FDFFFAFF012400FCFFFAFF012000DF
:10666A00FBFFFCFF012800F9FFFCFF012900F8FFEE
:10667A00FEFF012900F8FFFEFF012D00F7FFFFFFD3
:10668A00013700F5FF0100013300F6FF0200012B7C
:10669A0000F8FF0300012800F9FF0400012300FBB2
:1066AA00FF0500012000FCFF0500012000FEFF0697
:1066BA0000011E00FFFF0600011E00010006000186
:1066CA002000020006000120000400050001240049
:1066DA0006000400013700F5FF0000020100000077
:1066EA00000001320000000000014B002D000000F4
:1066FA000200000000000001320000000000014614
:10670A0000F2FFFFFF012F00F7FFFDFF011D00FB55
:10671A00FFFDFF011C00FCFFFCFF011600FEFFFC51
:10672A00FF011900FFFFFBFF0115000100FCFF013B
:10673A0010000100FDFF0119000300FCFF01190010
:10674A000400FDFF011B000500FEFF011B00050000
:10675A00FEFF0123000700FFFF0128000800FFFFDA
:10676A000128000800010001230007000100011EA2
:10677A000006000100011D000500030001150003C9
:10678A0000030001150003000300011600020004C3
:10679A0000011400000004000114000000040001BC
:1067AA001200FEFF0300011900FDFF04000115009D
:1067BA00FDFF0300011D00FBFF0300011E00FAFF9D
:1067CA000100012400F9FF0200012300F9FF000083
:1067DA000100000000000002010000000000013278
:1067EA000000000000016900FFFFC1FF0200000075
:1067FA0000000001320000000000013C000C00FF14
:10680A00FF0133000A00FEFF012D000800FCFF0112
:10681A002B000700FBFF0120000400FBFF011D0005
:10682A000300FBFF0120000200FAFF012300000021
:10683A00F9FF0123000000F9FF012600FDFFF9FF1F
:10684A00011D00FDFFFBFF012A00FAFFFAFF0124E8
:10685A0000FAFFFCFF012B00F8FFFDFF012E00F7F5
:10686A00FFFEFF013200F6FF0000014B00F1FF01BD
:10687A0000011E00FAFF0100011B00FBFF020001DC
:10688A003300F7FF0500013100F9FF07000131006D
:10689A00FCFF0900012D00FFFF090001280001008B
:1068AA00080001200002000600012400040006007E
:1068BA000123000500050001240006000400012B45
:1068CA0000080003000133000A0002000132000A36
:1068DA0000010001000000000000020100000000A9
:1068EA0000013200000000000116000000F3FF0260
:1068FA000000000000000132000000000001280032
:10690A00F8FF0000012400F9FFFEFF011E00FAFF54
:10691A00FFFF011900FCFFFDFF011900FCFFFDFF4D
:10692A00011900FDFFFCFF011500FFFFFCFF011923
:10693A0000FFFFFBFF0115000100FCFF011500012C
:10694A0000FCFF0119000300FCFF0119000400FD0F
:10695A00FF011D000500FDFF011B000500FEFF01F0
:10696A0028000800FFFF012800080000000123009A
:10697A0007000000012300070001000120000600B3
:10698A000200011D000500030001150003000300B9
:10699A00011900030004000115000100040001159B
:1069AA000001000400011900FFFF0500011500FFA6
:1069BA00FF0400011900FDFF0400011500FDFF039B
:1069CA0000011D00FBFF0300011E00FAFF01000188
:1069DA002400F9FF0200012800F8FF00000100006E
:1069EA000000000002010000000000013200000067
:1069FA00000001AB00E1FF9EFF0200000000000062
:106A0A0001320000000000014200F3FFFEFF012DE9
:106A1A0000FFFF0900011E0000000600011B000222
:106A2A00000500011500030003000116000400021E
:106A3A0000012300070001000137000B00010001DB
:106A4A00FF0033000000012D00000009000137009B
:106A5A000B000000012D000000F7FF016E00160078
:106A6A000000014F000900F3FF019B00E1FF000055
:106A7A00013C000000F4FF013700F5FF0000013C73
:106A8A000000000C00010401CCFF0000012800F8FE
:106A9A00FF0000011500FDFFFDFF011500FFFFFCCF
:106AAA00FF0119000000FBFF0100000000000002C6
:106ABA000100000000000132000000000001220075
:106ACA00F3FFF0FF020000000000000132000000A6
:106ADA000000015500110000000146000000F2FF0D
:106AEA00015500EFFF000001460000000E00020100
:106AFA0000000000000132000000000001960020A2
:106B0A0000ACFF020000000000000132000000009B
:106B1A0000013D00FEFFF4FF012300F9FF0100011F
:106B2A002000FAFF0200012200FAFF0300011C0004
:106B3A00FCFF0400011C00FCFF0400011D00FDFF16
:106B4A000500012000FEFF060001190000000500F3
:106B5A0001280001000800012000020006000124AB
:106B6A0000040006000123000500050001240006B8
:106B7A00000400012B0008000300012D0009000198
:106B8A00000137000B0001000141000D00FFFF0169
:106B9A003E000C00FDFF011B000500FEFF0119006D
:106BAA000400FDFF0119000400FDFF0119000300A4
:106BBA00FCFF012D000400F8FF0132000100F6FF7E
:106BCA000119000000FBFF011E00FFFFFAFF011977
:106BDA0000FDFFFCFF011900FDFFFCFF011C00FC8A
:106BEA00FFFCFF011D00FBFFFDFF011B00FBFFFE79
:106BFA00FF012300F9FFFFFF013D00FEFF0C00012A
:106C0A0029000800020001240006000400011D00FA
:106C1A0003000500011E0001000600011400000027
:106C2A000400011600FEFF0400011900FDFF040024
:106C3A00011500FDFF0300011D00FBFF03000120F9
:106C4A0000FAFF0200012300F9FF0100012800F801
:106C5A00FF0000012800F8FF0000012300F9FFFFF0
:106C6A00FF012000FAFFFEFF011D00FBFFFDFF01EF
:106C7A001500FDFFFDFF011500FDFFFDFF011500D9
:106C8A00FFFFFCFF011500FFFFFCFF0124000200CB
:106C9A00F9FF0124000400FAFF0112000300FEFFBD
:106CAA000116000400FEFF012E000900FEFF01008C
:106CBA000000000000020100000000000132000094
:106CCA000000000124000C00EEFF0200000000009A
:106CDA000001320000000000013C000C00FFFF012F
:106CEA0033000A00FEFF012D000800FCFF012B0003
:106CFA000700FBFF0120000400FBFF011D00030049
:106D0A00FBFF0120000200FAFF0123000000F9FF47
:106D1A000123000000F9FF012600FDFFF9FF01220F
:106D2A0000FDFFFAFF012700FAFFFBFF012400FA2A
:106D3A00FFFCFF012B00F8FFFDFF012E00F7FFFE0D
:106D4A00FF013200F6FF0000014B00F1FF010001D4
:106D5A001E00FAFF0100011B00FBFF0200013300C5
:106D6A00F7FF0500013100F9FF0700013100FCFFC0
:106D7A000900012D00FFFF0900012300010007009F
:106D8A000124000200070001240004000600012378
:106D9A00000500050001240006000400012B00087C
:106DAA000003000133000A0002000132000A000158
:106DBA0000010000000000000201000000000001C4
:106DCA003200000000000116000000F3FF0200007C
:106DDA000000000001320000000000012800F8FF56
:106DEA00FFFF012300F9FFFFFF012000FAFFFEFF6A
:106DFA00011600FCFFFEFF011C00FCFFFCFF011551
:106E0A0000FDFFFDFF011500FFFFFCFF011900FF58
:106E1A00FFFBFF0115000100FCFF0115000100FC4A
:106E2A00FF0119000300FCFF0119000400FDFF0126
:106E3A001D000500FDFF011B000500FEFF012800E3
:106E4A000800FFFF0128000800FFFF0123000700D8
:106E5A0001000123000700010001200006000200D2
:106E6A00011D0005000300011500030003000119BC
:106E7A0000030004000115000100040001150001CF
:106E8A00000400011900FFFF0500011500FFFF04BF
:106E9A0000011500FDFF0300011900FDFF040001B8
:106EAA001B00FBFF0200012000FAFF020001230081
:106EBA00F9FF0100012800F8FF01000100000000AD
:106ECA000000020100000000000132000000000082
:106EDA00018B00D4FFB9FF0200000000000001325C
:106EEA00000000000001B80158000000013700004E
:106EFA0000F5FF013C00F4FF00000124000600FC3D
:106F0A00FF0124000400FAFF0122000300FAFF0136
:106F1A0023000100F9FF012300FFFFF9FF0122000E
:106F2A00FDFFFAFF012300FBFFFBFF012000FAFF30
:106F3A00FEFF012B000700FBFF0127000500FAFFF7
:106F4A000120000200FAFF011E000100FAFF0119E8
:106F5A00000000FBFF011900FFFFFBFF011900FD04
:106F6A00FFFCFF011500FDFFFDFF011900FCFFFDFD
:106F7A00FF011B00FBFFFEFF011E00FAFFFFFF01DE
:106F8A002300F9FF0000013101C3FF0000013C00AA
:106F9A0000000C000118013800000001230007005E
:106FAA000100011E0006000100011000030001009B
:106FBA000115000300030001160002000400011479
:106FCA000000000400010F0000000300011500FF8B
:106FDA00FF0400011200FEFF0300011200FDFF0280
:106FEA0000011500FDFF0300011900FBFF0100016C
:106FFA003D00F4FF020001FF00CDFF0000013C004C
:10700A0000000C00011D0139000000012D000900DB
:10701A000100012000060002000112000300020024
:10702A00010B0001000200011E0001000600011907
:10703A000000000500011D00FDFF0500011C00FC09
:10704A00FF0400012000FAFF0200012900F8FF02F4
:10705A0000013200F6FF000001E600D2FF00000145
:10706A00410000000D000201000000000001320092
:10707A000000000001ED05CB0089FC0200000000C1
:10708A0000000132000000000001A400F5FFE1FF4A
:10709A0001A100F7FFE1FF012201F1FFC8FF01058D
:1070AA0001F5FFCDFF01DA00F9FFD5FF01B100FBC1
:1070BA00FFDDFF018700FEFFE5FF016E00FEFFEA2C
:1070CA00FF02010000000000013200000000000180
:1070DA00F8013E0028010200000000000001320011
:1070EA000000000001800280FF0000020100000091
:1070FA00000001320000000000010C02EC0030FF29
:10710A00020000000000000132000000000001AB94
:10711A0000F7FF2100019500F6FF1C00019600F51B
:10712A00FF1C00019D00F4FF1D0001C000F0FF23B9
:10713A000001CE00ECFF2400016300F6FF110001FC
:10714A006100F5FF1000016400F4FF100001600007
:10715A00F4FF0F00012A00FAFF0600012700FAFFD8
:10716A000500012400FAFF0400012000FAFF0200D2
:10717A00012000FAFF0200011E00FAFF0000013C94
:10718A0000F4FF0000013D00F4FFFEFF014200F39E
:10719A00FFFEFF014200F3FFFEFF014600F2FF007F
:1071AA0000013700F5FF0000012D00F7FFFFFF0186
:1071BA002B00F8FFFDFF012000FBFFFCFF010E0082
:1071CA00FEFFFEFF010F000000FDFF011000FFFFA0
:1071DA00FDFF0115000100FCFF012D000400F8FF6E
:1071EA000140000800F6FF0120000400FBFF012413
:1071FA00000200F9FF012E000200F7FF012D000036
:10720A0000F7FF012D00FFFFF7FF012E00FEFFF739
:10721A00FF012800FCFFF9FF012700FBFFFAFF022C
:10722A0001000000000001320000000000019E027F
:10723A00FF00C9FE02000000000000013200000049
:10724A000000011E000600000001150004000100F4
:10725A000112000300020001160002000400011BD3
:10726A00000200050001190001000500014600FFA7
:10727A00FF0E00014C00FEFF0F00014C00FDFF0F46
:10728A0000018E00FBFF1C00018F00FAFF1C0002A8
:10729A000100000000000132000000000001290284
:1072AA00E9FEB40002000000000000013200000004
:1072BA000000015D00EEFFFBFF014700F2FFFEFF49
:1072CA00013700F5FF0000012F00F7FF0300012737
:1072DA0000FAFF0500012700FBFF0600012600FD5A
:1072EA00FF0700012E00FEFF0900015600FDFF11F5
:1072FA0000012D00FFFF0900012900FEFF0800011F
:10730A002600FDFF0700012000FCFF050001240004
:10731A00FAFF0400012800F8FF0100018A01EFFFCB
:10732A00B3FF011E000000FAFF0119000100FBFF74
:10733A000136000400F6FF013A000600F6FF0136A6
:10734A00000600F7FF0160000C00F1FF01280004AD
:10735A0000F9FF0120000200FAFF010B00FFFFFE07
:10736A00FF011000FFFFFDFF012E00F9FFFAFF01E8
:10737A008A00EBFFEEFF014B00F4FFF7FF014A0022
:10738A00F6FFF5FF014300F7FFF6FF011D00FDFFC1
:10739A00FBFF011B00FEFFFBFF014B01F3FFBFFFD9
:1073AA00010401F6FFCDFF011900050000000119D3
:1073BA000005000100011600040002000116000485
:1073CA0000020001350007000800013A0006000A21
:1073DA00000194000C001B00015E0008001100016E
:1073EA00600009001100011D0003000500011C00D6
:1073FA00040004000144000B000800014A000D00CB
:10740A000700014A000E0005000147000E000200B5
:10741A00012300070000000123000700FFFF0120ED
:10742A00000600FEFF011D000500FDFF012000050A
:10743A0000FCFF0124000400FAFF0131000400F7F8
:10744A00FF013E000300F4FF0141000100F3FF01C8
:10745A0046000000F2FF02010000000000013200B5
:10746A0000000000010A00060000000200000000FF
:10747A000000013200000000000166001400040050
:10748A0001510010000200013C000C000000013311
:10749A00000A00FEFF012D000800FCFF013200086F
:1074AA0000FAFF0135000800F9FF0143000900F660
:1074BA00FF014E000A00F4FF014E000A00F4FF012A
:1074CA009E001200E6FF0138012100CBFF015500A2
:1074DA000800F1FF015C000900F0FF01BE000F0087
:1074EA00DDFF01BF000D00DCFF01B1000A00DEFF75
:1074FA0001F7000C00D0FF01F5000A00D0FF015A85
:10750A00000100EEFF011E00FFFFFAFF011500FF58
:10751A00FFFCFF011200FEFFFDFF011200FDFFFE4E
:10752A00FF011000FDFFFFFF011000FDFF01000138
:10753A002E00F7FF0200012F00F7FF0300013900B8
:10754A00F5FF0300013200F6FF0100013200F6FFE9
:10755A000000012E00F7FF0200013100F7FF0400CE
:10756A00013600F7FF0600013900F7FF0700013C6A
:10757A0000F8FF0900014300F7FF0A00014400F880
:10758A00FF0B00018900F1FF1700019200F1FF19BA
:10759A0000018B00F2FF1800018000F3FF160002C1
:1075AA0001000000000001320000000000019B0100
:1075BA00C4FFEF00020000000000000132000000DA
:1075CA000000015F00EDFF0000015100F0FFFEFF27
:1075DA00013D00F4FFFEFF013100F7FFFCFF01153A
:1075EA0000FDFFFDFF011500FDFFFDFF011600FE76
:1075FA00FFFCFF011500FFFFFCFF013C00FFFFF449
:10760A00FF014C000200F1FF0156000300EFFF01E9
:10761A0061000400EDFF0162000500EDFF01650055
:10762A000700EDFF0165000900EEFF0132000600C8
:10763A00F8FF0132000600F8FF0135000700F8FFE5
:10764A000131000700F9FF0132000800FAFF013397
:10765A00000900FBFF0201000000000001320000E7
:10766A00000000011D00F1FF0900020000000000F7
:10767A00000132000000000001FF00F6FFCEFF010A
:10768A005601F2FFBDFF02010000000000013200B6
:10769A00000000000186023D01DF00020000000038
:1076AA00000001320000000000019300F7FFE4FF30
:1076BA00018200F9FFE7FF010701F3FFCDFF019FF8
:1076CA0000F9FFE1FF01C500FAFFD9FF01D400FA72
:1076DA00FFD6FF01DD00FCFFD4FF0201000000001D
:1076EA000001320000000000018F01F7FFEF0002E5
:1076FA0000000000000001320000000000017F00CD
:10770A000B00E9FF014600F2FFFFFF017D00F6FFD3
:10771A0017000141000D00010001000000000000F7
:10772A000201000000000001320000000000011701
:10773A0000F2FF0000020000000000000132000019
:10774A00000000016A00FDFFEBFF0172000900EB77
:10775A00FF015D00050012000201000000000001A7
:10776A00320000000000012700F4FF1400020000AC
:10777A000000000001320000000000014F01BDFFBF
:10778A00FFFF0201000000000001320000000000BB
:10779A00016E004000EFFF0200000000000001320D
:1077AA000000000000010901CBFF000002010000F7
:1077BA0000000001320000000000016F003F00EBF2
:1077CA00FF0200000000000001320000000000017A
:1077DA00FA00CEFF000002010000000000013200A2
:1077EA00000000000179003A002C000200000000AD
:1077FA0000000132000000000001F2021D009400A6
:10780A000201000000000001320000000000010433
:10781A0001D5FF6AFF0200000000000001320000EB
:10782A0000000001F7021D0095000201000000009F
:10783A000001320000000000011D01FCFF55FF029B
:10784A000000000000000132000000000001BF0239
:10785A001B008A0002010000000000013200000043
:10786A000000012B0002001A0002000000000000C4
:10787A0001320000000000012800FFFF0800012477
:10788A0000FEFF0700010700FFFF0100010700FFDC
:10789A00FF0100010E00FEFFFEFF012800FCFFF9B8
:1078AA00FF02010000000000013200000000000198
:1078BA001800F2FFFEFF0200000000000001320083
:1078CA000000000001240002000700011500030067
:1078DA000300010B00020001000141000D0000003D
:1078EA00020100000000000132000000000001EF68
:1078FA00007AFF330002000000000000013200009D
:10790A000000000126000700FDFF0126000700FD18
:10791A00FF0132000800FAFF012E000700FAFF01FA
:10792A0035000700F8FF0136000600F7FF013600B0
:10793A000600F7FF013A000600F6FF0138000500CD
:10794A00F6FF013B000400F5FF0139000300F5FFD3
:10795A000133000200F6FF0137000100F5FF012D97
:10796A00000000F7FF013200FFFFF6FF012D00FCC7
:10797A00FFF8FF012600FDFFF9FF012300FBFFFBD3
:10798A00FF011D00FBFFFDFF012200FAFFFDFF01C1
:10799A001E00FAFFFFFF011E00FAFFFFFF011E0093
:1079AA00FAFF0100012300F9FF0100013F00F4FF83
:1079BA000400014300F4FF0600013900F7FF070045
:1079CA00013500F8FF070002010000000000013243
:1079DA00000000000001F30085003C0002000000E6
:1079EA000000000132000000000001D600D7FFF4B9
:1079FA00FF02010000000000013200000000000147
:107A0A0040002500F5FF02000000000000013200DE
:107A1A000000000001C100DBFF0B000201000000B2
:107A2A00000001320000000000016B003F000C0062
:107A3A0002000000000000013200000000000140C6
:107A4A0001400000000136013E0000000176027E7E
:107A5A0000FDFF014C000F00FEFF012D000900FF91
:107A6A00FF0110000300FFFF010B000100FEFF01F0
:107A7A0010000100FDFF0119000000FBFF012800B2
:107A8A00FFFFF8FF010B00FFFFFEFF010B00FEFFE7
:107A9A00FFFF012D00F7FFFFFF015000F0FFFFFF7E
:107AAA00017B0281FF0100013B01C1FF010001408E
:107ABA0001C0FF0300010B00FEFF0100010E00FEE2
:107ACA00FF0200011500FFFF040001190000000574
:107ADA000001190001000500011500010004000160
:107AEA00120002000300011000030001000100005F
:107AFA000000000002010000000000013200000046
:107B0A0000000147001500DBFF0200000000000032
:107B1A000132000000000001BA00EFFFDFFF015947
:107B2A0000F8FFF0FF015E00F8FFEFFF020100001E
:107B3A0000000001320000000000016D00EBFFC2EE
:107B4A00FF020000000000000132000000000001F6
:107B5A006200FBFFEDFF016000FEFFEDFF01600028
:107B6A00FEFFEDFF015F00FFFFEDFF01C300010013
:107B7A00D9FF01B9000100DBFF020100000000008B
:107B8A0001320000000000015B014300C500020051
:107B9A0000000000000132000000000001C800D807
:107BAA00FFFFFF0201000000000001320000000098
:107BBA0000015002EBFE22FF02000000000000015B
:107BCA003200000000000128000800010001260020
:107BDA000700030001270006000500012300050035
:107BEA00050001550008000F00016200080012009C
:107BFA0001B6000D0022000201000000000001325F
:107C0A00000000000001F20156001E0102000000FF
:107C1A0000000001320000000000010C01E8FF3002
:107C2A000002010000000000013200000000000113
:107C3A0054002100DAFF02000000000000013200B7
:107C4A000000000001FF00EAFF2E00020100000010
:107C5A00000001320000000000019B00B4FFCAFFCF
:107C6A0002000000000000013200000000000111C3
:107C7A0001E6FF30000201000000000001320000AE
:107C8A0000000001EC008A001F0002000000000052
:107C9A000001320000000000011C01E9FF3400026B
:107CAA0001000000000001320000000000017C0019
:107CBA00E6FFBAFF020000000000000132000000E7
:107CCA00000001C201A6FF0100020100000000003D
:107CDA0001320000000000019C005C00F0FF02007D
:107CEA0000000000000132000000000001C701A5E9
:107CFA00FF02000201000000000001320000000043
:107D0A000001E60068005B000200000000000001BC
:107D1A0032000000000001BD01A7FF0100020100BE
:107D2A000000000001320000000000019400590028
:107D3A00FFFF020000000000000132000000000006
:107D4A00018C01F2FFB2FF020100000000000132C3
:107D5A000000000000017C0019004600020000003B
:107D6A0000000001320000000000018701F2FFB3A9
:107D7A00FF020100000000000132000000000001C3
:107D8A00CB00AAFF560002000000000000013200EA
:107D9A0000000000018E01F0FFB2FF0201000000A6
:107DAA0000000132000000000001DD007400C0FF85
:107DBA00020000000000000132000000000001BDC6
:107DCA0001A7FF01000201000000000001320000CB
:107DDA00000000019B004B00370002000000000079
:107DEA000001320000000000014100F5FF07000217
:107DFA00010000000000013200000000000117002D
:107E0A000000F2FF02000000000000013200000042
:107E1A000000014600FFFF0E000201000000000002
:107E2A00013200000000000119000100F1FF020008
:107E3A000000000000013200000000000144000BB5
:107E4A0000080002010000000000013200000000EA
:107E5A000001B60093FF01000200000000000001CB
:107E6A00320000000000013500070008000201008E
:107E7A000000000001320000000000011B000200A7
:107E8A00F0FF0200000000000001320000000000C4
:107E9A00013900F7FF07000201000000000001326B
:107EAA00000000000001F2007B004D00020000000B
:107EBA0000000001320000000000014400F5FF0844
:107ECA000002010000000000013200000000000171
:107EDA00A000A0FFF9FF020000000000000132002C
:107EEA0000000000018A01EFFFB3FF020100000059
:107EFA00000001320000000000015C001A00CFFF00
:107F0A00020000000000000132000000000001131E
:107F1A0001E7FF3100020100000000000132000009
:107F2A00000000016D002200C8FF020000000000EE
:107F3A000001320000000000013900F7FF070002CB
:107F4A000100000000000132000000000001A4004E
:107F5A006200F9FF02000000000000013200000088
:107F6A000000014E0007000E0002010000000000A0
:107F7A000132000000000001D40086FF2400020044
:107F8A000000000000013200000000000141000072
:107F9A00000D000201000000000001320000000094
:107FAA0000017700080047000200000000000001FD
:107FBA003200000000000131000700070002010042
:107FCA0000000000013200000000000143026200CC
:107FDA00B3FE0200000000000001320000000000B1
:107FEA00015101F2FFBEFF02010000000000013250
:107FFA000000000000016B0019003B0002000000B5
:10800A0000000001320000000000014B01F3FFBF35
:10801A00FF02010000000000013200000000000120
:10802A004500230016000200000000000001320093
:10803A0000000000014B01F3FFBFFF020100000036
:10804A0000000132000000000001FD009EFF7400E4
:10805A00020000000000000132000000000001558B
:10806A0001F3FFBDFF020100000000000132000021
:10807A000000000118000300F2FF020000000000E7
:10808A00000132000000000001FB001A00D5FF02C7
:10809A0001000000000001320000000000017B0026
:1080AA003000380002000000000000013200000029
:1080BA000000018101B3FF0100020100000000007D
:1080CA00013200000000000186004F00F2FF0200AA
:1080DA00000000000001320000000000017C01B431
:1080EA00FF00000201000000000001320000000051
:1080FA0000017F004C0000000200000000000001A7
:10810A0032000000000001F4001700D5FF02010050
:10811A000000000001320000000000015600F3FFD9
:10812A0032000200000000000001320000000000DE
:10813A0001ED001600D6FF02010000000000013226
:10814A00000000000001C400ECFF740002000000FF
:10815A0000000001320000000000018101B3FF00AD
:10816A0000020100000000000132000000000001CE
:10817A00FD00580084FF02000000000000013200E8
:10818A0000000000016D01B7FF00000201000000BD
:10819A0000000132000000000001E4004900740000
:1081AA00020000000000000132000000000001EDA2
:1081BA00001600D6FF020100000000000132000094
:1081CA00000000015B00D3FFE1FF02000000000095
:1081DA000001320000000000013D000A0007000211
:1081EA00010000000000013200000000000116003A
:1081FA00F4FF060002000000000000013200000047
:10820A0000000143000C00FAFF0201000000000018
:10821A0001320000000000011700F4FF070002000D
:10822A0000000000000132000000000001470002C7
:10823A0000F2FF020100000000000132000000000D
:10824A0000018500B1FF0D000200000000000001DE
:10825A00320000000000013E000300F4FF020100AA
:10826A000000000001320000000000017F0004004D
:10827A004C00020000000000000132000000000073
:10828A00015001F3FFBEFF020100000000000132AD
:10829A0000000000000102000000FFFF02000000D1
:1082AA00000000013200000000000143000900F64E
:1082BA00FF0201000000000001320000000000017E
:1082CA001600F7FF0A000200000000000001320059
:1082DA000000000001240006000400020100000062
:1082EA00000001320000000000010D00FAFFFBFF50
:1082FA00020000000000000132000000000001023C
:10830A00011B00D4FF02010000000000013200003E
:10831A000000000102000000FFFF02000000000050
:10832A0000013200000000000135000800F9FF02D8
:10833A000100000000000132000000000001CB0033
:10834A00EBFF78000200000000000001320000008C
:10835A0000000120000500040002010000000000E6
:10836A00013200000000000182004E0000000200FD
:10837A000000000000013200000000000141000B73
:10838A0000F9FF02010000000000013200000000B5
:10839A000001C30001008BFF020000000000000181
:1083AA003200000000000139000800080002010044
:1083BA00000000000132000000000001AF0E320090
:1083CA00CF08020100000000000132000000000096
:1083DA000201000000000000000000000000D8CFE9
:1083EA00E4FFE0CFE4FFE46EE9CFE4FFEACFE4FF85
:1083FA00F3CFE4FFF4CFE4FFE652D9CFE6FFDACFBA
:10840A00E6FFE1CFD9FFE2CFDAFFE652E652E652C3
:10841A00E652020EDB6A030EDB6AA4A6E8D2A49631
:10842A000E01002B0E01AB510E01005D01E255D188
:10843A00006B0E01A951EA6A310FE96E0E0EEA22AB
:10844A00EF500E01EA6AAC25E96EAD51EA22EF6AF5
:10845A0079907B6A7A6A0E01A92B0E01AA510E0144
:10846A00A95D01E3A96BA951E96EEA6AD890E936D8
:10847A00EA36010EE9260E0EEA22EE50ED1001E16F
:10848A002CD1A951E96EEA6AD890E936EA36490E42
:10849A00E9260E0EEA22EECF48F0EFCF49F0A951B5
:1084AA00E96EEA6AD890E936EA36010EE9260E0E36
:1084BA00EA22EECF4AF0EFCF4BF04A50481802E1D9
:1084CA004B50491801E1CBD0A951E96EEA6AD8901C
:1084DA00E936EA36790EE9260E0EEA22EE50ED105A
:1084EA0001E1A1D0A951E96EEA6AD890E936EA36E3
:1084FA00490EE9260E0EEA22EECF4AF0EFCF4BF0F4
:10850A00A951E96EEA6AD890E936EA36010EE926F7
:10851A000E0EEA22EE504A5C486EEE504B58496EF7
:10852A00020E48C0DBFF030E49C0DBFF020EDBCFA1
:10853A0048F0030EDBCF49F049343BE248500008CB
:10854A00000E495436E2020EDBCF48F0030EDBCFB1
:10855A0049F0A951E96EEA6AD890E936EA36790E05
:10856A00E9260E0EEA22EECF4AF0EFCF4BF0485042
:10857A004A5C49504B5857E2A951E96EEA6AD890C9
:10858A00E936EA36790EE9260E0EEA22EECF48F0EF
:10859A00EFCF49F0A951E96EEA6AD890E936EA368E
:1085AA00010EE9260E0EEA224850EE264950ED2227
:1085BA0056D0020EDBCF48F0030EDBCF49F0486CF1
:1085CA00491E000E4922A951E96EEA6AD890E93695
:1085DA00EA36790EE9260E0EEA22EECF4AF0EFCFFE
:1085EA004BF048504A5C49504B581DE2A951E96E7C
:1085FA00EA6AD890E936EA36790EE9260E0EEA22B8
:10860A00EECF48F0EFCF49F0A951E96EEA6AD89067
:10861A00E936EA36010EE9260E0EEA224850EE5EE7
:10862A004950ED5A1CD0A951E96EEA6AD890E93648
:10863A00EA36490EE9260E0EEA22EECF48F0EFCFCF
:10864A0049F0A951E96EEA6AD890E936EA36010E8C
:10865A00E9260E0EEA2248C0EEFF49C0EDFFA951F5
:10866A00EA6A310FE96E0E0EEA22EF500E01EA6A4B
:10867A00AC25E96EAD51EA22120EEF6EF29E0E01A2
:10868A00A951E96EEA6AD890E936EA36010EE92676
:10869A000E0EEA22EECF48F0EFCF49F049C048F07B
:1086AA00496A4850B66EA951E96EEA6AD890E93625
:1086BA00EA36010EE9260E0EEA22EECF48F0EFCF97
:1086CA0049F04850B56EF00EB4140009B46EF00EBD
:1086DA00B4140909B46E7980F28E0701000ED880AD
:1086EA00AA55000EAB552EE2B82B000EB923AA519B
:1086FA00B85DAB51B95926E3B86BB96B030EAE5DE1
:10870A001FE2AC51EA6A200FE96E010EEA2280CF1D
:10871A00EFFFAC51EA6A230FE96E010EEA2281CF1C
:10872A00EFFFAC51EA6A260FE96E010EEA2282CF08
:10873A00EFFFAC2B030EAC5D01E3AC6BAE2B02D0AA
:10874A00AA6BAB6B000ED880AF55000EB0551CE279
:10875A00000ED880BE55000EBF5516E2BA2B000E89
:10876A00BB23AF51BA5DB051BB590EE3BA6BBB6BB9
:10877A00030EB35D07E2B12B030EB15D01E3B16BEA
:10878A00B32B02D0AF6BB06BBE51BF110BE0050E1D
:10879A00BD5D07E3C18C9E9C9D8CC280C282BD6B6D
:1087AA0001D0BD2B0601005101E11DD1DE6ADD6A4F
:1087BA00DECF48F0DDCF49F0040E485C000E495880
:1087CA0001E311D1DECFE9FFDDCFEAFF010ED89038
:1087DA00E936EA36E806FBE1010EE926060EEA2248
:1087EA00EE50ED1001E1D3D0DECFE9FFDDCFEAFF95
:1087FA00010ED890E936EA36E806FBE1110EE926C1
:10880A00060EEA22EE50ED1026E1D9CFE9FFDACFC3
:10881A00EAFFEE50ED1001E18180D9CFE9FFDACF0E
:10882A00EAFF010EEE1803E1ED5001E18182D9CF92
:10883A00E9FFDACFEAFF020EEE1803E1ED5001E19B
:10884A008184D9CFE9FFDACFEAFF030EEE1803E1FC
:10885A00ED5001E18186DECFE9FFDDCFEAFF010EAF
:10886A00D890E936EA36E806FBE1110EE926060E4B
:10887A00EA22EECF48F0EFCF49F0DECFE9FFDDCFB5
:10888A00EAFF010ED890E936EA36E806FBE1010E66
:10889A00E926060EEA22EECF4AF0EFCF4BF04A5015
:1088AA00481829E14B50491826E1D9CFE9FFDACF18
:1088BA00EAFFEE50ED1001E18190D9CFE9FFDACF5E
:1088CA00EAFF010EEE1803E1ED5001E18192D9CFE2
:1088DA00E9FFDACFEAFF020EEE1803E1ED5001E1FB
:1088EA008194D9CFE9FFDACFEAFF030EEE1803E14C
:1088FA00ED5001E18196DECFE9FFDDCFEAFF010EFF
:10890A00D890E936EA36E806FBE1110EE926060EAA
:10891A00EA22EE2A000EEF22DECFE9FFDDCFEAFFE0
:10892A00010ED890E936EA36E806FBE1110EE9268F
:10893A00060EEA22EECF48F0EFCF49F0DECFE9FF8C
:10894A00DDCFEAFF010ED890E936EA36E806FBE108
:10895A00090EE926060EEA22EECF4AF0EFCF4BF0D7
:10896A004A5048183AE14B50491837E1DECFE9FF3F
:10897A00DDCFEAFF010ED890E936EA36E806FBE1D8
:10898A00110EE926060EEA22EE6AED6A26D0D9CF42
:10899A00E9FFDACFEAFFEE50ED1001E18190D9CF7D
:1089AA00E9FFDACFEAFF010EEE1803E1ED5001E12B
:1089BA008192D9CFE9FFDACFEAFF020EEE1803E17E
:1089CA00ED5001E18194D9CFE9FFDACFEAFF030E36
:1089DA00EE1803E1ED5001E18196DF2A010E01E272
:1089EA00E7D6DB2AE5D60501E05101E0E0079EACB7
:1089FA0042D09E9CC1AC07D0C19C010E0701C06F3A
:108A0A00C16BBC6B1DD0C4504A6E4B6E4A6AC350D0
:108A1A0000014A10486E4BC049F00701BC51E96E8B
:108A2A00EA6AD890E936EA36000EE926010EEA2209
:108A3A0048C0EEFF49C0EDFFD890C037C137BC2B04
:108A4A00100EBC5D0EE2C051BE15486EC151BF1575
:108A5A00496E4850491005E1BC2BD890C037C13740
:108A6A00EFD7100EBC5D02E39D9C05D0BC51040DEE
:108A7A00F328C26EC282F2A444D0D59EF294F29A2E
:108A8A00040E486E0701B751EA6A290FE96E010E12
:108A9A00EA22EF50485C35E1080EB75D0DE2070E99
:108AAA00B715486E010E485204E0E846FE0B480628
:108ABA00FCE1E81C89161CD0100EB75D0DE2070E0A
:108ACA00B715486E010E485204E0E846FE0B480608
:108ADA00FCE1E81C8A160CD0070EB715486E010E89
:108AEA00485204E0E846FE0B4806FCE1E81C8B16F7
:108AFA000701B751EA6A290FE96E010EEA22020E4E
:108B0A00EF6E040EE15C02E2E16AE552E16EE552C3
:108B1A00E5CFDAFFE7CFD9FFE552E5CFF4FFE5CF9E
:108B2A00F3FFE5CFEAFFE5CFE9FFE550E5CFE0FF48
:108B3A00E5CFD8FF1000D9CFE6FFDACFE6FFE1CFC5
:108B4A00D9FFE2CFDAFFE652E652E652E652896AE6
:108B5A0092680701BE6BBF6B8A6A93688B6A9468D6
:108B6A008C968C9495969594928E010EE36F0501DE
:108B7A00F369F4690701B26BB16BB36BAD6BAC6BA4
:108B8A00AE6BAA6BAB6BAF6BB06BB86BB96BBA6BF6
:108B9A00BB6BBC6B76827680769C769A7688769664
:108BAA00FA0E776EDE6ADD6ADECF00F0DDCF01F005
:108BBA00D890015004E6100E005C000E015812E233
:108BCA00DECFE9FFDDCFEAFFD890E936EA36000EBC
:108BDA00E926010EEA22EE6AED6ADF2A010EE4E3D3
:108BEA00DB2AE2D70701DD6BDE6BDB6BDC6BDE6A4F
:108BFA00DD6ADECF00F0DDCF01F0D890015004E647
:108C0A00400E005C000E01580EE2DECFE9FFDDCF18
:108C1A00EAFF000EE926020EEA22EF6ADF2A010EB7
:108C2A00E8E3DB2AE6D7DE6ADD6ADECF00F0DDCFD5
:108C3A0001F0D890015004E6400E005C000E015885
:108C4A000EE2DECFE9FFDDCFEAFF400EE926020E93
:108C5A00EA22EF6ADF2A010EE8E3DB2AE6D7DE6AB8
:108C6A00DD6ADECF00F0DDCF01F0D890015004E6D6
:108C7A00000E005C010E01580EE2DECFE9FFDDCFE7
:108C8A00EAFF000EE926030EEA22EF6ADF2A010E46
:108C9A00E8E3DB2AE6D70701DF6BE06BE16BE26B07
:108CAA00B56BB66BB76BDE6ADD6ADECF00F0DDCF7F
:108CBA0001F0D890015004E6180E005C000E01582D
:108CCA001BE2DECFE9FFDDCFEAFFD890E936EA36CC
:108CDA00410EE926010EEA22EE6AED6ADECFE9FFCD
:108CEA00DDCFEAFF290EE926010EEA22010EEF6E18
:108CFA00DF2ADBE3DB2AD9D7D586D59AD59CF2942D
:108D0A00F29AF1940F01498FBE0EC16ED08E7694FD
:108D1A00A386A5962DEC0BF016EC74F0F28EF28C6D
:108D2A007684040EE15C02E2E16AE552E16EE55204
:108D3A00E5CFDAFFE7CFD9FF1200D9CFE6FFDACFC6
:108D4A00E6FFE1CFD9FFE2CFDAFFE652E652E6527A
:108D5A00E652E652020EDB6A030EDB6A040EDB6A97
:108D6A00A0EC58F00701AE5100080AE2A9EC4EF057
:108D7A000701AD2B030EAD5D01E1AD6BAE07F2D776
:108D8A00B35100080AE2DDEC4EF00701B22B030EE4
:108D9A00B25D01E1B26BB307F3D7200E0201E76EB1
:108DAA008019E8AE02D0E73402D0E750805D01E2D4
:108DBA00C4D16550020B01E0C0D1400EE66E400EF0
:108DCA00E66E020EE66E36EC70F0E552E552E552BA
:108DDA00E76E030EE7CFDBFFDB50000801E328D183
:108DEA00040EDB6A030EDB50F36E040EDBCFF4FFD6
:108DFA00F350F45C01E31CD1040EDB50EA6A400F25
:108E0A00E96E020EEA22EFCFDFFF06015D5141E172
:108E1A000D0E006EDF50005C05E00A0E016EDF5099
:108E2A00015C37E1010E5D6F0701DD51EA6A000F4F
:108E3A00E96E030EEA220D0EEF6EDD2B010EDB6AE0
:108E4A00DD51F36E010EDBCFF4FFF350F45C1CE24C
:108E5A00010EDBCFE9FFEA6AE9BEEA68000EE926FD
:108E6A00030EEA22EF50E66E010EDBCFE9FFEA6A53
:108E7A00E9BEEA68190EE926060EEA22E552E7502B
:108E8A00EF6E010EDB2ADCD7F0D90701DD6BDE6B52
:108E9A00BFD01B0EDF5C09E1595107E1010E596F82
:108EAA001B0E5A6F5B6B5C6BB3D059050BE15B0E03
:108EBA00DF5C08E11B0E5A5D05E15B5103E15B0EC5
:108ECA005B6FA6D059056AE1410EDF5C67E11B0EB4
:108EDA005A5D64E15B0E5B5D61E15A6B5B6B5C6BD7
:108EEA00596B010EDB6ADBCFE9FFEA6AE9BEEA6881
:108EFA00000EE926030EEA22EF500D081CE0010ECF
:108F0A00DBCFE9FFEA6AE9BEEA68190EE926060E2E
:108F1A00EA22EF50E66E010EDBCFE9FFEA6AE9BE0C
:108F2A00EA68000EE926030EEA22E552E750EF6EE0
:108F3A00010EDB2AD8D7010EDBCFDDF70701DD51A1
:108F4A00EA6A000FE96E030EEA22EF6AB70E006EB4
:108F5A00DE0E016E026A00C0E6FFE66E02C0E6FFA0
:108F6A001FEC79F0E552E552E552000EE66E030E6B
:108F7A00E66EB40E006EDE0E016E026A00C0E6FFF7
:108F8A00E66E02C0E6FF1FEC79F0036E050EE15CA7
:108F9A0002E2E16AE552E16E03503AD0080EDF5C64
:108FAA001CE10701DD51000818E2DD07DD51EA6A1C
:108FBA00000FE96E030EEA22EF6AB10E006EDE0EB2
:108FCA00016E026A00C0E6FFE66E02C0E6FF1FEC11
:108FDA0079F0E552E552E5521BD00D0EDF5C18E040
:108FEA000A0EDF5C15E0200EDF5C12E306015A6B05
:108FFA005B6B5C6B596B0701DD51EA6A000FE96E26
:10900A00030EEA22DFCFEFFF06015D6B0701DD2BBE
:10901A000701DD51006E016A000E001806E1010E1B
:10902A00011803E1B487DD6BDE6B040EDB2ADAD6A6
:10903A000701B45101E180D0B4A10FD0AB0E006E8C
:10904A00DE0E016E026A00C0E6FFE66E02C0E6FFAF
:10905A001FEC79F0E552E552E5520701B4A30FD0AF
:10906A008C0E006EDE0E016E026A00C0E6FFE66E2E
:10907A0002C0E6FF1FEC79F0E552E552E55207011E
:10908A00B4A50FD0700E006EDE0E016E026A00C02B
:10909A00E6FFE66E02C0E6FF1FEC79F0E552E55204
:1090AA00E5520701B4A70FD0540E006EDE0E016E12
:1090BA00026A00C0E6FFE66E02C0E6FF1FEC79F026
:1090CA00E552E552E5520701B4A90FD0350E006EFC
:1090DA00DE0E016E026A00C0E6FFE66E02C0E6FF1F
:1090EA001FEC79F0E552E552E5520701B4AD0FD015
:1090FA00140E006EDE0E016E026A00C0E6FFE66E16
:10910A0002C0E6FF1FEC79F0E552E552E552000E87
:10911A000701B4150FE0FB0E006EDD0E016E026A48
:10912A0000C0E6FFE66E02C0E6FF1FEC79F0E552EA
:10913A00E552E5520701B46B47D8050EE15C02E23D
:10914A00E16AE552E16EE552E5CFDAFFE7CFD9FFF2
:10915A001200D9CFE6FFDACFE6FFE1CFD9FFE2CF9F
:10916A00DAFFE652DBC7DFFFDF2A400E006EDF5070
:10917A00005C01E1DF6A0701DC51DF5C01E124D810
:10918A000701DB51EA6A000FE96E020EEA22FD0EC0
:10919A00DBCFEFFFDB2B400EDB5D01E1DB6BDC514C
:1091AA00DB5D01E1B485FD0EDBCF00F0016A00BE94
:1091BA00016800C0F3FF01C0F4FFE552E552E5CFB4
:1091CA00DAFFE7CFD9FF1200D9CFE6FFDACFE6FF01
:1091DA00E1CFD9FFE2CFDAFFE6520701DB51DC5DCE
:1091EA003DE00701905105E046EC71F09BEC5AF026
:1091FA00F8D70701DC51D880DB5517E2DC51DB5D7B
:10920A00DF6EDFCFE6FFDC51016A000F006E020E4F
:10921A00012200C0E6FF01C0E6FFA0EC70F0E552B3
:10922A00E552E552DBC7DCF717D0400ED880DC5593
:10923A00DF6EDFCFE6FFDC51016A000F006E020E1F
:10924A00012200C0E6FF01C0E6FFA0EC70F0E55283
:10925A00E552E5520701DC6B46EC71F0E552E55246
:10926A00E5CFDAFFE7CFD9FF1200D9CFE6FFDACF91
:10927A00E6FFE1CFD9FFE2CFDAFFE652E652E65245
:10928A00E652DE6ADD6A020EDB6A030EDB6A07015A
:10929A00DE51EA6A000FE96E030EEA22EF50E66E2B
:1092AA00E66A2DEC7AF0E552E552020EF3CFDBFFC7
:1092BA000701DE2BDE51006E016A000E001804E180
:1092CA00010E011801E1DE6B020EDB50DE6EDD6A73
:1092DA00DE51EA6A000FE96E030EEA22EF502C080B
:1092EA0036E0DE51EA6A000FE96E030EEA22EF5019
:1092FA000D082DE0DE51EA6A000FE96E030EEA223C
:10930A00EF50E66EE66A2DEC7AF0E552E552030E6E
:10931A00F3CFDBFF0701DE2BDE51006E016A000E80
:10932A00001804E1010E011801E1DE6B020EDBCF29
:10933A0002F002C003F0026A030EDB5000010224AD
:10934A00006E000E0320016E00C0DEFFDD6E000E0F
:10935A00DFCF3AF0010EDBCF3BF0530E3A1802E1B1
:10936A00430E3B1801E113D2530E3A1802E1510E93
:10937A003B1801E109D24D0E3A1802E1580E3B188A
:10938A0001E1FFD1530E3A1802E1450E3B1801E103
:10939A00F5D1430E3A1802E1410E3B1801E1ECD136
:1093AA004D0E3A1802E1510E3B1801E1E2D14D0E81
:1093BA003A1802E1520E3B1801E1D8D1320E3A189E
:1093CA0002E1530E3B1801E1CED1450E3A1802E1F3
:1093DA00530E3B1801E1C4D1430E3A1802E1510E73
:1093EA003B1801E1BAD14B0E3A1802E1430E3B1881
:1093FA0001E1B0D14C0E3A1802E1420E3B1801E1EC
:10940A00A6D1440E3A1802E14E0E3B1801E19CD156
:10941A00490E3A1802E14E0E3B1801E192D1420E72
:10942A003A1802E1510E3B1801E188D14C0E3A1864
:10943A0002E1510E3B1801E17ED14C0E3A1802E1CD
:10944A00530E3B1801E174D14E0E3A1802E1510E47
:10945A003B1801E16AD14E0E3A1802E1530E3B184D
:10946A0001E160D1430E3A1802E1530E3B1801E1C3
:10947A0056D14D0E3A1802E1450E3B1801E14CD186
:10948A00500E3A1802E1510E3B1801E142D1500E3A
:10949A003A1802E1540E3B1801E138D1500E3A183D
:1094AA0002E1530E3B1801E12ED14D0E3A1802E1AA
:1094BA00410E3B1801E124D14D0E3A1802E1530E38
:1094CA003B1801E11AD1470E3A1802E1500E3B1837
:1094DA0001E110D1430E3A1802E1500E3B1801E1A6
:1094EA0006D1490E3A1802E1430E3B1801E1FCD0BD
:1094FA00490E3A1802E1520E3B1801E1F2D0490E28
:10950A003A1802E1530E3B1801E1E8D0530E3A181B
:10951A0002E1520E3B1801E1DED0530E3A1802E185
:10952A00530E3B1801E1D4D0530E3A1802E1420E11
:10953A003B1801E1CAD0430E3A1802E1420E3B1829
:10954A0001E1C0D0430E3A1802E1520E3B1801E184
:10955A00B6D04F0E3A1802E1420E3B1801E1ACD0E8
:10956A00570E3A1802E14D0E3B1801E1A2D0520EF5
:10957A003A1802E14D0E3B1801E198D0440E3A1810
:10958A0002E1500E3B1801E18ED04F0E3A1802E16B
:10959A00500E3B1801E184D0490E3A1802E1500EF0
:1095AA003B1801E17AD0580E3A1802E1540E3B18E2
:1095BA0071E0540E3A1801E13B506AE0410E3A1844
:1095CA0001E13B5063E0560E3A1801E13B505CE082
:1095DA00490E3A1801E13B5055E04F0E3A1801E1A5
:1095EA003B504EE0550E3A1802E1430E3B1846E056
:1095FA00580E3A1802E1430E3B183DE0430E3A1862
:10960A0001E13B5036E0520E3A1801E13B502FE09F
:10961A00580E3A1802E1520E3B1826E04D0E3A183F
:10962A0002E14C0E3B181DE0030EDB5001E0B2D004
:10963A00020EDBCFE6FFE66ADBCFE6FFE66AD80E6C
:10964A00006EDD0E016E026A00C0E6FFE66E02C021
:10965A00E6FF1FEC79F0036E070EE15C01E3BCD074
:10966A00B9D039EC12F0BAD097EC52F0B7D0EED8A4
:10967A00B5D0ABD9B3D099EC52F0B0D0EBD8AED0CC
:10968A00D3DAACD061DBAAD083DBA8D091DBA6D039
:10969A004CD9A4D095EC52F0A1D0EDEC50F09ED06C
:1096AA00ABEC51F09BD001EC50F098D0B5EC4FF0F8
:1096BA0095D071EC4FF092D059EC53F08FD09BECCF
:1096CA0052F08CD057EC53F089D05BEC53F086D033
:1096DA005DEC53F083D05FEC53F080D061EC53F033
:1096EA007DD063EC53F07AD065EC53F077D067EC19
:1096FA0053F074D004EC54F071D092EC14F06ED0A4
:10970A0048EC0DF06BD002EC21F068D0C8EC20F0E8
:10971A0065D0A9EC20F062D0DFEC21F05FD007EC35
:10972A000CF05CD08CEC22F059D0C5EC22F056D06B
:10973A00E3EC22F053D0F6EC22F050D015EC23F0F3
:10974A004DD06EEC22F04AD07FEC22F047D04EEC9E
:10975A0054F044D056EC54F041D036EC23F03ED0CD
:10976A0056EC23F03BD0C3EC74F038D033EC24F041
:10977A0035D034EC24F032D01DDA30D0BCEC1FF0F6
:10978A002DD025EC17F02AD03EEC25F027D0A1ECFD
:10979A0025F024D0030EDBCFE6FFE66A020EDBCF0C
:1097AA00E6FFE66A030EDBCFE6FFE66A020EDBCFD0
:1097BA00E6FFE66AB00E006EDD0E016E026A00C0B8
:1097CA00E6FFE66E02C0E6FF1FEC79F0036E0B0EB1
:1097DA00E15C02E2E16AE552E16E03500701DE5103
:1097EA00EA6A000FE96E030EEA22EF500D080DE057
:1097FA00B4510BE1520E006E016ADF50001803E10A
:10980A00DE52DD50011801E0B48FDDC7DEF7040E29
:10981A00E15C02E2E16AE552E16EE552E5CFDAFF88
:10982A00E7CFD9FF12000701E3510FE0EE0E006EF9
:10983A00F40E016E026A00C0E6FFE66E02C0E6FFA1
:10984A001FEC79F0E552E552E5521200A0EC45F022
:10985A0018EF4CF0D9CFE6FFDACFE6FFE1CFD9FF18
:10986A00E2CFDAFFE652E652E652E66AD9CFE6FFDF
:10987A00DACFE6FF010EE66EBCEC55F0E552E55292
:10988A00E552E552E66AD950010FE66E000EDA207B
:10989A00E66E020EE66EBCEC55F0E552E552E55274
:1098AA00E5520701B45138E1DF0418E1D950010F3C
:1098BA00E96E000EDA20EA6EEE50ED100AE0010EB3
:1098CA00006E016ADB50001808E1020EDB50011835
:1098DA0004E1010EDBCFE3F701D0B48D020E006E76
:1098EA00DF50005C18E1D950010FE96E000EDA2052
:1098FA00EA6EEE50ED100AE0010E006E016ADB50CE
:10990A00001808E1020EDB50011804E1010EDBCF5A
:10991A00BFFE01D0B48D87DFE552E552E552E5522C
:10992A00E5CFDAFFE7CFD9FF1200D9CFE6FFDACFCA
:10993A00E6FFE1CFD9FFE2CFDAFFE652E652E6527E
:10994A00020EDB6AE66AA80EE66E070EE66E030EE4
:10995A00E66EBCEC55F0E552E552E552E552E66A90
:10996A00D950020FE66E000EDA20E66E010EE66EA0
:10997A00BCEC55F0E552E552E552E5520701B45107
:10998A001BE1020EDB500CE1A851A91103E1AA6BFD
:10999A00AB6B11D07684A8C7AAF7A9C7ABF70BD0CF
:1099AA00A851A91103E1AF6BB06B05D07684A8C7A3
:1099BA00AFF7A9C7B0F737DFE552E552E552E552EE
:1099CA00E5CFDAFFE7CFD9FF1200D9CFE6FFDACF2A
:1099DA00E6FFE1CFD9FFE2CFDAFFE652E652E652DE
:1099EA00E652E652E66AD9CFE6FFDACFE6FF010E83
:1099FA00E66EBCEC55F0E552E552E552E552E66AF0
:109A0A00D950010FE66E000EDA20E66E010EE66E00
:109A1A00BCEC55F0E552E552E552E552E66AD950FA
:109A2A00020FE66E000EDA20E66E010EE66EBCEC60
:109A3A0055F0E552E552E552E552E66AD950030F70
:109A4A00E66E000EDA20E66E010EE66EBCEC55F00C
:109A5A00E552E552E552E552E66AD950040FE66E40
:109A6A00000EDA20E66E010EE66EBCEC55F0E55209
:109A7A00E552E552E5520701B4510FE1DF50926E0B
:109A8A00010EDB50936E020EDB50946E030EDB5018
:109A9A00956E040EDB50966EC6DE050EE15C02E2A0
:109AAA00E16AE552E16EE552E5CFDAFFE7CFD9FF89
:109ABA001200D9CFE6FFDACFE6FFE1CFD9FFE2CF36
:109ACA00DAFFFD0EDB50100805E2100EF36EFD0EF4
:109ADA00F3CFDBFFFC0EDB5032E0FD0EDB50D4ECA3
:109AEA007AF0F3500701BE13F450BF13080EF36E59
:109AFA00FD0EDBCFF4FFF350F45C0EE2010EF36EC1
:109B0A00FD0EDB5004E0D890F336E806FCE1F35092
:109B1A00F31C0F01481748D0FD0EDB500C0844E334
:109B2A00FD0EDB50F80F006E010E005204E0E8460D
:109B3A00FE0B0006FCE1E81C0F01491735D0FD0EAB
:109B4A00DB50D4EC7AF0F3CF00F0F4CF01F0001E32
:109B5A00011E00500701BE170150BF17080EF36E11
:109B6A00FD0EDBCFF4FFF350F45C0DE2010EF36E51
:109B7A00FD0EDB5004E0D890F336E806FCE1F35022
:109B8A000F01481311D0FD0EDB500C080DE3FD0E3A
:109B9A00DB50F80F006E010E005204E0E846FE0B9F
:109BAA000006FCE10F014913E552E5CFDAFFE7CFE2
:109BBA00D9FF1200D9CFE6FFDACFE6FFE1CFD9FF0E
:109BCA00E2CFDAFFE652E652E66AD9CFE6FFDACF0B
:109BDA00E6FF010EE66EBCEC55F0E552E552E552A1
:109BEA00E552E66AD950010FE66E000EDA20E66EFB
:109BFA00010EE66EBCEC55F0E552E552E552E5522F
:109C0A000701B45109E1010EDBCFE6FFDFCFE6FF22
:109C1A0050DFE552E55207DEE552E552E552E5CF5F
:109C2A00DAFFE7CFD9FF1200D9CFE6FFDACFE6FF96
:109C3A00E1CFD9FFE2CFDAFFE652E652E66AD9CFA0
:109C4A00E6FFDACFE6FF010EE66EBCEC55F0E55210
:109C5A00E552E552E552E76E010EE7CFDBFF070159
:109C6A00B4516AE1010EDB5002E1DF50896E010E48
:109C7A00E66ED9CFE6FFDACFE6FFE66EBCEC55F02A
:109C8A00E552E552E552E552E76E010EE7CFDBFFFA
:109C9A000701B45151E1010EDB5002E1DF508A6E37
:109CAA00010EE66ED9CFE6FFDACFE6FFE66EBCEC30
:109CBA0055F0E552E552E552E552E76E010EE7CF5F
:109CCA00DBFF0701B45138E1010EDB5002E1DF503E
:109CDA008B6E010EE66ED9CFE6FFDACFE6FFE66EAF
:109CEA00BCEC55F0E552E552E552E552E76E010E3D
:109CFA00E7CFDBFF0701B4511FE1010EDB5002E1A0
:109D0A00DF508C6E010EE66ED9CFE6FFDACFE6FFA2
:109D1A00E66EBCEC55F0E552E552E552E552E76EC7
:109D2A00010EE7CFDBFF0701B45106E1010EDB505C
:109D3A0002E1DF508D6E77DDE552E552E552E5CF5F
:109D4A00DAFFE7CFD9FF12008450E66EE66A835045
:109D5A00E66EE66A8250E66EE66A8150E66EE66A6A
:109D6A008050E66EE66A930E006EDD0E016E026AA0
:109D7A0000C0E6FFE66E02C0E6FF1FEC79F0036E54
:109D8A000D0EE15C02E2E16AE552E16E0350120057
:109D9A00F60E006EF40E016E026A00C0E6FFE66E71
:109DAA0002C0E6FF1FEC79F0E552E552E5521200D7
:109DBA00D9CFE6FFDACFE6FFE1CFD9FFE2CFDAFF6C
:109DCA00E652E652E652DF6A010EF36EDB6E020ECF
:109DDA00DB6A910E006EDD0E016E026A00C0E6FFBC
:109DEA00E66E02C0E6FF1FEC79F0E552E552E55255
:109DFA009DBCFED7DF6ADFCF00F0100EE76E0018B9
:109E0A00E8AE02D0E73402D0E750005C4DE2010E22
:109E1A00DB500701BE150001006E020EDB50070180
:109E2A00BF150001016E005001102DE0DFCFE9FFE0
:109E3A00EA6AE9BEEA68D890E936EA36000EE92607
:109E4A00010EEA22EECFE6FFEFCFE6FFDFCF00F00A
:109E5A00016A00BE016800C0E6FF01C0E6FF860E87
:109E6A00026EDD0E036E046A02C0E6FFE66E04C0EF
:109E7A00E6FF1FEC79F0056E070EE15C02E2E16A8B
:109E8A00E552E16E0550010EDBCF00F0020EDBCF8A
:109E9A0001F0D89000360136010E00C0DBFF020E39
:109EAA0001C0DBFFDF2AA7D7F30E006EF40E016EA6
:109EBA00026A00C0E6FFE66E02C0E6FF1FEC79F018
:109ECA00E552E552E552E552E552E552E552E5CF53
:109EDA00DAFFE7CFD9FF1200D9CFE6FFDACFE6FFE4
:109EEA00E1CFD9FFE2CFDAFFE652E652E652E66A5E
:109EFA00D9CFE6FFDACFE6FF030EE66EBCEC55F0EB
:109F0A00E552E552E552E552E66AD950020FE66E8D
:109F1A00000EDA20E66E010EE66EBCEC55F0E55254
:109F2A00E552E552E5520701B45111E1DECF00F0E6
:109F3A00DDCF01F0000E005C100E015807E2DECF03
:109F4A00E9FFDDCFEAFF020EDBCFEFFF6CDCE55263
:109F5A00E552E552E552E5CFDAFFE7CFD9FF120025
:109F6A00D9CFE6FFDACFE6FFE1CFD9FFE2CFDAFFBA
:109F7A00E652E652E652E66AD9CFE6FFDACFE6FFC4
:109F8A00030EE66EBCEC55F0E552E552E552E55299
:109F9A000701B45128E1DECF00F0DDCF01F0000E59
:109FAA00005C100E015807E2DECFE9FFDDCFEAFFC1
:109FBA00020EEFCFDBFF020EDBCFE6FFE66A7C0E76
:109FCA00006EDD0E016E026A00C0E6FFE66E02C098
:109FDA00E6FF1FEC79F0036E050EE15C02E2E16A2E
:109FEA00E552E16E0350E552E552E552E552E5CFFE
:109FFA00DAFFE7CFD9FF1200D9CFE6FFDACFE6FFC3
:10A00A00E1CFD9FFE2CFDAFFE652E652E652E66A3C
:10A01A00D9CFE6FFDACFE6FF050EE66EBCEC55F0C7
:10A02A00E552E552E552E552E66AD950010FE66E6D
:10A03A00000EDA20E66E010EE66EBCEC55F0E55233
:10A04A00E552E552E552E66AD950020FE66E000E75
:10A05A00DA20E66E010EE66EBCEC55F0E552E552EA
:10A06A00E552E5520701B45101E0A9D0020EDB50D6
:10A07A00010801E2A0D0010EDB50070801E29BD0E3
:10A08A00410E006EDF50005C1AE1020EDB500CE15B
:10A09A00010EF36EDB5004E0D890F336E806FCE1DB
:10A0AA00F350F31C921689D0010EF36EDB5004E0D4
:10A0BA00D890F336E806FCE1F35092127ED0420EB5
:10A0CA00006EDF50005C1AE1020EDB500CE1010E5B
:10A0DA00F36EDB5004E0D890F336E806FCE1F35067
:10A0EA00F31C93166AD0010EF36EDB5004E0D8908D
:10A0FA00F336E806FCE1F35093125FD0430E006E8C
:10A10A00DF50005C1AE1020EDB500CE1010EF36E27
:10A11A00DB5004E0D890F336E806FCE1F350F31C78
:10A12A0094164BD0010EF36EDB5004E0D890F33650
:10A13A00E806FCE1F350941240D0440E006EDF5062
:10A14A00005C1AE1020EDB500CE1010EF36EDB50EB
:10A15A0004E0D890F336E806FCE1F350F31C9516B8
:10A16A002CD0010EF36EDB5004E0D890F336E806EB
:10A17A00FCE1F350951221D0450E006EDF50005CD1
:10A18A001AE1020EDB500CE1010EF36EDB5004E023
:10A19A00D890F336E806FCE1F350F31C96160DD07E
:10A1AA00010EF36EDB5004E0D890F336E806FCE1CA
:10A1BA00F350961202D0B48D02D018EC4CF0E5524E
:10A1CA00E552E552E552E5CFDAFFE7CFD9FF1200B3
:10A1DA00D9CFE6FFDACFE6FFE1CFD9FFE2CFDAFF48
:10A1EA00E652E652E652020EDB6AE66AD9CFE6FF8B
:10A1FA00DACFE6FF050EE66EBCEC55F0E552E55205
:10A20A00E552E552E66AD950010FE66E000EDA20F1
:10A21A00E66E010EE66EBCEC55F0E552E552E552EB
:10A22A00E5520701B45101E088D0010EDB5007085E
:10A23A0065E3410E006EDF50005C0EE1010EDB2883
:10A24A00006E010E005204E0E846FE0B0006FCE137
:10A25A00E8407F0B80144BD0420E006EDF50005C4A
:10A26A000EE1010EDB28006E010E005204E0E84602
:10A27A00FE0B0006FCE1E8407F0B811438D0430E48
:10A28A00006EDF50005C0EE1010EDB28006E010E4D
:10A29A00005204E0E846FE0B0006FCE1E8407F0BB2
:10A2AA00821425D0440E006EDF50005C0EE1010ED0
:10A2BA00DB28006E010E005204E0E846FE0B0006A1
:10A2CA00FCE1E8407F0B831412D0450E006EDF508C
:10A2DA00005C14E1010EDB28006E010E005204E05E
:10A2EA00E846FE0B0006FCE1E8407F0B8414E76EAB
:10A2FA00020EE7CFDBFFDB5008E002D0B48D1DD0A1
:10A30A00010EF36E020EF3CFDBFF020EDBCFE6FF88
:10A31A00E66A730E006EDD0E016E026A00C0E6FF89
:10A32A00E66E02C0E6FF1FEC79F0036E050EE15CF3
:10A33A0002E2E16AE552E16E0350E552E552E55266
:10A34A00E552E5CFDAFFE7CFD9FF1200D9CFE6FF12
:10A35A00DACFE6FFE1CFD9FFE2CFDAFFE652E652E3
:10A36A00E652E66AD9CFE6FFDACFE6FF050EE66ED9
:10A37A00BCEC55F0E552E552E552E552E66AD95091
:10A38A00010FE66E000EDA20E66E010EE66EEFDBD6
:10A39A00E552E552E552E552E66AD950020FE66EF9
:10A3AA00000EDA20E66E010EE66EE1DBE552E552BA
:10A3BA00E552E5520701B45101E0A9D0020EDB5083
:10A3CA00010801E2A0D0010EDB50070801E29BD090
:10A3DA00410E006EDF50005C1AE1020EDB500CE108
:10A3EA00010EF36EDB5004E0D890F336E806FCE188
:10A3FA00F350F31C891689D0010EF36EDB5004E08A
:10A40A00D890F336E806FCE1F35089127ED0420E6A
:10A41A00006EDF50005C1AE1020EDB500CE1010E07
:10A42A00F36EDB5004E0D890F336E806FCE1F35013
:10A43A00F31C8A166AD0010EF36EDB5004E0D89042
:10A44A00F336E806FCE1F3508A125FD0430E006E41
:10A45A00DF50005C1AE1020EDB500CE1010EF36ED4
:10A46A00DB5004E0D890F336E806FCE1F350F31C25
:10A47A008B164BD0010EF36EDB5004E0D890F33606
:10A48A00E806FCE1F3508B1240D0440E006EDF5018
:10A49A00005C1AE1020EDB500CE1010EF36EDB5098
:10A4AA0004E0D890F336E806FCE1F350F31C8C166E
:10A4BA002CD0010EF36EDB5004E0D890F336E80698
:10A4CA00FCE1F3508C1221D0450E006EDF50005C87
:10A4DA001AE1020EDB500CE1010EF36EDB5004E0D0
:10A4EA00D890F336E806FCE1F350F31C8D160DD034
:10A4FA00010EF36EDB5004E0D890F336E806FCE177
:10A50A00F3508D1202D0B48D02D018EC4CF0E55203
:10A51A00E552E552E552E5CFDAFFE7CFD9FF12005F
:10A52A0018EF4CF018EF4CF018EF4CF0D9CFE6FFCB
:10A53A00DACFE6FFE1CFD9FFE2CFDAFFE652E65201
:10A54A00E652E652E66AD9CFE6FFDACFE6FF050E13
:10A55A00E66E0DDBE552E552E552E552E66AD95060
:10A56A00010FE66E000EDA20E66E010EE66EFFDAE5
:10A57A00E552E552E552E552E66AD950020FE66E17
:10A58A00000EDA20E66E030EE66EF1DAE552E552C7
:10A59A00E552E5520701B45101E078D0D950020FD3
:10A5AA00E96E000EDA20EA6E720ED880EE542E0E94
:10A5BA00ED5442E3D950020FE96E000EDA20EA6E3A
:10A5CA00EE50ED101FE003680468056A2D0EE76E71
:10A5DA00020EDBCF06F0030EDBCF07F0E7500626AC
:10A5EA00000E0722086A0650035C006E07500458E2
:10A5FA00016E08500558026E020E00C0DBFF030E02
:10A60A0001C0DBFF010EDB50070816E3410E006EA6
:10A61A00DF50005C02E1DF6A11D0420E006EDF50AB
:10A62A00005C02E1080E06D0430E006EDF50005CAB
:10A63A0003E1100EDF6E02D0B48D28D0010EDB507C
:10A64A00DF24E96EEA6AD890E936EA36410EE9264D
:10A65A00010EEA22020EDBCFEEFF030EDBCFEDFF87
:10A66A00010EDB50DF24EA6A290FE96E010EEA22A5
:10A67A00EF040AE1010EDB50DF24EA6A290FE96ED2
:10A68A00010EEA22020EEF6E18EC4CF0040EE15CA9
:10A69A0002E2E16AE552E16EE552E5CFDAFFE7CF81
:10A6AA00D9FF120018EF4CF018EF4CF018EF4CF0ED
:10A6BA0018EF4CF018EF4CF018EF4CF018EF4CF084
:10A6CA0018EF4CF0D9CFE6FFDACFE6FFE1CFD9FF9A
:10A6DA00E2CFDAFF070EE12402E3E168E652E16E17
:10A6EA00E66AD9CFE6FFDACFE6FF030EE66E3FDA77
:10A6FA00E552E552E552E552E66AD950020FE66E96
:10A70A00000EDA20E66E030EE66E31DAE552E55205
:10A71A00E552E5520701B45166E1DECF01F6DDCF1D
:10A72A0002F6020EDBCF09F6030EDBCF0AF6040EA1
:10A73A00DB6A030EF36E040EDBCFF4FFF350F45C16
:10A74A0050E2010EE66ED9CFE6FFDACFE6FF030E3E
:10A75A00E66E0DDAE552E552E552E552E76E050E70
:10A76A00E7CFDBFF010EE66ED950020FE66E000E50
:10A77A00DA20E66E030EE66EFAD9E552E552E552A4
:10A78A00E552E76E060EE7CFDBFF0701B4512BE176
:10A79A00050EDB5026E1060EDB5023E1040EDB2812
:10A7AA00E96EEA6AD890E936EA36010EE926060E1B
:10A7BA00EA22DECFEEFFDDCFEDFF040EDB28E96EE5
:10A7CA00EA6AD890E936EA36090EE926060EEA223E
:10A7DA00020EDBCFEEFF030EDBCFEDFF040EDB2A0A
:10A7EA00A8D718EC4CF0070EE15C02E2E16AE552E8
:10A7FA00E16EE552E5CFDAFFE7CFD9FF1200D9CFF4
:10A80A00E6FFDACFE6FFE1CFD9FFE2CFDAFFE65281
:10A81A00E66AD9CFE6FFDACFE6FF010EE66EA7D9E0
:10A82A00E552E552E552E5520701B4510DE1DF5018
:10A83A0007E0F00E9314936E0601010E006F02D02A
:10A84A000601006B18EC4CF0E552E552E5CFDAFF51
:10A85A00E7CFD9FF1200D9CFE6FFDACFE6FFE1CF83
:10A86A00D9FFE2CFDAFFE652DF6AFF0EDF5C0AE2C7
:10A87A00E868E85005E0E80600D000D000D0F9D733
:10A88A00DF2AF3D7E552E552E5CFDAFFE7CFD9FF62
:10A89A001200F29EF29C6592656ADDDF0FEF00F00E
:10A8AA001200D9CFE6FFDACFE6FFE1CFD9FFE2CF38
:10A8BA00DAFF100EE12402E3E168E652E16EE66A8D
:10A8CA00D950010FE66E000EDA20E66EE66A4FD91D
:10A8DA00E552E552E552E552E66AD9CFE6FFDACF0C
:10A8EA00E6FF010EE66E43D9E552E552E552E5521E
:10A8FA00E66AD950040FE66E000EDA20E66E020E02
:10A90A00E66E35D9E552E552E552E552E66AD95086
:10A91A00020FE66E000EDA20E66E030EE66E27D907
:10A92A00E552E552E552E552E66AD9500A0FE66E5B
:10A93A00000EDA20E66E060EE66E19D9E552E552E9
:10A94A00E552E552E66AD950060FE66E000EDA20A5
:10A95A00E66E070EE66E0BD9E552E552E552E55270
:10A96A00E66AD9500E0FE66E000EDA20E66E040E85
:10A97A00E66EFDD8E552E552E552E552E66AD9504F
:10A98A000F0FE66E000EDA20E66E050EE66EEFD8C1
:10A99A00E552E552E552E552010EDBCF00F0016ABD
:10A9AA0000BE016800C0E6FF01C0E6FF670E026E46
:10A9BA00DD0E036E046A02C0E6FFE66E04C0E6FF1F
:10A9CA001FEC79F0056E050EE15C02E2E16AE552E0
:10A9DA00E16E0550DFCFE6FFE66A5B0E006EDD0E24
:10A9EA00016E026A00C0E6FFE66E02C0E6FF1FECD7
:10A9FA0079F0036E050EE15C02E2E16AE552E16E6E
:10AA0A000350040EDBCFE6FF050EDBCFE6FF4F0E49
:10AA1A00006EDD0E016E026A00C0E6FFE66E02C03D
:10AA2A00E6FF1FEC79F0036E050EE15C02E2E16AD3
:10AA3A00E552E16E0350020EDBCFE6FF030EDBCFD9
:10AA4A00E6FF430E006EDD0E016E026A00C0E6FFED
:10AA5A00E66E02C0E6FF1FEC79F0036E050EE15CBC
:10AA6A0002E2E16AE552E16E0350D9500A0FE96E3B
:10AA7A00000EDA20EA6EEECFE6FFEECFE6FFEECF6B
:10AA8A00E6FFEFCFE6FF360E006EDD0E016E026ABC
:10AA9A0000C0E6FFE66E02C0E6FF1FEC79F0036E27
:10AAAA00070EE15C02E2E16AE552E16E0350D95019
:10AABA00060FE96E000EDA20EA6EEECFE6FFEECF61
:10AACA00E6FFEECFE6FFEFCFE6FF290E006EDD0EC2
:10AADA00016E026A00C0E6FFE66E02C0E6FF1FECE6
:10AAEA0079F0036E070EE15C02E2E16AE552E16E7B
:10AAFA0003500E0EDBCFE6FFE66A1D0E006EDD0E7A
:10AB0A00016E026A00C0E6FFE66E02C0E6FF1FECB5
:10AB1A0079F0036E050EE15C02E2E16AE552E16E4C
:10AB2A0003500F0EDBCFE6FFE66A110E006EDD0E54
:10AB3A00016E026A00C0E6FFE66E02C0E6FF1FEC85
:10AB4A0079F0036E050EE15C02E2E16AE552E16E1C
:10AB5A00035018EC4CF0100EE15C02E2E16AE55297
:10AB6A00E16EE552E5CFDAFFE7CFD9FF1200D9CF80
:10AB7A00E6FFDACFE6FFE1CFD9FFE2CFDAFF090E2F
:10AB8A00E12402E3E168E652E16E080EDB6A0D0E8B
:10AB9A00006E0701DE51EA6A000FE96E030EEA222F
:10ABAA00EF50005C05E1FA0EDB5049E1B48947D069
:10ABBA00DE51EA6A000FE96E030EEA22EF502C0812
:10ABCA0024E0FA0EDB501FE1DE51EA6A000FE96E5B
:10ABDA00030EEA22EF50E66EE66AEA0E006EDC0E1B
:10ABEA00016E026A00C0E6FFE66E02C0E6FF1FECD5
:10ABFA0079F0036E050EE15C02E2E16AE552E16E6C
:10AC0A0003500701B48B020EE5D1DE2BDE51006E34
:10AC1A00016A000E001804E1010E011801E1DE6B61
:10AC2A000D0E006EDE51EA6A000FE96E030EEA228B
:10AC3A00EF50005C06E1FA0EDB5001E1B489030E25
:10AC4A00C9D12D0E006EDE51EA6A000FE96E030EBD
:10AC5A00EA22EF50005C2EE1040E016EFD0EDB507D
:10AC6A00015C28E0050E026EFD0EDB50025C22E05C
:10AC7A00FD0EDB0401E147D1030E006EFD0EDB5031
:10AC8A00005C01E140D1070E016EFD0EDB50015C54
:10AC9A0001E139D1010EF36E080EF3CFDBFFDE2B93
:10ACAA00DE51006E016A000E001804E1010E01185F
:10ACBA0001E1DE6B040E006EFD0EDB50005C11E05C
:10ACCA00050E016EFD0EDB50015C0BE00A0EE66E0E
:10ACDA00D9CFE6FFDACFE6FF8BD9E552E552E55246
:10ACEA0042D0DE51EA6A000FE96E030EEA22EFCF84
:10ACFA0000F0000E00C0DFFF010EDB6A020EDB6A05
:10AD0A00030EDB6A050E006EFD0EDB50005C1FE1D0
:10AD1A00000EDFCFE6FF010EDBCFE6FF2DEC7AF067
:10AD2A00E552E552F3CF00F0F4CF01F0026A036A6C
:10AD3A0001AE02D00268036800C0DFFF010E01C045
:10AD4A00DBFF020E02C0DBFF030E03C0DBFF0701BD
:10AD5A00DE2BDE51006E016A000E001804E1010EBE
:10AD6A00011801E1DE6B080EDB506EE0FD0EDB50D0
:10AD7A000EE1D9CFE9FFDACFEAFFD880800EEE5490
:10AD8A00000EEE54000EEE54000EEE5428E3020EAE
:10AD9A00006EFD0EDB50005C0EE1D9CFE9FFDACF81
:10ADAA00EAFFD880000EEE54800EEE54000EEE54E8
:10ADBA00000EEE5414E3060E016EFD0EDB50015C2C
:10ADCA0010E1D9CFE9FFDACFEAFFD880000EEE54BE
:10ADDA00000EEE54000EEE54800EEE5402E207010D
:10ADEA0092D0D9CFE9FFDACFEAFF040EEECFDBFF2C
:10ADFA00050EEECFDBFF060EEECFDBFF070EEECF22
:10AE0A00DBFF080EDB5001E197D0040EDBCF38F0F0
:10AE1A00050EDBCF39F0060EDBCF3AF0070EDBCF9B
:10AE2A003BF03D683E683F684068F5EC79F0040EF7
:10AE3A0034C0DBFF050E35C0DBFF060E36C0DBFF74
:10AE4A00070E37C0DBFF78D0FD0EDB500EE1D9CFFD
:10AE5A00E9FFDACFEAFFD8807F0EEE54000EEE54F7
:10AE6A00000EEE54000EEE544DE3FD0EDB040EE12F
:10AE7A00D9CFE9FFDACFEAFFD880FF0EEE54000EF1
:10AE8A00EE54000EEE54000EEE543CE3020E006E39
:10AE9A00FD0EDB50005C0EE1D9CFE9FFDACFEAFF05
:10AEAA00D880FF0EEE547F0EEE54000EEE54000EC4
:10AEBA00EE5428E3030E016EFD0EDB50015C0EE139
:10AECA00D9CFE9FFDACFEAFFD880FF0EEE54FF0EA2
:10AEDA00EE54000EEE54000EEE5414E3060E026E0B
:10AEEA00FD0EDB50025C12E1D9CFE9FFDACFEAFFAF
:10AEFA00D880FF0EEE54FF0EEE54FF0EEE547F0E76
:10AF0A00EE5404E20701B48D010E64D0070E006E00
:10AF1A00FD0EDB50005C10E0D9CFE9FFDACFEAFF83
:10AF2A00040EEECFDBFF050EEECFDBFF060EEECFF3
:10AF3A00DBFF070EEECFDBFFFD0EDB50070A38E022
:10AF4A00010A25E0050A16E0010A14E0030A08E0EE
:10AF5A00050A06E0010A04E0050A02E0040E3AD0F6
:10AF6A00FB0EDBCFE9FFFC0EDBCFEAFF040EDBCFE3
:10AF7A00EFFF2FD0FB0EDBCFE9FFFC0EDBCFEAFFA2
:10AF8A00040EDBCFEEFF050EDBCFEDFF22D0FB0E6A
:10AF9A00DBCFE9FFFC0EDBCFEAFF040EDBCFEEFFCF
:10AFAA00050EDBCFEEFF060EDBCFEEFF070E0FD04E
:10AFBA00FB0EDBCFE9FFFC0EDBCFEAFFDFCFEEFFB4
:10AFCA00010EDBCFEEFF020EDBCFEEFF030EDBCF6F
:10AFDA00EEFF000E006E090EE15C02E2E16AE55244
:10AFEA00E16E0050E552E5CFDAFFE7CFD9FF120054
:10AFFA00D9CFE6FFDACFE6FFE1CFD9FFE2CFDAFF1A
:10B00A00E652E652FC0EDBCFE9FFFD0EDBCFEAFF8C
:10B01A00EE6AEE6AEE6AEE6A010EDB6AFB0EDB503E
:10B02A00F36E010EDBCFF4FFF350F45C62E207012A
:10B03A00DE51EA6A000FE96E030EEA22EFCFDFFF64
:10B04A00300EDF5C51E3DF5039084EE3FC0EDBCFF4
:10B05A00E9FFFD0EDBCFEAFFEECF00F0EECF01F005
:10B06A00EECF02F0EFCF03F00A0E3D6E3E6A3F6A62
:10B07A00406A00C038F001C039F002C03AF003C09B
:10B08A003BF0F5EC79F034C000F035C001F036C081
:10B09A0002F037C003F0300EDF5C046E056A066A00
:10B0AA00076AE8500026055001220650022207507E
:10B0BA000322FC0EDBCFE9FFFD0EDBCFEAFF00C067
:10B0CA00EEFF01C0EEFF02C0EEFF03C0EEFF070174
:10B0DA00DE2BDE51006E016A000E001807E1010E38
:10B0EA00011804E1DE6B02D0000E04D0010EDB2A47
:10B0FA0095D7010EE552E552E552E5CFDAFFE7CFE3
:10B10A00D9FF12000701AE51E66EE66ADE0E006E46
:10B11A00DC0E016E026A00C0E6FFE66E02C0E6FFC0
:10B12A001FEC79F0036E050EE15C02E2E16AE5527A
:10B13A00E16E035012000201805108E0010E006E18
:10B14A006550020B01E0010E005C1BE1060161077C
:10B15A00000E625B63510BE16151621111E18C8651
:10B16A00A00E616F0F0E626F010E636F12006151C4
:10B17A00621163E18C96A00E616F0F0E626F636BB2
:10B18A001200800509E0020E805D06E0040E805D73
:10B19A0003E0100E805D1BE106016107000E625B91
:10B1AA0063510BE16151621111E18C86200E616FCE
:10B1BA004E0E626F010E636F1200615162113DE122
:10B1CA008C96200E616F4E0E626F636B1200200E1A
:10B1DA00805D33E106016107000E625B63510AE19B
:10B1EA00615162112AE18C86100E616F270E626F1F
:10B1FA00010E18D063050AE1615162111EE18C96B5
:10B20A00100E616F270E626F020E0CD0020E635D84
:10B21A000BE16151621111E18C86A00E616F860EFD
:10B22A00626F030E636F12006151621106E18C9620
:10B23A00100E616F270E626F636B1200D9CFE6FFA3
:10B24A00DACFE6FFE1CFD9FFE2CFDAFFFD0EDBCF9F
:10B25A0000F0190EE76E0018E8AE02D0003403D0F1
:10B26A00E750D880005453E3FC0EDB5028E0FD0E73
:10B27A00DBCFE9FFEA6AE9BEEA68C80EE926060EEC
:10B28A00EA22EF50016E010E015204E0E846FE0B7D
:10B29A000106FCE1006EFD0EDBCFE9FFEA6AE9BEBA
:10B2AA00EA68D890E936EA36960EE926060EEA22C8
:10B2BA00EE50EFCFEAFFE96E0050EF1228D0FD0EF4
:10B2CA00DBCFE9FFEA6AE9BEEA68C80EE926060E9C
:10B2DA00EA22EF50016E010E015204E0E846FE0B2D
:10B2EA000106FCE1E81C006EFD0EDBCFE9FFEA6A0D
:10B2FA00E9BEEA68D890E936EA36960EE926060EDD
:10B30A00EA22EE50EFCFEAFFE96E0050EF16E5525F
:10B31A00E5CFDAFFE7CFD9FF1200D9CFE6FFDACFC0
:10B32A00E6FFE1CFD9FFE2CFDAFFFD0EDBCF00F077
:10B33A00190EE76E0018E8AE02D0003403D0E750C9
:10B34A00D880005453E3FC0EDB5029E1FD0EDBCF1D
:10B35A00E9FFEA6AE9BEEA68C80EE926060EEA22A9
:10B36A00EF50016E010E015204E0E846FE0B0106A1
:10B37A00FCE1E81C006EFD0EDBCFE9FFEA6AE9BEDC
:10B38A00EA68D890E936EA36640EE926060EEA2219
:10B39A00EE50EFCFEAFFE96E0050EF1627D0FD0E10
:10B3AA00DBCFE9FFEA6AE9BEEA68C80EE926060EBB
:10B3BA00EA22EF50016E010E015204E0E846FE0B4C
:10B3CA000106FCE1006EFD0EDBCFE9FFEA6AE9BE89
:10B3DA00EA68D890E936EA36640EE926060EEA22C9
:10B3EA00EE50EFCFEAFFE96E0050EF12E552E5CFDB
:10B3FA00DAFFE7CFD9FF1200D9CFE6FFDACFE6FFAF
:10B40A00E1CFD9FFE2CFDAFFE652A098636A626A17
:10B41A000F01266B020EE66EE66AE66A270EE66EF4
:10B42A000F0EE66ED2EC78F0006E050EE15C02E2D9
:10B43A00E16AE552E16E00500F01160E396F9F0E58
:10B44A00376F7B0E366FDF6ADF50006E016A0C0EB3
:10B45A00005C000E015810E2DF50040DF3CFE9FF43
:10B46A00F4CFEAFF000EE926040EEA22EE6AEE6A3B
:10B47A00EE6AEE6ADF2AE8D7658C0F01386B6598A9
:10B48A00659C62A607D062960201976B9C6B9D6BC6
:10B49A009E6BF7D70201010EB06FB16FB26BB36B3F
:10B4AA00A46BDF6A030EDF5C26E2EA6ADF34FE0B76
:10B4BA00EA36E96E8D0EE926020EEA22EE6AED6A96
:10B4CA00EA6ADF34FE0BEA36E96E870EE926020ED7
:10B4DA00EA22EE6AED6ADF50EA6AA80FE96E020E06
:10B4EA00EA22EF6ADF50EA6AAB0FE96E020EEA223D
:10B4FA00EF6ADF2AD7D70201080E8D6F040E8E6F0E
:10B50A000F01160E266F0401300E026F040E036F30
:10B51A00400E016F840E006F0201816B806BE55251
:10B52A00E552E5CFDAFFE7CFD9FF1200D9CFE6FF20
:10B53A00DACFE6FFE1CFD9FFE2CFDAFFE65282BEE9
:10B54A0006D0656A0F01366B0201806B90D002014A
:10B55A00805110E1656A0F01366B160E396F9F0E26
:10B56A00376F7B0E366F65B602D06586FCD702014F
:10B57A00010E806F80050AE165BA08D0626A0F0180
:10B58A00366B368136890201020E806F6250040BD7
:10B59A0007E00F013651040B03E06294CEEC60F031
:10B5AA0065B265D06250010B09E00F013651010BFB
:10B5BA0005E022DF0201040E806F62906250100BD8
:10B5CA0007E00F013651100B03E0B4EC60F062980B
:10B5DA0062AC1ED00F0136AD13D0010EE66EE66ADC
:10B5EA00000EE66EE66A730EE66EE66A7CEC76F0AC
:10B5FA00006E060EE15C02E2E16AE552E16E00507D
:10B60A00629C0201AE5101E0AE07AE5101E1F8D9E8
:10B61A006250200B06E00F013651200B02E09AEC33
:10B62A0060F06250020B18E00F013651020B14E071
:10B63A00010EE66EE66A000EE66EE66AE6687F0EC0
:10B64A00E66E7CEC76F0006E060EE15C02E2E16AE0
:10B65A00E552E16E0050636A040E0201E76E80193A
:10B66A00E8AE02D0E73402D0E750805D02E2A1984A
:10B67A003ED00F0136A73AD0DF6A040EDF5C36E20D
:10B68A0062A634D064CFA5F20201A551780BE84234
:10B69A00E842E842A66F6296A5B506D0A651EA6AC4
:10B6AA00AB0FE96E020E05D0A651EA6AA80FE96E41
:10B6BA00020EEA22EF70A65103E1EAEC60F014D020
:10B6CA00000EE66EE66AA50EE66E020EE66E720ED3
:10B6DA00E66EE66A7CEC76F0006E060EE15C02E24B
:10B6EA00E16AE552E16E0050DF2AC7D7A198E55218
:10B6FA00E552E5CFDAFFE7CFD9FF1200D9CFE6FF4F
:10B70A00DACFE6FFE1CFD9FFE2CFDAFFE652E6521F
:10B71A00FC0EDBA407D0E66AFD0EDBCFE6FFFFD9FD
:10B72A00E552E552FC0EDBA208D0010EE66EFD0ED4
:10B73A00DBCFE6FFF4D9E552E552FD0EDB50016A94
:10B74A00260F006E0F0E012200C0DEFF01C0DDFFD2
:10B75A00DECFE9FFDDCFEAFFFC0EDBCFEFFFE552DC
:10B76A00E552E552E5CFDAFFE7CFD9FF1200D9CF8C
:10B77A00E6FFDACFE6FFE1CFD9FFE2CFDAFFE65202
:10B78A00E652FC0EDB500AE0FD0EEA6ADB34FE0BE1
:10B79A00EA36E96E8D0EE926020E09D0FD0EEA6A36
:10B7AA00DB34FE0BEA36E96E870EE926020EEA2240
:10B7BA00EECFDEFFEDCFDDFFD9CFE9FFDACFEAFF2B
:10B7CA00EE50ED1003E1F36AF46A44D0DECFE9FFEC
:10B7DA00DDCFEAFF020EE926000EEA22FA0EDBCFDF
:10B7EA00EEFFFB0EDBCFEDFFDECFE9FFDDCFEAFF99
:10B7FA00EE52F90EDBCFEFFF400EDECFE9FFDDCFD1
:10B80A00EAFFE850EF16880EDECFE9FFDDCFEAFF48
:10B81A00E850EF12FC0EDB500AE0FD0EEA6ADB3458
:10B82A00FE0BEA36E96E8D0EE926020E09D0FD0EF0
:10B83A00EA6ADB34FE0BEA36E96E870EE926020E67
:10B84A00EA22EF74DECF00F0DDCF01F000C0F3FF93
:10B85A0001C0F4FFE552E552E552E5CFDAFFE7CF42
:10B86A00D9FF1200D9CFE6FFDACFE6FFE1CFD9FF41
:10B87A00E2CFDAFFE652E652FD0EDB5020E185C246
:10B88A00E9FF86C2EAFFEE52400EEF6E85C2E9FF7B
:10B89A0086C2EAFF020EE926000EEA22300EEE6E9A
:10B8AA00040EED6E85C2E9FF86C2EAFF8C0EEF6ECA
:10B8BA008DC2E9FF8EC2EAFF840EEF6E3BD0FC0E0A
:10B8CA00DB50E824026EFD0EDB50040DF350022417
:10B8DA00040DF3CF00F0F4CF01F0000E0026040EA1
:10B8EA00012200C0DEFF01C0DDFF840EDECFE9FFCA
:10B8FA00DDCFEAFFE850EF12FC0EDB50E824026EBF
:10B90A00FD0EDB50040DF3500224010F040DF3CF9A
:10B91A0000F0F4CF01F0000E0026040E012200C050
:10B92A00DEFF01C0DDFF840EDECFE9FFDDCFEAFFD7
:10B93A00E850EF12E552E552E552E5CFDAFFE7CFDC
:10B94A00D9FF1200D9CFE6FFDACFE6FFE1CFD9FF60
:10B95A00E2CFDAFF65A84ED0FD0EEA6ADB34FE0BB1
:10B96A00EA36E96E8D0EE926020EEA22EE50EFCF94
:10B97A00EAFFE96E400EEE16EE6AEE6AEE6AFD0E18
:10B98A00EA6ADB34FE0BEA36E96E8D0EE926020E10
:10B99A00EA22EE50EFCFEAFFE96EEE7CFD0EEA6A8C
:10B9AA00DB34FE0BEA36E96E8D0EE926020EEA2238
:10B9BA00EF74400E006EFD0EEA6ADB34FE0BEA36C7
:10B9CA00E96E8D0EE926020EEA22EE50EFCFEAFF6B
:10B9DA00E96E0050EF16FD0EEA6ADB34FE0BEA361A
:10B9EA00E96E8D0EE926020EEA22EE50EFCFEAFF4B
:10B9FA00E96EEF7CE552E5CFDAFFE7CFD9FF120017
:10BA0A000201B0514DE1010EB06FB15149E1010E91
:10BA1A00B16F020E945D0DE18DC2E9FF8EC2EAFF9D
:10BA2A00EE52EF6A8DC2E9FF8EC2EAFFC80EEF6ED0
:10BA3A001200940535E1A76B83C2E9FF84C2EAFFCD
:10BA4A00EE52400EEF6E83C2E9FF84C2EAFF020E95
:10BA5A00E926000EEA22300EEE6E040EED6E83C267
:10BA6A00E9FF84C2EAFF840EEF6E010EA76F85C25A
:10BA7A00E9FF86C2EAFFEE52400EEF6E85C2E9FF89
:10BA8A0086C2EAFF020EE926000EEA22300EEE6EA8
:10BA9A00040EED6E85C2E9FF86C2EAFF800EEF6EE4
:10BAAA0012000201B26BB36B020E945D18E185C2FB
:10BABA00E9FF86C2EAFFEE52400EEF6E85C2E9FF49
:10BACA0086C2EAFF020EE926000EEA22380EEE6E60
:10BADA00040EED6E85C2E9FF86C2EAFF1DD09851B9
:10BAEA000401365D020199510401375904E236C452
:10BAFA0098F237C499F2CCD88DC2E9FF8EC2EAFF18
:10BB0A00020EE926000EEA22380EEE6E040EED6EE3
:10BB1A008DC2E9FF8EC2EAFFC80EEF6E1200D9CFBE
:10BB2A00E6FFDACFE6FFE1CFD9FFE2CFDAFFE6524E
:10BB3A00E652000EDE6E040EDD6EFC0EDB50E824CB
:10BB4A00026EFD0EDB50040DF3500224040DF4CFF7
:10BB5A0001F0D9CFE9FFDACFEAFFF350EE26015020
:10BB6A00ED22DECFE9FFDDCFEAFFEF9EFC0EDB50D0
:10BB7A000AE1FD0EEA6ADB34FE0BEA36E96E870E4D
:10BB8A00E926020E09D0FD0EEA6ADB34FE0BEA361C
:10BB9A00E96E8D0EE926020EEA22DECFEEFFDDCF38
:10BBAA00EDFFDECFE9FFDDCFEAFFEF9CDECFE9FF55
:10BBBA00DDCFEAFF040EE926000EEA22EF8CE552F9
:10BBCA00E552E552E5CFDAFFE7CFD9FF12006598D3
:10BBDA00020197BF2BD09CAF09D0020E946FB351CC
:10BBEA0001E15FDF0201B16BB06B120085C2E9FFB0
:10BBFA0086C2EAFFEE52400EEF6E85C2E9FF86C2A8
:10BC0A00EAFF020EE926000EEA22300EEE6E040E5C
:10BC1A00ED6E85C2E9FF86C2EAFF8C0EEF6E8DC219
:10BC2A00E9FF8EC2EAFF840EEF6E1200040130AF04
:10BC3A000DD00201010E946FB25101E132DF02010F
:10BC4A00B16BB06BAF5123E105EF5DF00201020E5B
:10BC5A00946F85C2E9FF86C2EAFFEE52400EEF6E8C
:10BC6A0085C2E9FF86C2EAFF020EE926000EEA2231
:10BC7A00300EEE6E040EED6E85C2E9FF86C2EAFF53
:10BC8A00840EEF6EB16BB06BAF5101E1B9DE1200F9
:10BC9A00D9CFE6FFDACFE6FFE1CFD9FFE2CFDAFF6D
:10BCAA00E652400EDF6E0201985D000E99590AE2D3
:10BCBA0098C2DFFF935102E1010E03D0930502E11E
:10BCCA00020E936FDF50016AE850985D986F015039
:10BCDA009959996F8DC2E9FF8EC2EAFFEE52DFCF02
:10BCEA00EFFF380EA16F040EA26F97B118D0DF5084
:10BCFA002DE095C2F6FF96C2F7FF952B000E96230C
:10BD0A000800F550E66EA1C2E9FFA2C2EAFFA12B24
:10BD1A00000EA223E552E750EF6EDF06E8D7DF50A8
:10BD2A0015E095C2E9FF96C2EAFF952B000E96230D
:10BD3A00EF50E66EA1C2E9FFA2C2EAFFA12B000EF4
:10BD4A00A223E552E750EF6EDF06E9D7E552E55246
:10BD5A00E5CFDAFFE7CFD9FF1200D9CFE6FFDACF76
:10BD6A00E6FFE1CFD9FFE2CFDAFFE652E65283C21D
:10BD7A00E9FF84C2EAFFEE52EFCFDFFFDFCF00F028
:10BD8A00005002019D5D000E9E5902E29DC2DFFF36
:10BD9A00DF50006E016AE8509D5D9D6F01509E590B
:10BDAA009E6F010EDB6ADF50F36E010EDBCFF4FFEC
:10BDBA00F350F45C16E2010EDB50EA6A380FE96EC2
:10BDCA00040EEA22EF50E66E9AC2E9FF9BC2EAFF2E
:10BDDA009A2B000E9B23E552E750EF6E010EDB2AE9
:10BDEA00E2D7000ED8809D55000E9E5527E285C2E7
:10BDFA00E9FF86C2EAFFEE52400EEF6E85C2E9FF06
:10BE0A0086C2EAFF020EE926000EEA22380EEE6E1C
:10BE1A00040EED6E83C2E9FF84C2EAFFEF50400BC5
:10BE2A0006E185C2E9FF86C2EAFFC80E05D085C2CF
:10BE3A00E9FF86C2EAFF880EEF6E28D085C2E9FFC5
:10BE4A0086C2EAFFEE52400EEF6E85C2E9FF86C255
:10BE5A00EAFF020EE926000EEA22300EEE6E040E0A
:10BE6A00ED6E85C2E9FF86C2EAFF840EEF6E9F512E
:10BE7A00A01107E005D0A0C2FAFF02019F51F96E96
:10BE8A00FADF02019C9FAF5101E1BADDE552E552AA
:10BE9A00E552E5CFDAFFE7CFD9FF1200D9CFE6FFA7
:10BEAA00DACFE6FFE1CFD9FFE2CFDAFFE6520201AD
:10BEBA00978F020EE66EE66AE66A270EE66E0F0EA8
:10BECA00E66ED2EC78F0006E050EE15C02E2E16A01
:10BEDA00E552E16E0050300EE66EE66AE66A000E42
:10BEEA00E66E040EE66ED2EC78F0006E050EE15CAA
:10BEFA0002E2E16AE552E16E0050658CDF6A030EE8
:10BF0A00DF5C10E2DF50EA6AA80FE96E020EEA224D
:10BF1A00EF6ADF50EA6AAB0FE96E020EEA22EF6AB5
:10BF2A00DF2AEDD7010EE66EE66AE66A820EE66E53
:10BF3A00020EE66ED2EC78F0006E050EE15C02E2CB
:10BF4A00E16AE552E16E0050659C0201080E8D6FB0
:10BF5A00040E8E6F000E836F040E846F83C285F207
:10BF6A00866F32C481F2815102E1100E16D0010EA1
:10BF7A00E66EE66A810EE66E020EE66E010EE66E69
:10BF8A00E66A7CEC76F0006E060EE15C02E2E16A9B
:10BF9A00E552E16E00500201200E806FE552E55233
:10BFAA00E5CFDAFFE7CFD9FF1200800E0401305D3A
:10BFBA0058E10201C00E976F04013351030A2FE0C2
:10BFCA00010A09E0030A4BE10201D60E956FF20E4F
:10BFDA00966F120E3ED03251F66EF76AD890F63648
:10BFEA00F7365D0EF626F30EF7220900F5CF95F225
:10BFFA000A00F5CF96F2020E0201F76A9525F66E4F
:10C00A009651F7220800F5CF98F2030EF76A9525A4
:10C01A00F66E9651F7220800F5CF99F21200030E38
:10C02A00325D1AE23251F66EF76AD890F636F73672
:10C03A005F0EF626F30EF7220900F5CF95F20A00F5
:10C04A00F5CF96F295C2F6FF96C2F7FF0800F550B3
:10C05A000201986F996B12000201976B120002019C
:10C06A00976B1200D9CFE6FFDACFE6FFE1CFD9FF0F
:10C07A00E2CFDAFFE652E6520401386B396B3051EF
:10C08A001F0B020A11E0030A0CE0010A3CE102015B
:10C09A00978F040138810201A30535E10401388331
:10C0AA0032D00201978F2FD00201978F040134BF3B
:10C0BA000BD034510F0BE96EEA6AD890E936EA36AA
:10C0CA00870EE926020E0AD034510F0BE96EEA6A8E
:10C0DA00D890E936EA368D0EE926020EEA22EECF2C
:10C0EA00DEFFEDCFDDFFDECFE9FFDDCFEAFFEF5068
:10C0FA00800B09E0DECFE9FFDDCFEAFFEF50040B4A
:10C10A0002E0010E386F020197AF07D0380E956F23
:10C11A00040E966F9781020E986FE552E552E5522A
:10C12A00E5CFDAFFE7CFD9FF12000F0126A115D01C
:10C13A0083C2E9FF84C2EAFFEF5080080DE18DC295
:10C14A00E9FF8EC2EAFFEF50840806E183C2E9FFE5
:10C15A0084C2EAFF8C0EEF6E2691629A12000F01DA
:10C16A003685629865820201010EA46F000EE66EA2
:10C17A00E66AE66EE66A750EE66EE66A7CEC76F0CC
:10C18A00006E060EE15C02E2E16AE552E16E0050E1
:10C19A0012000201A46B000EE66EE66AE66EE66A1B
:10C1AA00740EE66EE66A7CEC76F0006E060EE15CD2
:10C1BA0002E2E16AE552E16E005065920F0136959E
:10C1CA0062A402D06294FCD71200D9CFE6FFDACF7C
:10C1DA00E6FFE1CFD9FFE2CFDAFFE65202012D0EE8
:10C1EA00AE6FFD0EA51553E17E0EA515E8407F0B37
:10C1FA00040DF3CF83F2F4CF84F2000E8327040EEA
:10C20A00842383C285F284C286F2857583C2E9FFDC
:10C21A0084C2EAFFEF503C0BE842E8420D0835E1E0
:10C22A00DF6A080EDF5C23E283C2E9FF84C2EAFF09
:10C23A00020EE926000EEA22EE50EFCFEAFFE96E7F
:10C24A00EF50E66EDF50EA6A300FE96E040EEA221A
:10C25A00E552E750EF6E83C2E9FF84C2EAFF020E9D
:10C26A00E926000EEA22EE2AEF22DF2ADAD783C273
:10C27A00E9FF84C2EAFF020EE926000EEA22300E26
:10C28A00EE6E040EED6E0FD807D040D805D0FD0E25
:10C29A00A515040801E15FD8E552E552E5CFDAFFBA
:10C2AA00E7CFD9FF12000201936BAF6BB26BB36B8E
:10C2BA00A76B946B8DC2E9FF8EC2EAFFEF9E8D7564
:10C2CA008DC2E9FF8EC2EAFFEF9E8D7585C2E9FF36
:10C2DA0086C2EAFFEF9E976B986B996B9C6B9D6B7E
:10C2EA009E6B99D8000EE66EE66AE66EE66A030E63
:10C2FA00E66EE66A7CEC76F0006E060EE15C02E21F
:10C30A00E16AE552E16E0050ECEF5DF0020E0201C7
:10C31A00945D02E1B2EF5EF0946BA7511AE185C217
:10C32A00E9FF86C2EAFFEE52400EEF6E85C2E9FFD0
:10C33A0086C2EAFF020EE926000EEA22300EEE6EEF
:10C34A00040EED6E85C2E9FF86C2EAFF8C0EEF6E1F
:10C35A001200A76B1200D9CFE6FFDACFE6FFE1CFD2
:10C36A00D9FFE2CFDAFFE6528DC2E9FF8EC2EAFFB9
:10C37A00EF50400B01E0010EDF6E02018D75080ED1
:10C38A00805D0BE132C438FF0F01385103E002012E
:10C39A00100E02D00201040E806F940526E18DC2B0
:10C3AA00E9FF8EC2EAFF020EE926000EEA22380EE3
:10C3BA00EE6E040EED6E6CDC020E0201935D06E178
:10C3CA008DC2E9FF8EC2EAFF840E0DD0DF5006E16E
:10C3DA008DC2E9FF8EC2EAFFC80E05D08DC2E9FF01
:10C3EA008EC2EAFF880EEF6E0FD09CAF0CD09F5121
:10C3FA00A01107E005D0A0C2FAFF02019F51F96E11
:10C40A00FADF02019C9F946BE552E552E5CFDAFF11
:10C41A00E7CFD9FF120004013051600BE842E8422D
:10C42A00E842E842E842000901E0120031510C0AF0
:10C43A0054E00B0A3FE00C0A31E0010A22E00B0A41
:10C44A001EE0020A1CE0030A18E0080A10E0010ACA
:10C45A000CE00F0A08E0030A01E012000201978FBC
:10C46A00080E806F1200DAEF5FF053EF5FF00201FF
:10C47A00810E956F020E966F0CD037EF60F073EF56
:10C48A0062F034510201956F966B820E9527020E67
:10C49A0096239781010E986F978F12000201978F4A
:10C4AA0004013451EA6A820FE96E020EEA2232C4AA
:10C4BA00EFFF1200000EE66EE66AE66EE66A020E0C
:10C4CA00E66EE66A7CEC76F0006E060EE15C02E24D
:10C4DA00E16AE552E16E005012001200D9CFE6FF80
:10C4EA00DACFE6FFE1CFD9FFE2CFDAFFE652E65232
:10C4FA00E652E652E6520401320510E130511F0BB2
:10C50A0000090CE10201978F030E0401315D04E179
:10C51A000201010EA36F02D00201A36B0401325182
:10C52A0001E01AD130511F0B020801E015D1345134
:10C53A000F0B000901E110D134510F0B020801E27F
:10C54A000BD1200E0201805D01E006D1978F040114
:10C55A0034BF16D034510F0BE96EEA6AD890E93627
:10C56A00EA36870EE926020EEA22EECFDEFFEDCF8B
:10C57A00DDFF34510F0BEA6AAB0FE96E020E15D0DC
:10C58A0034510F0BE96EEA6AD890E936EA368D0E15
:10C59A00E926020EEA22EECFDEFFEDCFDDFF3451AF
:10C5AA000F0BEA6AA80FE96E020EEA22020EEFCF1B
:10C5BA00DBFFD950020FE96E000EDA20EA6EEF5067
:10C5CA00010B02E1DF9401D0DF8434BF0BD0345178
:10C5DA000F0BE96EEA6AD890E936EA36870EE92641
:10C5EA00020E0AD034510F0BE96EEA6AD890E93686
:10C5FA00EA368D0EE926020EEA22DECFEEFFDDCF05
:10C60A00EDFF030E315D20E1DECFE9FFDDCFEAFF6A
:10C61A00EF50800B11E034BF07D034510F0BEA6A98
:10C62A00AB0FE96E020E06D034510F0BEA6AA80F5F
:10C63A00E96E020EEA22EF82840EDECFE9FFDDCF39
:10C64A00EAFFE850EF1288D0DF74DECFE9FFDDCFD2
:10C65A00EAFFEF50800B1FE0DECFE9FFDDCFEAFFF4
:10C66A00EF9EDECFE9FFDDCFEAFFEF8C020EE66E2A
:10C67A00E66ADECFE6FFDDCFE6FF050EE66EE66A86
:10C68A007CEC76F0006E060EE15C02E2E16AE552AD
:10C69A00E16E005005D0DECFE9FFDDCFEAFFEF8C77
:10C6AA00DF74D950020FE96E000EDA20EA6EEF50FD
:10C6BA00020B07E1DECFE9FFDDCFEAFFEF50800B87
:10C6CA002FE0040134BF07D034510F0BEA6AAB0FD5
:10C6DA00E96E020E06D034510F0BEA6AA80FE96E12
:10C6EA00020EEA22EF923B0E006EDECFE9FFDDCFAB
:10C6FA00EAFFE850EF16020EE66EE66ADECFE6FFC4
:10C70A00DDCFE6FF050EE66EE66A7CEC76F0006E9B
:10C71A00060EE15C02E2E16AE552E16E005007D0E2
:10C72A003B0EDECFE9FFDDCFEAFFE850EF1604014A
:10C73A0034510F0B016A260F006E0F0E0122030EF1
:10C74A0000C0DBFF040E01C0DBFF030EDBCFE9FFF5
:10C75A00040EDBCFEAFFEF90050EE15C02E2E16A2C
:10C76A00E552E16EE552E5CFDAFFE7CFD9FF1200D5
:10C77A00F9EC68F0FB0EDBCFF3FFDB06F3500009A0
:10C78A000AE047EC69F0FA0EB2EC69F0F3E1011C39
:10C79A00F1E1010E01D0000E28EF69F0F9EC68F022
:10C7AA003B0EE12402E3E168E652E16E010EDB6A28
:10C7BA00020EDB6AF90EDBCFF6FFFA0EDBCFF7FFCC
:10C7CA00FB0EDBCFF8FF0800F550DF6EDF5002E109
:10C7DA004CEF68F0250EDF5C02E03FEF68F0030ED5
:10C7EA00DB6A040EDB6A050EDB6A060EDB6A070EDD
:10C7FA00DB6A61EC68F02D0EDF5C0CE02B0EDF5C6F
:10C80A0009E0200EDF5C06E0230EDF5C03E0300E59
:10C81A00DF5C1AE1DF50300A14E0130A0FE0030A62
:10C82A000AE00B0A05E0060AE4E1030EDB80E1D721
:10C83A00030EDB82DED7030EDB84DBD7030EDB8637
:10C84A00D8D7030EDB88D5D72A0EDF5C1BE15DEC57
:10C85A0068F0ABEC68F010E0030EDB803A683B68E6
:10C86A00130EDBCF3FF0140EDBCF40F096EC6CF0EA
:10C87A00040E38C0DBFF03D0130E94EC68F061ECB1
:10C88A0068F00BD0090EDB6A02EC69F003E076EC83
:10C89A0069F0FAD7090E94EC68F0030EDBB0DB9866
:10C8AA002E0EDF5C1BE161EC68F02A0EDF5C0BE107
:10C8BA005DEC68F0ABEC68F003E1130EE6EC68F0AF
:10C8CA0061EC68F00BD0090EDB6A02EC69F003E058
:10C8DA0076EC69F0FAD7090EE6EC68F0680EDF5CD0
:10C8EA0007E161EC68F0680EDF5C1DE1030E18D009
:10C8FA00740EDF5C17E07A0EDF5C14E0480EDF5C32
:10C90A0006E0540EDF5C03E05A0EDF5C02E1020E21
:10C91A0007D06C0EDF5C03E06A0EDF5C04E1010EF7
:10C92A0039EC69F0C9DBDF506E0A01E17FD31E0AD8
:10C93A0001E192D1200A01E18FD13F0A01E149D1F7
:10C94A001A0A01E146D10D0A01E143D1200A01E1A7
:10C95A0040D13A0A01E13DD1200A01E13AD1260A41
:10C96A0001E135D10D0A01E132D11A0A01E1D9D02A
:10C97A00200A4AE0300A1FE0460A0EE0250A01E0D2
:10C98A0083D3D950F90FE96EFF0EDA20EA6E010E51
:10C99A00EE5E000EEE5AEE5A47EC69F0250EE66E90
:10C9AA0095DB03E1011C01E169D343EC69F001E283
:10C9BA006BD3DB2A69D3080EDB6A040EDB5001084D
:10C9CA0006E2040EDB040BEC69F0DB508BDB080E8D
:10C9DA00DB5009E0030EDB50010B05E172DB01E0DD
:10C9EA004DD3080EDB6A64DBEFCFDFFFBBEC69F0E7
:10C9FA0003E1011C01E142D343EC69F001E3DB2AC4
:10CA0A0060DB01E141D33AD3070EDB5002080FE1A4
:10CA1A0087EC69F0030E4EEC69F00E0EEECFDBFFE9
:10CA2A000F0EEECFDBFF100EEECFDBFF20D0F70E9E
:10CA3A00DBCF03F0F80EDBCF04F0020E035E000E2C
:10CA4A00045AF70E03C0DBFFF80E04C0DBFF03C075
:10CA5A00E9FF04C0EAFF3EEC69F0026A0E0E00C06C
:10CA6A00DBFF0F0E01C0DBFF100E02C0DBFF0E0E54
:10CA7A00DBCFE6FF0F0EDBCFE6FF100EDBCFE6FFC4
:10CA8A00FAEC78F0E552E552E552130E39C0DBFFB5
:10CA9A00140E3AC0DBFF060EDB5005E0130E82ECE3
:10CAAA0069F001E26ADBA6EC69F002E2130E37DBF9
:10CABA0069EC69F006E0040E82EC69F002E2050E08
:10CACA002EDB030EDBB005D0FCDA01E0D7D2080E6C
:10CADA00DB6A090EDB6A0E0EDBCFF6FF0F0EDBCF29
:10CAEA00F7FF100EDBCFF8FF0800F550DF6EDF50BE
:10CAFA0014E0ACEC69F011E2BBEC69F003E1011C53
:10CB0A0001E1BCD2BBDB01E3DB2A090EDB2AD950E7
:10CB1A000E0FE96E000ECBDBE7D7D3DA01E1B4D210
:10CB2A00ADD2C6DA110EEECFDBFF120EEDCFDBFF70
:10CB3A00110EDBCFE6FF120EDBCFE6FFECEC78F04E
:10CB4A00E552E552130EF3CFDBFF140EF4CFDBFFF1
:10CB5A00060EDB5004E0130ED0DB01E20EDBA6EC7E
:10CB6A0069F002E2130EDBDAAFDB05E0040EC5DB87
:10CB7A0002E2050ED4DA030EDBB005D0A2DA01E038
:10CB8A007DD2080EDB6A090EDB6A110EDBCFE9FFE4
:10CB9A00120EDBCFEAFFEFCFDFFFDF5014E0D7DB67
:10CBAA0012E2E4DB03E1011C01E168D267DB01E385
:10CBBA00DB2A090EDB2A110EDB2ADBCFE9FF120E74
:10CBCA00E8E3DB2AE6D77DDA01E15ED257D2030E2B
:10CBDA00DB8E070EDB0410E195DB040E5ADB0A0E2E
:10CBEA00EECFDBFF0B0EEECFDBFF0C0EEECFDBFF43
:10CBFA000D0EEECFDBFF6CD0070EDB5003082CE1E5
:10CC0A00030EDBAE0DD0B2DA020E76DAEFCF00F009
:10CC1A00016A026A036A00AE39D00168026835D037
:10CC2A00F70EDBCF01F0F80EDBCF02F0020E015E49
:10CC3A00000E025AF70E01C0DBFFF80E02C0DBFF3E
:10CC4A0001C0E9FF02C0EAFFEFCF00F00A0E00C000
:10CC5A00DBFF0B0EDB6A38D0070EDB50020809E156
:10CC6A00030EDBAE04D059DB02AE10D00ED055DB7A
:10CC7A000DD0030EDBAE12D079DA020E3DDAF9DA04
:10CC8A00026A036A01AE02D002680368E2DA0C0E95
:10CC9A0002C0DBFF0D0E03C0DBFF1AD0F70EDBCF9D
:10CCAA0002F0F80EDBCF03F0020E025E000E035A0A
:10CCBA00F70E02C0DBFFF80E03C0DBFF02C0E9FF7C
:10CCCA0003C0EAFFD6DAC5DA0C0EDB6A0D0EDB6AA0
:10CCDA00060EDB5005E1010EF36E050EF3CFDBFF06
:10CCEA00150EDB6A160EDB6AD950370F006E000E7E
:10CCFA00DA20016E390E00C0DBFF3A0E01C0DBFFFD
:10CD0A00380EDB6A080EDB6A0A0EAEDADF50780AE2
:10CD1A0012E0200A10E0280A0CE0200A0AE03F0A82
:10CD2A0006E00D0A02E0200A08E1020E05D0080E0C
:10CD3A0003D0080EDF26100E97DA030EDBBE02D0F0
:10CD4A00DB92DB94DB50800B24E08ADAD890030E66
:10CD5A00EB50000A08E6000EEE5C000EEE58000EDC
:10CD6A00EE58000EEE5815E213DA3D683E683F6849
:10CD7A004068F5EC79F00A0E34C0DBFF0B0E35C0C3
:10CD8A00DBFF0C0E36C0DBFF0D0E37C0DBFF2D0EAE
:10CD9A0008D0030EDBA202D02B0E03D0DBA408D0EE
:10CDAA00200EF36E170EF3CFDBFF150EDB2A02D02F
:10CDBA00170EDB6A050EDB5003E1B7D901E189D012
:10CDCA00BE0E006EF50E016E000E026E070EDBCF70
:10CDDA0003F0046A056A066A03C03DF004C03EF027
:10CDEA0005C03FF006C040F0D3D953EC7AF00050AA
:10CDFA003424F36E01503520F46E02503620F86E5A
:10CE0A00F4CFF7FFF3CFF6FF0800090EF5CFDBFFEB
:10CE1A00580EDF5C0FE1610EF36E090E7BD90AE34F
:10CE2A00200E006E090EDBCFE7FF0050E75E090E09
:10CE3A00E7CFDBFF070EDBCF00F0016A026A036A65
:10CE4A000FDA00C03DF001C03EF002C03FF003C05F
:10CE5A0040F0EECF38F0EECF39F0EECF3AF0EFCF28
:10CE6A003BF053EC7AF03BC0EDFF3AC0EDFF39C01E
:10CE7A00EDFF38C0EFFF390EDBCFE9FFDB063A0ED4
:10CE8A00DBCFEAFF01E2DB06090EDBCFEFFF150E6F
:10CE9A00DB2A4BD995E1030EDBA61DD06F0EDF5CB2
:10CEAA0006E1C1D918E3150EDB285BDA14D0780E37
:10CEBA00DF5C09E0580EDF5C06E0620EDF5C03E02F
:10CECA00420EDF5C08E1020EF36E160EF3CFDBFFB3
:10CEDA0002D0150EDB6A030EDB50100B0EE0040EB7
:10CEEA00DBCF00F0050EDB50D880005406E2060EB8
:10CEFA00DB5003E1040EDB5034DA95D90AE2050E61
:10CF0A00DBCFE7FF150EDB50E75E050EE7CFDBFF51
:10CF1A0002D0050EDB6A040EDBCF00F0160E45D9EF
:10CF2A00D880005414E2160EDBCFE6FF150EDBCFD5
:10CF3A00E6FF040EDBCFE6FF050EDB50E552E75CA9
:10CF4A00E552D880E754E552D880E7545FD9030EFA
:10CF5A00DB50010B0BE1080EDB5008E0B2D801E010
:10CF6A008DD0080EDB50BED8080EDB6A170EDB50D8
:10CF7A0007E088D9170EF1D903E1011C01E17ED03F
:10CF8A00160EDB5016E07ED9300EE66E9FD802E10F
:10CF9A00011C74E077D9DFCFE6FFB3EC79F0E552F4
:10CFAA00E552E552F4CF01F00001F31C02E1011C45
:10CFBA0065E0050EDBCF00F0160EDB50D88000547A
:10CFCA0009E2050EDBCFE7FF160EDB50E75E050E22
:10CFDA00E7CFDBFF300EE66E050ECBD94FE1390EF7
:10CFEA00DB2ADBCFE9FF3A0E01E3DB2ADBCFEAFFDC
:10CFFA00090EEFCFDBFFDB500EE044D9090EADD9A5
:10D00A0002E1011C3BE0390EDB2ADBCFE9FF3A0ED5
:10D01A00EDE3DB2AEBD755D831E1160EDBCFE6FF7D
:10D02A00080EC3D8E552E7245DD82ED0070EDB5090
:10D03A00030A1CE0010A14E0030A07E07BD9DBCFEC
:10D04A00EEFF020EDBCFEDFF1FD0F5D8056A03AE67
:10D05A0002D0046805682CD8BCD805C0EEFF14D0ED
:10D06A00EAD803BE046824D8B4D80ED063D9DBCF7B
:10D07A00EFFF0AD07BD905E1011C03E1F368F468EC
:10D08A0010D0FCD801E3DB2A79D9E8EF63F0010E6E
:10D09A00DBCF00F0020EDBCF01F000C0F3FF01C0CE
:10D0AA00F4FF3B0EE15C02E2E16AE552E16ECBD0AD
:10D0BA0029D9020E4EEF69F061D90800F550DF6EEA
:10D0CA001200200EE66E080EBEEF69F0B3EC79F09E
:10D0DA00E552E552E552F3CF00F0F4CF01F000013A
:10D0EA00F31C1200006E016AD950010F4DD900508D
:10D0FA00EE260150ED221200045E000E055AF70ECC
:10D10A0004C0DBFFF80E05C0DBFF04C0E9FF05C061
:10D11A00EAFF1200DBCFF4FFF350F45C1200DB509D
:10D12A00E76E040EE7CFDBFF12000A0EDBCF00F03A
:10D13A000B0EDBCF01F00C0EDBCF02F00D0EDBCFB6
:10D14A0003F000500110021003101200130EEECF6C
:10D15A00DBFF140EEDCFDBFF130EDBCF00F0140E56
:10D16A00DBCF01F00001800E01141200F70EDBCFB5
:10D17A0004F0F80EDBCF05F01200050EDB50E66E68
:10D18A00D950130F01D9E552E750EE6EED6A12003D
:10D19A000A0EDBCF38F00B0EDBCF39F00C0EDBCFEB
:10D1AA003AF00D0EDBCF3BF01200DBCFE6FF150E97
:10D1BA00DBCFE6FF050EDB50E552E724E552E72414
:10D1CA001200DB50CED8010EF36E060EF3CFDBFF52
:10D1DA001200EE50EFCFEAFFE96E02C0EEFF03C085
:10D1EA00EEFF04C0EEFF1200D9CFE6FFDACFE6FF6A
:10D1FA00E1CFD9FFE2CFDAFF1200DFCFE6FFE66A1E
:10D20A0041EC7AF0E552E552F3501200E76E080E4F
:10D21A00E7CFDBFF1200EECF00F0EECF01F0EFCF49
:10D22A0002F0036A1200050EDBCF00F0150EDB5088
:10D23A00D88000541200010EDBCF02F0020EDBCFC1
:10D24A0003F0046A1200E552E5CFDAFFE7CFD9FF0F
:10D25A0012000A0E00C0DBFF0B0E01C0DBFF12003A
:10D26A00D9500A0FC9EF69F0F36E070EF3CFDBFF4F
:10D27A001200EECF00F0EFCF01F01200010EDB2A10
:10D28A00020E1200FC0EDBCFE6FFFD0EDBCFE6FF3F
:10D29A001200005E000E015AF70E00C0DBFFF80E06
:10D2AA0001C0DBFF00C0E9FF01C0EAFF1200DA207B
:10D2BA00EA6EEF2AEECFF6FF000EEF22EECFF7FF6F
:10D2CA00EF22EECFF8FF1200040EDBCFE6FF130EBB
:10D2DA00DB50E552E75C9ADFDB5004DF060EDB50D9
:10D2EA001200090EDB500A0DF350DF24D00FE76E4F
:10D2FA00090EE7CFDBFF61EF68F0DB50F36E050E36
:10D30A008FEF68F0F70EDBCF00F0F80EDBCF01F0FD
:10D31A001200DFCFE6FF6BEF68F028DF030EECDECA
:10D32A0010EF69F0BDEC63F0E552E552E552E552C3
:10D33A0000091200BDDEEE50EFCFEAFFE96E010EE2
:10D34A001200130EDB50F36E040E8FEF68F0040E1A
:10D35A00DB50F36E090E8FEF68F0DBCFE6FF6BEF61
:10D36A0068F0E76E050EE7CFDBFF12008BDF8EEF6A
:10D37A0069F0DBCFE6FF86DF97EF69F0D950F90F46
:10D38A00E96EFF0E5CEF69F0E96E000EDA20EA6ED4
:10D39A001200439E08D0439E3BAE05D03A6C3B1E1A
:10D3AA00E86A3B22438E3BC035F03AC034F0476A04
:10D3BA00466A8E0E366E376AA8EF6BF0439E0CD023
:10D3CA00439E3BAE09D0386C391E3A1E3B1EE86AB2
:10D3DA0039223A223B22438E3BC035F03AC034F020
:10D3EA0039C047F038C046F09E0E366E376AA8EF4D
:10D3FA006BF0436AE4EC6BF0FCEC6BF043B68CEF39
:10D40A006BF043A205D043BA8CEF6BF093EF6BF04D
:10D41A0043BA9FEF6BF043A005D043B88CEF6BF093
:10D42A009FEF6BF043B893EF6BF0376A7F0E3C24A3
:10D43A00366EE86A37224150365EE86A375A1A0E63
:10D44A00446E3C6A466A476A346A356A3E50395EB7
:10D45A003F503A5A40503B5A000E3C5A09E73E5058
:10D46A0039263F503A2240503B22000E3C2201D03E
:10D47A00468AD89039363A363B363C36D8904636C4
:10D48A00473634363536442EE1D73B503A103910F8
:10D49A00D8A4468AA8EF6BF0436AE4EC6BF0FCEC84
:10D4AA006BF043B68CEF6BF043A205D043B88CEF18
:10D4BA006BF093EF6BF043AA05D043B08CEF6BF09F
:10D4CA0093EF6BF043B002D043A802D09FEF6BF00A
:10D4DA00376A41503C24366EE86A37227E0E365E41
:10D4EA00E86A375A466A476A346A356A40503B02E4
:10D4FA00F4CF35F0F3CF34F03F503B02F3504726D8
:10D50A00F4503422000E352240503A02F350472696
:10D51A00F4503422000E35223E503B02F350462688
:10D52A00F4504722000E342235223F503A02F3507B
:10D53A004626F4504722000E342235224050390242
:10D54A00F3504626F4504722000E342235223E502C
:10D55A003A02F4504626000E4722342235223F5022
:10D56A003902F4504626000E472234223522A8EF0B
:10D57A006BF0417E436AE4EC6BF0FCEC6BF043B673
:10D58A008CEF6BF043A20AD043AA03D043BE8CEFC0
:10D59A006BF043A498EF6BF095EF6BF043AA05D0BC
:10D5AA0043AC98EF6BF095EF6BF043A00AD043A819
:10D5BA0008D043BE04D043A402D0A1EF6BF0A5EF7C
:10D5CA006BF0466A376A41503C5C456E10E339C0DD
:10D5DA0047F03AC034F03BC035F03CC044F03EC09E
:10D5EA0039F03FC03AF040C03BF0433A09D03EC060
:10D5FA0047F03FC034F040C035F041C044F0456CBC
:10D60A00439E43BC438E44C036F043B0D4EF6BF024
:10D61A001A0E4560D4EF6BF0366A3C6A43A408D010
:10D62A00396C3A1E3B1E3C1EE86A3A223B223C22D7
:10D63A0043AC08D0476C341E351E361EE86A3422C5
:10D64A0035223622386A455207E03C343B323A32B8
:10D65A0039323832452EF9D7395047263A503422D2
:10D66A003B5035223C50362238C046F0439E36AEF7
:10D67A000BD0466C471E341E351E361EE86A4722FA
:10D68A00342235223622438E36A006D0D88035324F
:10D69A00343247324632442A44C036F0A8EF6BF09F
:10D6AA00436AE4EC6BF043B65FEF6BF043A20FD032
:10D6BA0043B407D07F0E3B6EFF0E3A6E396E386E5A
:10D6CA0025D0800E3B6E01D03B6A000EF6D743B0E0
:10D6DA00FBD7386A9F0E3C60EBD77E0E3C64F4D7CA
:10D6EA009E0E3C5C07E0D8903B323A3239323832EF
:10D6FA003C2AF6D743A40AD0386C391E3A1E3B1E80
:10D70A00E86A39223A223B223BAEDED712007F0E6C
:10D71A003C6EFF0E3B6E3A6E396E12007F0E43BEB0
:10D72A00FF0E3C6E02D07F0E3C6E800E3B6E3A6A54
:10D73A00396AF3D743AE04D0800E3C6E3B6AF7D702
:10D74A003C6A3B6AF4D73550341047104610F8E06B
:10D75A0037BEF0D735BE0CD036503710EBE0D89034
:10D76A0046364736343635363606D8A03706F2D727
:10D77A003750D4E13628D2E046AE11D07F0E461497
:10D78A0002E147A00CD0472AE86A3422352207E38F
:10D79A00D880353234324732362A3628BFE03650FE
:10D7AA00C9E047C039F034C03AF035343B6E363000
:10D7BA003C6E3B323C9E43BE3C8E92EF6BF03B3656
:10D7CA003C3602E34384437E06E143803C6A3B6A7B
:10D7DA003A6A396A12003C2803E0D8803B321200C8
:10D7EA00D8903B3202E1438212004386120040364F
:10D7FA00413602E3438C437E06E14388416A406A2C
:10D80A003F6A3E6A1200412803E0D8804032120083
:10D81A00D8904032EAE1438A1200426A40AE1BEFD6
:10D82A006CF03F6C401EE86A4022421E3BAE23EF7A
:10D83A006CF03A6C3B1EE86A3B22421E92EC7AF08C
:10D84A003BBE33EF6CF042AE000C3A6C3B1EE86A0A
:10D85A003B22366C371EE86A3722000C42BE2AEF9A
:10D86A006CF04388FF0C41EC6CF043B6000C43B0FB
:10D87A00000C43A4000C010C436AE4EC6BF0FCECD2
:10D88A006BF043B6120043AE08D043A004D043A8BD
:10D89A0002D0438012004390120041503C5C0BE1DD
:10D8AA0040503B5C08E13F503A5C05E13E50395C30
:10D8BA0002E143801200D8A002D0438E10D03C501F
:10D8CA0041C03CF0416E3B5040C03BF0406E3A5084
:10D8DA003FC03AF03F6E39503EC039F03E6E41507B
:10D8EA003C5C10E0FF0F09E0439043B403D043AE21
:10D8FA004384120043AE43941200412AD890403226
:10D90A003F323E323E50395E3F503A5A40503B5ABF
:10D91A003BBEEAD7D89039363A363B363C2EF8D752
:10D92A00C8D73BC047F03AC046F03A503F02F4CF5E
:10D93A0039F0F3CF38F03B504002F4CF3BF0F3CF4D
:10D94A003AF03F02F3503926F4503A22E86A3B2271
:10D95A0046504002F3503926F4503A22E86A3B22F4
:10D96A0040AEBCEF6CF046503A5E47503B5A47AE69
:10D97A00000C3F503A5E40503B5A000C256C692C13
:10D98A00256C690A0D00514D2C25692C25692C2519
:10D99A00692C25690A0D00253034692C2530346933
:10D9AA000D0A002531690D0A00253033690D0A0078
:10D9BA00253031306C750D0A0025640A0D00256486
:10D9CA002C256C752C256C752C256C752C256C7585
:10D9DA000A0D004D616A6F72206D616C66756E6327
:10D9EA0074696F6E2041786973322053746570438D
:10D9FA006F756E746572207A65726F0A0D004D61DB
:10DA0A006A6F72206D616C66756E6374696F6E20E1
:10DA1A0041786973322053746570436F756E74650B
:10DA2A007220746F6F2068696768203A20256C75C8
:10DA3A000A0D004D616A6F72206D616C66756E63C6
:10DA4A0074696F6E2041786973312053746570432D
:10DA5A006F756E746572207A65726F0A0D004D617A
:10DA6A006A6F72206D616C66756E6374696F6E2081
:10DA7A0041786973312053746570436F756E7465AC
:10DA8A007220746F6F2068696768203A20256C7568
:10DA9A000A0D002130204572723A203C6178697380
:10DAAA00323E20737465702072617465203C2031A7
:10DABA002E3331487A2E0A0D002130204572723AEF
:10DACA00203C61786973323E2073746570207261FC
:10DADA007465203E2032354B2073746570732F7342
:10DAEA0065636F6E642E0A0D002130204572723A0A
:10DAFA00203C61786973313E2073746570207261CD
:10DB0A007465203C20312E3331487A2E0A0D0021CB
:10DB1A0030204572723A203C61786973313E207335
:10DB2A007465702072617465203E2032354B207313
:10DB3A00746570732F7365636F6E642E0A0D00210E
:10DB4A0030204572723A203C6D6F76655F6475725B
:10DB5A006174696F6E3E206C6172676572207468C9
:10DB6A00616E203136373737323135206D732E0AE0
:10DB7A000D002130204572723A203C617869733277
:10DB8A003E20616363656C65726174696F6E2076AD
:10DB9A00616C756520697320302E0A0D00213020D2
:10DBAA004572723A203C61786973313E2061636341
:10DBBA00656C65726174696F6E2076616C7565203B
:10DBCA00697320302E0A0D002130204572723A20E6
:10DBDA003C61786973323E206C61726765722074A9
:10DBEA0068616E20313637373732313520737465C4
:10DBFA0070732E0A0D002130204572723A203C6162
:10DC0A00786973313E206C6172676572207468614D
:10DC1A006E20313637373732313520737465707379
:10DC2A002E0A0D002130204572723A203C76656C2E
:10DC3A006F636974795F66696E616C3E206C6573A7
:10DC4A0073207468616E20342E0A0D00213020453D
:10DC5A0072723A203C76656C6F636974795F696E9B
:10DC6A00697469616C3E206C657373207468616EB7
:10DC7A0020342E0A0D002130204572723A203C765B
:10DC8A00656C6F636974795F66696E616C3E206C5E
:10DC9A006172676572207468616E20323530303087
:10DCAA002E0A0D002130204572723A203C76656CAE
:10DCBA006F636974795F696E697469616C3E206C1F
:10DCCA006172676572207468616E20323530303057
:10DCDA002E0A0D005374617475733D25690D0A008F
:10DCEA002135204572723A204E65656420636F6D56
:10DCFA006D61206E6578742C20666F756E643A20AB
:10DD0A00272563270D0A00506172616D383D25632E
:10DD1A000D0A00506172616D373D25630D0A00508E
:10DD2A006172616D363D256C750D0A005061726134
:10DD3A006D353D256C640D0A00506172616D343D8C
:10DD4A0025750D0A00506172616D333D25640D0A17
:10DD5A0000506172616D323D25640D0A0050617296
:10DD6A00616D313D25640D0A0050492C2531750D30
:10DD7A000A004D522C253033750D0A002C253032FD
:10DD8A00753A25303475004100492C253033692C09
:10DD9A00253033692C253033692C253033692C25FD
:10DDAA003033690D0A002138204572723A20556EC7
:10DDBA006B6E6F776E20636F6D6D616E64202725C1
:10DDCA006325633A253258253258270D0A0021382F
:10DDDA00204572723A20556E6B6E6F776E20636FB4
:10DDEA006D6D616E64202725633A253258270D0A26
:10DDFA00002137204572723A20457874726120708A
:10DE0A0061726D617465720D0A0021362045727265
:10DE1A003A20496E76616C696420706172616D7432
:10DE2A0065722076616C75650D0A00213420457291
:10DE3A00723A204D697373696E6720706172616D01
:10DE4A00657465722873290D0A00213320457272A0
:10DE5A003A20525820427566666572206F7665725E
:10DE6A0072756E0D0A002132204572723A2054589A
:10DE7A0020427566666572206F76657272756E0DE0
:10DE8A000A002131204572723A2043616E277420BC
:10DE9A0073746570207468617420666173740D0A06
:10DEAA00002130200D0A002008002573001B5B4268
:09DEBA001B5B314B1B5B30470080
:10DEC400040130511F0B010801E012003051600BB6
:10DED400E842E842E842E842E842010801E0120070
:10DEE400345103E0340501E012003151220A31E0DB
:10DEF400030A24E0010A15E0210A0DE0010A01E009
:10DF040012000201A00E956F070E966F080E986F0F
:10DF1400996B978121D00201A00E956F070E966F21
:10DF24001BD036C49DF237C49EF20201800E9A6F54
:10DF3400070E9B6F9F6BA06B9C8F12000201800EDB
:10DF4400956F070E966F070E986F996BC10E976FBA
:10DF5400120032C49BF70201978F12000701806BF5
:10DF64004B0E816F826B836B846B856B080E866F9F
:10DF74008F6B1A0EE66E010EE66E83EC5BF0E552D3
:10DF8400E5521E0EE66E020EE66E83EC5BF0E55281
:10DF9400E552400EE66E400EE66E070EE66EE66A49
:10DFA400020EE66EBCEC5BF0006E050EE15C02E274
:10DFB400E16AE552E16E0050F3CF97F7F4CF98F79A
:10DFC4000701996B9A6B906B1200D9CFE6FFDACFF9
:10DFD400E6FFE1CFD9FFE2CFDAFFFC0EDBCF3AF068
:10DFE400FD0EDBCF3BF0050E3A1801E13B5002E099
:10DFF400000E34D0FA0EDBCF00F0FB0EDBCF01F0C5
:10E004000701975100181AE19851011817E1400EC1
:10E01400E66E400EE66E070EE66EE66A020EE66EE9
:10E02400BCEC5BF0006E050EE15C02E2E16AE552D5
:10E03400E16E0050F3CF97F7F4CF98F7FA0EDBCFE9
:10E0440000F0FB0EDBCF01F007019951001805E148
:10E054009A51011802E1906B956B010EE552E5CFE0
:10E06400DAFFE7CFD9FF1200D9CFE6FFDACFE6FF18
:10E07400E1CFD9FFE2CFDAFF07018F6B97519811F7
:10E0840002E1000E08D097C7E9FF98C7EAFFEF50F6
:10E09400800B01E0010E000949E1FB0EDBCF00F02B
:10E0A40097C7E9FF98C7EAFFEE52EF50D8800054B3
:10E0B40008E297C7E9FF98C7EAFFEE52FB0EEFCFDD
:10E0C400DBFF8F6BFB0EDB508F5D19E28F51EA6A29
:10E0D400400FE96E070EEA22EF50E66E8F51E76EAD
:10E0E400FC0EDBCFE9FFFD0EDBCFEAFFE750E926AC
:10E0F400000EEA22E552E750EF6E8F2BE3D7400E75
:10E10400E66E400EE66E070EE66EE66A020EE66EF8
:10E11400BCEC5BF0006E050EE15C02E2E16AE552E4
:10E12400E16E0050F3CF97F7F4CF98F707018F51C2
:10E13400E552E5CFDAFFE7CFD9FF1200D9CFE6FFEA
:10E14400DACFE6FFE1CFD9FFE2CFDAFF0701905142
:10E154000CE1FC0EDBCF91F7FD0EDBCF92F7FB0E4B
:10E16400DBCF95F7010E966F906FE552E5CFDAFF9E
:10E17400E7CFD9FF1200D9CFE6FFDACFE6FFE1CF30
:10E18400D9FFE2CFDAFFE652E652E6520701905198
:10E194002DE1DF6AFC0EDBCF3AF0FD0EDBCF3BF066
:10E1A400DE523AC0DEFF3BC0DDFFDD52DF2ADF5026
:10E1B400006E016AFF0E001802E101500BE0010E2F
:10E1C400DBCFE9FFDB2A020EDBCFEAFF01E3DB2A28
:10E1D400EF50ECE1FC0EDBCF91F7FD0EDBCF92F7B5
:10E1E400DFCF95F70701010E966F906FE552E55268
:10E1F400E552E552E5CFDAFFE7CFD9FF1200D9CFD8
:10E20400E6FFDACFE6FFE1CFD9FFE2CFDAFFE6524D
:10E21400E652E652070190512EE1DF6AFC0EDBCF95
:10E224003AF0FD0EDBCF3BF0DE523AC0DEFF3BC0DE
:10E23400DDFFDD52DF2ADF50006E016AFF0E001899
:10E2440002E101500CE0010EDBCFF6FFDB2A020EE7
:10E25400DBCFF7FF01E3DB2A0800F550EBE1FC0E0E
:10E26400DBCF91F7FD0EDBCF92F7DFCF95F70701F8
:10E27400966B010E906FE552E552E552E552E5CFFB
:10E28400DAFFE7CFD9FF1200D9CFE6FFDACFE6FFF6
:10E29400E1CFD9FFE2CFDAFFE652E6520701995106
:10E2A4009A1102E1000E08D099C7E9FF9AC7EAFF64
:10E2B400EF50800B01E0010E000901E08CD0030E49
:10E2C400905D01E1906B905101E185D0020E905D6B
:10E2D4001AE1E66A000EE66EE66A010EE66E020ECA
:10E2E400E66EBCEC5BF0006E050EE15C02E2E16AF6
:10E2F400E552E16E0050F3CF99F7F4CF9AF7070196
:10E30400030E906F68D0900566E1400E006E016ABE
:10E314009551005C000E015803E2400EDF6E02D0FE
:10E3240095C7DFFFDF50955D956F000E936F070E65
:10E33400946F010EDFCFDBFF965116E1010EDB5027
:10E3440028E091C7F6FF92C7F7FF0800F55093C77E
:10E35400E9FF94C7EAFFEF6E932B000E9423912BF1
:10E364009223010EDB06EAD7010EDB5012E091C7BF
:10E37400E9FF92C7EAFFEF5093C7E9FF94C7EAFFAA
:10E38400EF6E932B000E9423912B9223010EDB0648
:10E39400EBD70701955107E1400EDF5C02E1020E65
:10E3A40001D0030E906FDFCFE6FF000EE66E070E7E
:10E3B400E66E010EE66E020EE66EBCEC5BF0006EDD
:10E3C400050EE15C02E2E16AE552E16E0050F3CF32
:10E3D40099F7F4CF9AF7E552E552E552E5CFDAFF23
:10E3E400E7CFD9FF1200D9CFE6FFDACFE6FFE1CFBE
:10E3F400D9FFE2CFDAFF240EE12402E3E168E6521A
:10E40400E16ED950FA0FE96EFF0EDA20EA6E020EC1
:10E41400EECFDBFF030EEECFDBFF040EEECFDBFF10
:10E42400050EEECFDBFFE8D9F2D968EC77F0006E89
:10E43400060EE15C02E2E16AE552E16E0050E76E2D
:10E444000D0EE7CFDBFFDB50800815E0A0D93E6A54
:10E454003F6A406A416A00C039F001C03AF002C024
:10E464003BF003C03CF038EC6CF0010A10E1210EE3
:10E474000501F16FF26B020EDB68030EDB68040E1C
:10E48400DB687F0EF36E050EF3CFDBFF66D10D0E56
:10E49400DB50050B01E061D10A0EDBCF00F00B0E5F
:10E4A400DBCF01F0830E0026FF0E012200C0DEFF49
:10E4B40001C0DDFFD950060F65D976D9DF50010BB5
:10E4C4000FE0DF06010E01E2DB06D950180F5AD91E
:10E4D400D890EF36010EEB36020EEB36030EEB3618
:10E4E400D9CFE9FFDACFEAFF020E3F6E406AEECFE2
:10E4F4003AF0EDCF3BF012EC6CF03AC0EEFF3BC0CB
:10E50400EDFF140EDB6A150EDB6A160EDB6A170EBE
:10E51400DB6A1C0EDB6A1D0EDB6A1E0EDB6A010E53
:10E52400F36E1F0EF3CFDBFF010EF36E0E0EF3CF6F
:10E53400DBFF0F0EDB6A0E0EDBCF00F00F0EDBCF1E
:10E5440001F0D890015004E61A0E005C000E015848
:10E5540001E398D0180EDBCF00F0190EDBCF01F0E9
:10E564001A0EDBCF02F01B0EDBCF03F0010E1F0BE4
:10E5740007E0D8900036013602360336E806F9E1A2
:10E58400180E00C0DBFF190E01C0DBFF1A0E02C01B
:10E59400DBFF1B0E03C0DBFF140EDBCF08F0150EF0
:10E5A400DBCF09F0160EDBCF0AF0170EDBCF0BF032
:10E5B400010E1F0B07E0D890083609360A360B36D1
:10E5C400E806F9E1D9501C0FDDD80850EE24046E9A
:10E5D4000950EE20056E0A50EE20066E0B50EE2018
:10E5E400076ED950180FCED80450EE5C006E05505B
:10E5F400EE58016E0650EE58026E0750EE58036E48
:10E60400200E00C0DBFF210E01C0DBFF220E02C082
:10E61400DBFF230E03C0DBFF200EDBCF39F0210E1E
:10E62400DBCF3AF0220EDBCF3BF0230EDBCF3CF006
:10E634003C34000E3C1809E6D880000E3954000E14
:10E644003A54000E3B54000E3C5411E2D950200FB2
:10E6540099D8AAD8D8D81C0EDB50EE121D0EDB5068
:10E66400EE121E0EDB50EE121F0EDB50EE12D950CE
:10E674001C0F88D8AFD80E0EDB2A0F0E01E25BD731
:10E68400DB2A59D7C9D8100E00C0DBFF110E01C018
:10E69400DBFF180EDBCF3AF0190EDBCF3BF0120E86
:10E6A4003AC0DBFF130E3BC0DBFFADD893D8D95083
:10E6B400100F68D8EE50ED1012E0D950120F62D846
:10E6C400EE50ED1006E1A8D800500110021003101E
:10E6D40006E099D8EE2A000EEE22EE22EE220C0E6F
:10E6E400DB6A91D8060EEECFDBFF070EEECFDBFF21
:10E6F400080EEECFDBFF090EEECFDBFF7E0EF36ECE
:10E704000A0EF3CFDBFF0B0EDB6AD950020FE66E65
:10E71400000EDA20E66E70D8F6EC77F0E552E5529A
:10E72400E552E552DECFE6FFDDCFE6FF70D8CCEC54
:10E7340076F0006E060EE15C02E2E16AE552E16EFB
:10E744000050020E38C0DBFF030E39C0DBFF040E9D
:10E754003AC0DBFF050E3BC0DBFF19D800C038F020
:10E7640001C039F002C03AF003C03BF0240EE15C72
:10E7740002E2E16AE552E16EE552E5CFDAFFE7CF66
:10E78400D9FF1200E96E000EDA20EA6E1200020EC2
:10E79400DBCF00F0030EDBCF01F0040EDBCF02F081
:10E7A400050EDBCF03F01200180EEECFDBFF190EBF
:10E7B400EECFDBFF1A0EEECFDBFF1B0EEECFDBFF3F
:10E7C4001200EECFE6FFEECFE6FFEECFE6FFEFCF8F
:10E7D400E6FF1200D890030EEB32020EEB32010E6C
:10E7E400EB32EF321200EE500016EE500116EE50EE
:10E7F4000216EE5003161200D950060FE66E000EF4
:10E80400DA20E66E1200D950140FC4EF73F0D95019
:10E81400020FB8DFE3EF73F0010E006E016A026AC3
:10E82400036AF1DFF5EF73F0D9CFE6FFDACFE6FF45
:10E83400E1CFD9FFE2CFDAFFE6520E01006BA96BFC
:10E84400DF6A180EDF5C2AE2EA6ADF34FE0BEA367E
:10E85400E96E010EE9260E0EEA22EE6AED6ADF5039
:10E86400EA6A310FE96E0E0EEA22EF6AEA6ADF34D1
:10E87400FE0BEA36E96E490EE9260E0EEA22EE6A2E
:10E88400ED6AEA6ADF34FE0BEA36E96E790EE926B0
:10E894000E0EEA22EE6AED6ADF2AD3D70E01C60E07
:10E8A400AC6F0E0EAD6F3F0E79140009796ECF0E6A
:10E8B40079140009796E79827B6A7A6A79900F01FA
:10E8C40052815293F00EB4140909B46E0E01080E6D
:10E8D400AA6F030EAB6F800EAE6F3E0EAF6FE00EED
:10E8E400B06F2E0EB16F040EB66F900EB26F010EA4
:10E8F400B36F900EB46F010EB56F000EE66EE66A4C
:10E90400010EE66E93EC21F0E552E552E552E55234
:10E91400E552E5CFDAFFE7CFD9FF1200D9CFE6FF02
:10E92400DACFE6FFE1CFD9FFE2CFDAFFE652DF6AC2
:10E93400180EDF5C0EE2DF50EA6A310FE96E0E0E4C
:10E94400EA22EFCF00F0FD0EDB50005C0EE0DF2A80
:10E95400EFD7DF6A180EDF5C0CE2DF50EA6A310F92
:10E96400E96E0E0EEA22EF5002E1DF2803D0DF2A1F
:10E97400F1D7000EE552E552E5CFDAFFE7CFD9FF34
:10E984001200D9CFE6FFDACFE6FFE1CFD9FFE2CF1D
:10E99400DAFF070EE12402E3E168E652E16EDE6A83
:10E9A400DD6A020EDB6A030EDB6A040EDB6A050E07
:10E9B400DB6A060EDB6A010EE66ED9CFE6FFDACF1C
:10E9C400E6FF030EE66EBCEC55F0E552E552E55267
:10E9D400E552010EE66ED950020FE66E000EDA2003
:10E9E400E66E010EE66EBCEC55F0E552E552E552DA
:10E9F400E552010EE66ED950030FE66E000EDA20E2
:10EA0400E66E030EE66EBCEC55F0E552E552E552B7
:10EA1400E552010EE66ED950050FE66E000EDA20BF
:10EA2400E66E030EE66EBCEC55F0E552E552E55297
:10EA3400E5520701B45124E1020EDB50180802E24A
:10EA4400B48D1ED0050EDBCFE6FF060EDBCFE6FF4E
:10EA5400030EDBCFE6FF040EDBCFE6FF020EDBCFB7
:10EA6400E6FFDECFE6FFDDCFE6FF16D8006E070E29
:10EA7400E15C02E2E16AE552E16E005018EC4CF010
:10EA8400070EE15C02E2E16AE552E16EE552E5CF90
:10EA9400DAFFE7CFD9FF1200D9CFE6FFDACFE6FFDE
:10EAA400E1CFD9FFE2CFDAFFE652E652FB0EDBCF2D
:10EAB400E6FF34DFE552E76E010EE7CFDBFFDB5004
:10EAC40002E1000EB2D0D950FC0FE96EFF0EDA203D
:10EAD400EA6EEE50ED103FE1010EDB04EA6A310FFD
:10EAE400E96E0E0EEA22EF500E01EA6AAC25E96ED9
:10EAF400AD51EA22EF6A010EDB04E96EEA6AD890AE
:10EB0400E936EA36790EE9260E0EEA22EE6AED6A55
:10EB1400010EDB04E96EEA6AD890E936EA36490E5A
:10EB2400E9260E0EEA22EE6AED6A010EDB04EA6AB9
:10EB3400310FE96E0E0EEA22EF6A010EDB04E96E74
:10EB4400EA6AD890E936EA36010EE9260E0EEA2280
:10EB5400EE6AED6A68D0010EDB04006E0E01AA5164
:10EB6400005C61E2FB0EDB5018085DE3FB0EDB503A
:10EB7400070802E10501E36B010EDB04E96EEA6AB2
:10EB8400D890E936EA36010EE9260E0EEA22EE5056
:10EB9400ED1010E1E66AFB0EDBCFE6FF92EC59F0D4
:10EBA400E552E552E66AFB0EDBCFE6FF23EC59F0B3
:10EBB400E552E55205012751FDE00501030E346FCE
:10EBC400F70EDBCF4EF5F80EDBCF4FF5506B516BE4
:10EBD400190E3D6E3E6A3F6A406A4EC538F04FC515
:10EBE40039F050C53AF051C53BF0F5EC79F034C03A
:10EBF4004EF535C04FF536C050F537C051F5010E0E
:10EC0400DBCF55F5FB0EDBCF54F5FC0EDBCF52F515
:10EC1400FD0EDBCF53F5F90EDBCF56F5FA0EDBCF45
:10EC240057F50501276B010EDB50E552E552E5521D
:10EC3400E5CFDAFFE7CFD9FF120005D89BEC5AF0F5
:10EC4400A2EC46F0FBD7D9CFE6FFDACFE6FFE1CF5F
:10EC5400D9FFE2CFDAFFE652E6520F01486949696B
:10EC6400600ED36E9B8C580EDE6E020EDD6EDFCF0F
:10EC740000F0DF06010EDBCF01F001E2DB060050FD
:10EC84000110F5E1948EA0EC45F001EC5AF0E55248
:10EC9400E552E552E5CFDAFFE7CFD9FF12001200C3
:10ECA40012001200120062EF6FF01200B0EF6FF06A
:10ECB4000201A3051EE10201A4051BE1F1DF659237
:10ECC4000201A46B0501100EEF6F0E0EF06FEF073B
:10ECD400000EF05BEF51F011FAE16584080EEF6F5E
:10ECE400070EF06FEF07000EF05BEF51F011FAE141
:10ECF40065941200D9CFE6FFDACFE6FFE1CFD9FF62
:10ED0400E2CFDAFFFC0EDBCF3AF0FD0EDBCF3BF0B7
:10ED1400050E3A1801E13B5036E0E8683A1802E182
:10ED24007F0E3B182FE0030E3A1801E13B5028E018
:10ED3400020E3A1801E13B5021E0010E3A1801E1BC
:10ED44003B501AE0740E3A1801E13B5013E0750E83
:10ED54003A1801E13B500CE0730E3A1801E13B50C4
:10ED640005E0720E3A180FE13B500DD09ADF0BD03C
:10ED740096DF09D095DF07D099DF05D096DF03D061
:10ED840092DF01D08FDF010EE552E5CFDAFFE7CF46
:10ED9400D9FF120096D8E1CFD9FFE2CFDAFF0C0EEB
:10EDA400E12402E3E168E652E16ED950FA0FE96E1C
:10EDB400FF0EDA20EA6E080EEECFDBFF090EEECF6F
:10EDC400DBFF0A0EEECFDBFF0B0EEECFDBFF79D8B5
:10EDD400D950080FE96E000EDA20EA6EEECFE6FF96
:10EDE400EECFE6FFEECFE6FFEFCFE6FF68EC77F07D
:10EDF400006E060EE15C02E2E16AE552E16E00504B
:10EE0400E76E070EE7CFDBFFDB50840B3AE1070E1A
:10EE1400DB041AE1060EDB5006E0006A016A026AAE
:10EE2400800E036E04D0006A016A026A036A080E47
:10EE340000C0DBFF090E01C0DBFF0A0E02C0DBFFCE
:10EE44000B0E03C0DBFF1DD0F80EDBCF00F0F90E74
:10EE5400DBCF01F0D950040FE96E000EDA20EA6E20
:10EE64000050EE260150ED22D950080FE66E000E38
:10EE7400DA20E66E26D8F6EC77F0E552E552E55254
:10EE8400E552080EDBCF00F0090EDBCF01F00A0ECD
:10EE9400DBCF02F00B0EDBCF03F000C038F001C073
:10EEA40039F002C03AF003C03BF00C0EE15C02E220
:10EEB400E16AE552E16EE552E5CFDAFFE7CFD9FF2B
:10EEC4001200D9CFE6FFDACFE6FF1200D9CFE6FF72
:10EED400DACFE6FFE1CFD9FFE2CFDAFFE6520068EE
:10EEE40001687F0E026E036AD950FA0FE96EFF0EB5
:10EEF400DA20EA6EEE500016EE500116EE500216BD
:10EF0400EE5003166AD800C0EEFF01C0EEFF02C047
:10EF1400EEFF03C0EEFFFD0EDB50800B02E0010E9E
:10EF240001D0000EE66E59D8060EE926000EEA223C
:10EF3400E552E750EF6EFC0EDBCF00F0FD0EDBCFA9
:10EF440001F0D89000360136FC0E00C0DBFFFD0E48
:10EF540001C0DBFFDB50E66E40D8040EE926000E4C
:10EF6400EA22E552E750EE6EED6AFD0EDB50006ECC
:10EF7400016AFF0E001818E1015016E12ED8EECFF9
:10EF840000F0EECF01F0EECF02F0EFCF03F000502F
:10EF940001100210031006E0210E0501F16FF26B5F
:10EFA400800E0BD0040E09D0FD0EDB5008E115D8FD
:10EFB400EE6AEE6AEE6AEE6A010EDF6E06D0020EAB
:10EFC400DF6E0BD8EE52EE52EE8EDF50E552E55274
:10EFD400E5CFDAFFE7CFD9FF1200F80EDBCFE9FF68
:10EFE400F90EDBCFEAFF1200D9CFE6FFDACFE6FF56
:10EFF400E1CFD9FFE2CFDAFF5BD8013411E2005050
:10F00400FE08000E01540CE276D805E06CD8800EA0
:10F01400EE6EEE6847D067D8800EEE6E7F0E0ED08F
:10F0240047D8D890015004E6010E005C000E015848
:10F034000BE261D805E057D8EE6A800EEE6E32D04E
:10F0440052D8EE6AEE6A2ED047D8EECF00F0EECF5B
:10F0540001F0EECF02F0EFCF03F032D800C0EEFFA4
:10F0640001C0EEFF02C0EEFF03C0EEFF21D8005046
:10F07400010B05E025D8020E3AD8EF8E04D020D833
:10F08400020E35D8EF9E14D8D8900132003218D829
:10F09400030E2DD800C0EFFF1AD804E011D8030ED8
:10F0A40026D8EF8EE552E5CFDAFFE7CFD9FF12007D
:10F0B40013D8040E1CD8EECF00F0EFCF01F01200ED
:10F0C400FA0EDBCFE9FFFB0EDBCFEAFF120004D818
:10F0D400060E0DD8EF501200FC0EDBCFE9FFFD0E3B
:10F0E400DBCFEAFF1200ECDFEE6AEE6A1200E926DB
:10F0F400000EEA221200220E0501F16FF26B69EF95
:10F1040078F02A0EF66E100EF76E000EF86E0501FA
:10F114000900F550EA6F0900F550EB6F03E1EA6767
:10F1240001D03DD00900F550E56F0900F550E66FB8
:10F134000900F550E76F09000900F550E96E090070
:10F14400F550EA6E090009000900F550E86F09005E
:10F15400F550E96F09000900F6CFECF5F7CFEDF5AE
:10F16400F8CFEEF5E5C5F6FFE6C5F7FFE7C5F8FF0E
:10F174000501E85302E1E95307E00900F550EE6E9A
:10F18400E807F8E2E907F9D7ECC5F6FFEDC5F7FFA4
:10F19400EEC5F8FF0501EA07000EEB5BBFD71200CE
:10F1A400FE0EE3CFE9FFFF0EE3CFEAFFE9CFF3FF63
:10F1B400EACFF4FFFB0EE35003E1FC0EE35009E059
:10F1C400FB0EE30602E2FC0EE306FD0EE350EE6ED8
:10F1D400F1D71200FE0EE3CFE9FFFF0EE3CFEAFF03
:10F1E400F36AF46AEE5203E0F34AF42AFBD71200FE
:10F1F400FF0EE3CFF8FFE552FF0EE3CFF7FFE55232
:10F20400FF0EE3CFF6FFE552E66AE66AE66A090016
:10F21400F55209E0FD0EE32A05E1FE0EE32A02E1C0
:10F22400FF0EE32AF4D7FD0EE3CF39F0FE0EE3CF51
:10F234003AF0FF0EE3CF3BF01200D9CFE6FFDACF6E
:10F24400E6FFE1CFD9FFE2CFDAFFE652E652E6521B
:10F25400E652D950FB0F006EFF0EDA20016E00C09B
:10F26400DEFFDD6EDECFE6FFDDCFE6FFFB0EDBCF9C
:10F27400E6FFFC0EDBCFE6FFFD0EDBCFE6FFF3C5BA
:10F28400E6FFF4C5E6FFD3EC63F0006E070EE15C25
:10F2940002E2E16AE552E16E0050020EF3CFDBFFB9
:10F2A400030EF4CFDBFF020EDBCF00F0030EDBCF47
:10F2B40001F000C0F3FF01C0F4FF040EE15C02E2C0
:10F2C400E16AE552E16EE552E5CFDAFFE7CFD9FF17
:10F2D40012001201000202000040D80492FD8201D3
:10F2E4000102000109024300020100C032090400C6
:10F2F4000001020201000524001001042402020599
:10F304002406000105240100010705810308000209
:10F3140009040100020A000000070502024000007F
:10F324000705820240000004030904180353006324
:10F334000068006D0061006C007A0048006100758F
:10F3440000730016034500690042006F0074004218
:10F35400006F00610072006400E8F22BF32FF347A2
:01F36400F3B5
:10F36600D9CFE6FFDACFE6FFE1CFD9FFE2CFDAFF6A
:10F37600FB0EDBCF00F0FC0EDBCF01F00001800EB0
:10F3860001141AE1FB0EDBCFE9FFFC0EDBCFEAFF2F
:10F39600EECFF3FFEDCFF4FFEE2A000EEF22F3CF10
:10F3A600E9FFF4CFEAFFFD0EDBCFEFFFEF50016A76
:10F3B600F36E01C0F4FF10D0FB0EDB50FE0806E131
:10F3C600FD0EDBCFE6FFC6EC7AF005D0FD0EDBCFF7
:10F3D600E6FFAEEC48F0E552E552E5CFDAFFE7CFBF
:10F3E600D9FF120038503D02F3CF34F0F4CF35F098
:10F3F6003E02F3503526000EF420366E38503F029A
:10F40600F3503626000EF420376E38504002F35083
:10F41600372639503D02F3503526F4503622000E79
:10F42600372239503E02F3503626F45037223950EF
:10F436003F02F35037263A503D02F3503626F45039
:10F4460037223A503E02F35037263B503D02F350E6
:10F4560037261200FF0EE124E96EFF0EE220EA6E67
:10F46600EDCFF4FFEFCFF3FFF46607D0600EF36441
:10F4760004D07B0EF36001D0F39A1200F36AF46AAB
:10F48600FF0EE124E96EFF0EE220EA6EED6607D07C
:10F496002F0EEF6404D03A0EEF6001D0F32A12006B
:10F4A600376A366A356A346A200EE76ED89038367F
:10F4B60039363A363B3634363536363637363D50BB
:10F4C600345C3E5035583F5036584050375809E363
:10F4D6003D50345E3E50355A3F50365A4050375AAA
:10F4E600382AE72EE4D712004F4B0D0A000D0A000A
:10F4F6004542427631335F616E645F61626F766565
:10F50600204542204669726D7761726520566572A4
:0DF5160073696F6E20322E352E330D0A0002
:10F52400376A366A100EE76ED8903A363B3636366E
:10F5340037363F50365C4050375805E33F50365E0F
:10F544004050375A3A2AE72EF0D71200C00EF36E15
:10F5540000EE00F00E0E01D81200EA6002D0EE6A4E
:10F56400FCD7F350E9601200EE6AFCD71DEE00F000
:10F574002DEE00F0F86A439C83EC78F0E8EC7AF026
:10F584001FEC76F0FBD71200FF0EE350ADBA04D0A7
:10F59400B06AAC8EAD8A949CADA2FED7AE6EF36E0B
:10F5A400F46A1200F36AF46AF32A0F0B05E0D890A8
:10F5B400F336F436E804FBE11200303132333435EB
:0BF5C400363738396162636465660009
:10F5D0001200FEFF0000000000000000010000001B
:10F5E000000000000000000000000000000000001B
:10F5F000000000000000000000000000000000000B
:10F6000000000000000000000000000000000000FA
:10F6100000000000000000000000000000000000EA
:10F6200000000000000000000000000000000000DA
:10F6300000000000000000000000000000000000CA
:10F6400000920F920F920F930F930F930F930F93BC
:10F650000F930F930F930F940F940F940F940F9495
:10F660000F940F940F940F950F950F950F950F957D
:10F670000F950F890F890F890F8A0F8A0F8A0F8ABA
:10F680000F8A0F8A0F8A0F8A0F8B0F8B0F8B0F8BAE
:10F690000F8B0F8B0F8B0F8B0F8C0F8C0F8C0F8C96
:10F6A0000F8C0F8C0F0001050001020304050607F3
:0EF6B000000102030405060702030405060715
:08FFF800ACF70AFF63F801F009
:00000001FF
